:020000040000fa
:08000000ba0704000000000033
:020000040000fa
:020000040005f5
:045fe000dfff0000df
:020000040000fa
:020000040005f5
:045fe400ffff0000bb
:020000040000fa
:020000040005f5
:045fe80078ff00003e
:020000040000fa
:020000040005f5
:045fec007dff000035
:020000040000fa
:020000040005f5
:045ff00078ff000036
:020000040000fa
:1000080000000000000000000000000000000000e8
:10001800b20700000000000000000000000000001f
:100028000e0c00000000000000000000460c00005c
:1000380000000000000000000000000000000000b8
:10004800a00c00000000000000000000d40d00001b
:100058000000000000000000000000000000000098
:100068000000000000000000000000000000000088
:100078000000000000000000000000000000000078
:10008800000000000000000000000000ee0c00006e
:10009800a40d0000000000000000000000000000a7
:1000a8000000000000000000000000000000000048
:1000b8000000000000000000000000000000000038
:1000c8000000000000000000000000000000000028
:1000d8000000000000000000000000000000000018
:1000e8000000000000000000000000000000000008
:1000f80000000000000000000000000000000000f8
:1001080000000000000000000000000000000000e7
:1001180000000000000000000000000000000000d7
:10012800000000000c0e00000000000000000000ad
:1001380000000000000000000000000000000000b7
:1001480000000000000000000000000000000000a7
:100158000000000000000000000000000000000097
:100168000000000000000000000000000000000087
:100178000000000000000000000000000000000077
:100188000000000000000000000000000000000067
:100198000000000000000000400e00006c0e00008f
:1001a800980e0000000000000000000000000000a1
:1001b8000000000000000000000000000000000037
:1001c8000000000000000000000000000000000027
:1001d8000000000000000000000000000000000017
:1001e8000000000000000000000000000000000007
:1001f80000000000000000000000000000000000f7
:1002080000000000000000000000000000000000e6
:1002180000000000000000000000000000000000d6
:1002280000000000000000000000000000000000c6
:1002380000000000000000000000000000000000b6
:1002480000000000000000000000000000000000a6
:100258000000000000000000000000000000000096
:100268000000000000000000000000000000000086
:0c0278000000000000000000000000007a
:020000040000fa
:10040000f9d1bf00f851b7004220af00f871ec00fd
:10041000f9d1d600f9d1b60000c0d200f9d1bf00a1
:1004200000c0fd00f9f1b700f8d1bf0000c0fd0029
:100430000040d200f9d1b600f9d1bf0000c0fd00e4
:10044000f9f1b7001040b200f8f1d600f8f1b600ab
:10045000f9f1d600c08f800000000600803e200029
:10046000030007008100e900fcff3a0000000600dd
:10047000831f7800c20320000400bc006601510005
:10048000e0815900f23fb1000380b1000600350061
:10049000ee03090000000000423fb1000380b100fc
:1004a000fbff3d001200b000223fb000020035000b
:1004b0000280090000000000cf0178000000060063
:1004c000839f68000100e00002003d006000100012
:1004d000e08018000300e00002003d006001110010
:1004e000e0811900050007004f00e00002003b001a
:1004f00060001000e080180000000600861f7800f1
:100500006022b800060220000000d0008180d200e6
:100510000482d2008582d2000000a00002025200b4
:1005200083825a00030031000202420083824a00a3
:100530000000a1000603e900f3ff3a004f03780032
:10054000000006000001eb00869fbe00889fbe00f1
:100550008a9fbe008c9fbe00820578000004be000a
:10056000340207000800be006420e10007003900e3
:1005700002003a00f1ff2f00f0ff27000160a00009
:100580001202200012908800560037006120e1001e
:1005900003003a000b00a70001f8230051003700c8
:1005a00001f0a10002002100936424005200070022
:1005b0000800be0005003500b2fd2000930c2400a9
:1005c00004002000690007000004be000005eb00e5
:1005d0000b00a6004f0dde0001f0a1000004be00dc
:1005e00032982f0023ea2300620107000001eb008c
:1005f000030020000b00a70003f82300bc00070045
:10060000910107000000a7000a00a200d401070022
:100610000b00e000030032000200200003f0230082
:10062000b200070001f0a2000006be000200200098
:10063000930424004f0107000801be00ac0007002e
:10064000809fbe000c00be0022a22a00d3a7230078
:10065000480107004f01be00a50007000004be00ce
:1006600001f0a100020020000398230022000700ef
:100670000800be00190035000001be003d01070062
:100680000006be00b2c52900e3622300390107005d
:1006900022222b00f3942b00950007000c01be00d2
:1006a00034010700e273280083c023009000070094
:1006b0000c01be002f01070042aa2a00a3e22b0072
:1006c0008b0007000c01be002a0107000801be00d4
:1006d000280107000801be00850007000a00a700e6
:1006e00001f0a2004f06be004f05be004f04be0041
:1006f0004f03be000000060014002000889fbe00cb
:100700008a9fbe00841f7800c20107004f00780056
:1007100011003300f0ff2f00838f6c0006003b00b8
:10072000040565000a00a7000800370009f0a600cc
:100730001000200008003700820f5400838f5c00f7
:10074000030039001000200001003e0000002000de
:1007500009f0a7000000ea004f05be004f04be00ec
:100760000000e0000000060014002000869fbe008c
:10077000889fbe008a9fbe008c9fbe004f26dd0072
:10078000a4010700e60133006120e10043003200cc
:100790006250e10041003e003e0039006420e1006b
:1007a0003c003200058255000f003b000402e800c7
:1007b00038003a00800f5300818f5b003500340011
:1007c0000800be0003f0a10001f0a60003f0a000a5
:1007d0000cf0a70046000700da01370006034300cb
:1007e00087834b000c4646000005530081855b0063
:1007f000020033000a03be000c00a0000402e9005e
:10080000f6ff3b00850578000602430087824b0017
:1008100004003a006000b80009f0a70001f0a00051
:10082000c80137000002520081825a000704e0002c
:10083000040033000603430087834b008b05e90067
:10084000faff3700090578000604be000203be0067
:100850006011b8008c010700e00f5200e08f5a00d1
:100860000700350002003c000c08a3000400320021
:100870000601be0003f0a0000cf0a7001c0007005a
:100880000a85680001f0a1000af0a70001f0a000ad
:10089000ac0137000800be00aa013700100220009a
:1008a0000cf0a60010908800ab0137000002be00db
:1008b000e00f5000e08f58000200350028010700cb
:1008c000000006000401be0061006100010020007c
:1008d0008301d1000281d300020070008380700088
:1008e0001f0107000001be000100370003f0a20055
:1008f000869fbe00889fbe008a9fbe008c9fbe0060
:1009000044010700860133006450e1004f003200cb
:100910006420e1005200320003826c0007003b00bb
:100920000905d0000306d000820f54000c065d00bc
:1009300002003900020032008901780003067800c5
:100940008582550004003d000003fd008103fd0089
:100950008502ea008b854200840f720002003b0092
:1009600060001000e08018006011b8000005eb0086
:100970007a28e1000a00390006007800c75ddd0032
:10098000f707b200878075002d0037008281710063
:100990000a017800610560008180d1000080d300e9
:1009a0008502e900f9ff3b00060440008784480007
:1009b00002003b0060041400e0841c000988a300ce
:1009c000070032008a817100828171006101640038
:1009d0008904d1000884d3008b05e8001700370094
:1009e0000978a30013003a000b00e0001300340064
:1009f0008b05e9000804440089844c000a44740013
:100a00000978a3000d003a000b00e0000700340055
:100a10008b05e9000804440089844c0001003a0079
:100a20000b0020000978a300f7ff32000001eb0063
:100a300002003700828171000a017800120107006c
:100a40000cf0a70001f0a0003e0137006420e10097
:100a500002003a00838f6c003f0133000801be00a2
:100a60000200be0037013700869fbe00889fbe008f
:100a70008a9fbe008c9fbe00e6000700280133005d
:100a800003866c006450e1002e0032006420e10017
:100a9000330032006150e1002f0032006120e1009c
:100aa0003100320085855500eb07b00009002000b9
:100ab00008042000050037000804440089844c0025
:100ac0000a0031000603430087834b0000015300f6
:100ad00081815b00f8ff33000203be000800a00024
:100ae0000804440089844c00f6ff3900c639dd0053
:100af0008301730001003200130020008904d1003b
:100b00000884d3000998a300050032000800a7005c
:100b10000300a0008904d1000884d3008b05e800fd
:100b20008904d1000884d3000001eb000281d200c7
:100b3000d500070001f0a1000cf0a70001f0a00013
:100b4000000137006420e100030132000801be000b
:100b50000200be00f7ff37006120e100fe00320016
:100b60006000b800f3ff37000000200001f8270004
:100b7000f0ff3700869fbe00889fbe008a9fbe00a0
:100b80008c9fbe00a3000700e500330003866c00c5
:100b90006450e100240032006420e10027003200ac
:100ba0006150e100220032006120e10021003200aa
:100bb0008b854200eb07b1000134b800003ab80061
:100bc0000804420089844a00013ab8000030b800a5
:100bd0008880400009014a00040033000000400002
:100be00081804800020149008b05e900c909dd0048
:100bf000830170000100320013002000c814de00e1
:100c00004814dd004709de001200b200c808de000b
:100c1000088470009c00070001f0a1000cf0a70000
:100c200001f0a000c70037006120e100ca003200d7
:100c30000801be000200be00f7ff37006150e1006e
:100c4000fcff3a00c4003700829fbe000001be00d6
:100c5000780007000470a70003f0a1006509b10047
:100c6000180032000e0035006828e100070035004a
:100c7000f0ff2f00f1ff27000300e00015003b000c
:100c8000010028004f01be000000050000004000e8
:100c9000818048008502e900fcff3a000900370026
:100ca000f88f420003003c008000eb004f01be00c3
:100cb000000005008100d1000080d3008502e8001b
:100cc000fcff3a000300e00002003b00600010005f
:100cd000e08018004f01be0000000600829fbe00a9
:100ce0000001be00530007000470a70003f0a1003c
:100cf00003f8a30015003a006509b10011003200a5
:100d00000a0035006928e1000300350001002800d1
:100d10004f01be0000000500000040008180480037
:100d20008502e900fcff3a0006003700f88f420018
:100d3000060035008100d1000080d3008502e80064
:100d4000fcff3a004f01be00000006008000eb00ef
:100d50004f01be00000005000080fb008000eb009a
:100d6000829fbe00889fbe008a9fbe00010578005a
:100d70000100e0000400350008003c000000e00035
:100d8000200032000500370060001000e0801800ed
:100d900002003b0001f024001a0037000004be00ee
:100da0006011b8006b0920000982cf0002003900f1
:100db0000882cf000441b000694252000e003200a8
:100dc00008003b0082817100610164008904d10048
:100dd0000884d3008b05e8000442e800f9ff3a00dc
:100de000050037000804440089844c008b05e900a5
:100df0000442e900fbff3a00230007000af0a700c5
:100e000001f0a0004f05be004f04be004f01be0020
:100e1000000006000004be00060007000003be003c
:100e20000405be000200be0002000700844f7500ea
:100e300000000600c70ade00f107b200f50fb2009d
:100e400008003200e1cf4200020032000170a00031
:100e500024000500810f7000010032000408050025
:100e600044000500810f700002003a0014000500e4
:100e70008502e9000000400081c04800fcff3b0003
:100e80000170a00024000500810020006180550051
:100e90000b003d000b00200061fe2f000100e1006f
:100ea0001d00340082817100610164008904d10059
:100eb0000884d3000000e800faff3a007100200027
:100ec000610064000300700002006000090032004d
:100ed00061044400e0844c000988a500050032004c
:100ee0008b05e8006808e10002003a008904d1009f
:100ef0000884d300f20f20000258e10005003d00f5
:100f0000c75ddd00f907b200898075000800780030
:100f1000000006000bf827008b0078000000050099
:100f20000200be006450e100050036006420e100cc
:100f3000020036000968a30001003a000800be0064
:100f40000160a0004f06be004f05be004f04be006a
:100f50004f03be0000000600f0ff2f00f1ff270046
:100f6000f8ff37000020ef000220ef00c088a90042
:100f7000004006000f002100202b21000001880006
:100f8000000000000000eb00000778000c000900e2
:100f9000002f78000007eb005420ef000e2eef002a
:100fa0001e2eef0040a7a900a10020002bfd070086
:100fb000e0022000303a880044e7a90044c7a900b5
:100fc0004407a9004427a9004447a9004467a90091
:100fd0004487a9000700fc00300020003174200085
:100fe00082072000a3092000824878008348780007
:100ff000804878000700fc00113a80006180700092
:1010000021742000620420007305200082487800cb
:1010100083487800804878004427ef00e0022000f1
:10102000303a88000e00fc003000200031742000af
:1010300082072000a30920008248780083487800b6
:101040008048780000002000217420006204200005
:101050007305200082487800834878008048780033
:1010600042a7ae00feff3700813e2000fbfc0700d8
:1010700010c0b30086e6b70090c2b300c4e6b70064
:101080000002200000708800007825008070880031
:1010900010aea90010cea9004008a9004028a90060
:1010a0004048a8002008a8000008a900c208a8001d
:1010b00080c0b300c8e8b7004188a90041a8a800d3
:1010c00041c8a800000820001008880004a1a90059
:1010d0000481a90005e1a8000068a90011e1a900a8
:1010e00013e1a9001061a8001021a90011a1a90015
:1010f00010a1a8001081a8000821ef000621ef0030
:101100000c21ef0020002000700888004408a9008e
:101110004428a8004448a9000108a9002108a80003
:101120001fe1a8001fa1a9001ec1a9001ea1a800bf
:101130001e81a9001e61a9001e21a9001421ef0033
:1011400050412100d00888004d88a8004da8a80073
:101150004dc8a9000368a9002368a80021e1a800e0
:1011600021a1a90020c1a90020a1a8002081a800d8
:101170002021a9001821ef004e08a8004e28a90040
:101180004e48a9000388a9001ca1ef002388a800ed
:1011900021e1a8002002a9002022a9002042a900e4
:1011a00020a2a9002062a9002082a90020e2a900b3
:1011b0002102a9002122a900700720004011880007
:1011c00022a2a90022c2a90022e2a90021e2a800cd
:1011d0002182a9004588a80045a8a90045c8a80003
:1011e0002168a8002828a8002bc8a9002be8a9007e
:1011f0002c08a9000bc8a9000be8a9000c08a9003d
:1012000001eca90001aca900016ca900014ca800e7
:10121000012ca900010ca90000eca900008ca90078
:1012200000aca90000cca900000ca900002ca9006a
:10123000004ca900006ca900202cef00402cef000e
:10124000602cef0020eca800200ca80040eca800c7
:10125000400ca80060eca800600ca800f07f200003
:1012600020608800020ca900022ca900024ca900f1
:101270000040200030618800462cef00662cef0013
:10128000282cef00482cef00682cef000aacef0090
:1012900023eca80023cca80043eca80043cca90071
:1012a00063eca80063cca90023aca900238ca9009f
:1012b000dabc2a001b32240030002c00fa608800bf
:1012c000fb60880020618800dabc2a001b32240001
:1012d00020002c00fa608800fb6088001061880004
:1012e000dabc2a001b32240030002c00fa6088008f
:1012f000fb60880020628800dabc2a001b322400d0
:1013000000002800fa608800fb60880010628800f6
:10131000dabc2a001b32240030002c00fa6088005e
:10132000fb60880020638800dabc2a001b3224009e
:1013300000002800fa608800fb60880010638800c5
:10134000a70037003f003700002020000061880020
:101350000020200000628800002020000063880038
:10136000020ca900022ca800024ca80004acef005b
:1013700028acef0048acef0068acef00262cef0083
:10138000462cef00662cef000aacef0023eca8001f
:1013900023cca90043eca80043cca90063eca8002f
:1013a00063cca900dabc2a001b32240030002c00d8
:1013b000fa608800fb60880020618800dabc2a009f
:1013c0001b32240000002800fa608800fb608800bf
:1013d00010618800dabc2a001b32240030002c0087
:1013e000fa608800fb60880020628800dabc2a006e
:1013f0001b32240000002800fa608800fb6088008f
:1014000010628800dabc2a001b32240030002c0055
:10141000fa608800fb60880020638800dabc2a003c
:101420001b32240000002800fa608800fb6088005e
:101430001063880011eea90011aea900116ea90079
:101440006700370035003700001020000061880079
:101450000010200000628800001020000063880057
:10146000020ca900022ca800024ca8000a2cef00d4
:1014700004acef00282cef00505525004062880096
:10148000a0aa2a0040638800dabc2a001b3224008c
:1014900030002c00fa608800fb6088002061880022
:1014a000dabc2a001b32240000002c00fa608800fd
:1014b000fb60880010618800dabc2a001b3224001f
:1014c00030002c00fa608800fb60880020628800f1
:1014d000dabc2a001b32240000002c00fa608800cd
:1014e000fb60880010628800dabc2a001b322400ee
:1014f00030002c00fa608800fb60880020638800c0
:10150000dabc2a001b32240000002c00fa6088009c
:10151000fb6088001063880031003700300037001e
:101520000010200000618800001020000062880088
:10153000020ca900022ca800024ca8000a2cef0003
:1015400004acef00282cef0000002400406288006b
:10155000dabc2a001b32240030002c00fa6088001c
:10156000fb60880020618800dabc2a001b3224005e
:1015700000002c00fa608800fb6088001061880081
:10158000dabc2a001b32240030002c00fa608800ec
:10159000fb60880020628800dabc2a001b3224002d
:1015a00000002c00fa608800fb6088001062880050
:1015b000dabc2a001b32240030002c00fa608800bc
:1015c000fb60880020638800dabc2a001b322400fc
:1015d00000002c00fa608800fb608800106388001f
:1015e000218ca900418ca900618ca900216ca90063
:1015f000416ca900616ca900214ca900414ca900d3
:10160000614ca90020eca80040eca80060eca80008
:101610003e2cef005e2cef007e2cef0001eca800ca
:10162000404b210040918800200b220050918800ff
:10163000400b220060918800204b220070918800ae
:10164000404b220080918800206b220090918800fe
:10165000406b2200a091880020ab2200b09188004e
:1016600040ab2200c0918800202b2300d09188003d
:10167000402b2300e0918800206b2300f09188002c
:10168000406b23000092880020ab2300109288005a
:1016900040ab23002092880020eb2300309288008a
:1016a00040eb230040928800202b240050928800b9
:1016b000402b240060928800204b24007092880008
:1016c000404b240080928800208b24009092880058
:1016d000404b2200a0928800206b2200b09288002c
:1016e000404b2200c0928800206b2200d0928800dc
:1016f000404b2200e0928800206b2200f09288008c
:10170000404b220000938800206b22001093880039
:10171000c092800000918800d092800010918800d3
:10172000a0928000c0908800b0928000d090880085
:10173000e0928000e0908800f0928000f0908800b5
:1017400000938000209188001093800030918800e1
:1017500040ab2400b093880040bb2400c0938800b5
:1017600040cb2400d093880040db2400e093880025
:1017700040eb2400f093880040fb24000094880094
:10178000400b250010948800a0c2b300b0f2b7004f
:1017900030c2b300b1f2b70080c2b300b2f2b700fa
:1017a0000000eb00419b2600ff00090080587800f4
:1017b0009172ef009272ef00c70607000c32ef0043
:1017c000a1f2ef00984b070018560700fb0707002f
:1017d00055140700551a07009c1a07009c200700a3
:1017e0009c2c07009c3207009c3807009c3e070099
:1017f0009d4a07009b4407000d7a07004c3b2100df
:1018000040ab24007f000900301e78006f4b0700ba
:10181000b2070700837a07005b013700ff3ffc0037
:101820004200f8003600f8004400f8008e1f7800ef
:101830000e0020000d000900be1f78003200f800e5
:101840000100fc000008a9002068a9000068a900a8
:1018500000402000306188002108a900a512a900dd
:10186000ff3ffc003200f900ae0120000d0009002e
:101870004f1778004f0778004400f9003600f90050
:101880004200f9000100fc0000400600ff3ffc00a0
:101890004200f8003600f8004400f8008e1f78007f
:1018a0000e0020000d000900be1f78003200f80075
:1018b0000100fc000068a900809380006412b4005d
:1018c00010088800b2908000120078003061880013
:1018d00016b2ec001012ae000800370050918000e4
:1018e000b1908000808f5000030036001012a900d4
:1018f00090908000b090880006003700a090800093
:10190000b1908000808f50000200360090908000df
:10191000b0908800ff3ffc003200f900ae012000cb
:101920000d0009004f1778004f0778004400f900b8
:101930003600f9004200f9000100fc0000400600fa
:10194000ff3ffc004200f8003600f8004400f800b9
:101950008e1f78000e0020000d000900be1f7800c9
:101960003200f8000100fc000108a90011e1a90003
:10197000a752e2000a003600a512a800a8d2bf00b4
:101980000080fb0000004000412b210060807800b7
:10199000d00888002368a8001fe1a80001003700d4
:1019a000a512a9002108a900020eaa00000ea90094
:1019b000ff3ffc003200f900ae0120000d000900dd
:1019c0004f1778004f0778004400f9003600f900ff
:1019d0004200f9000100fc0000400600ff3ffc004f
:1019e0004200f8003600f8004400f8008e1f78002e
:1019f0000e0020000d000900be1f78003200f80024
:101a0000f411f800f611f8000100fc000368a900c9
:101a1000a8d2bf000080fb0000004000412b210045
:101a200060807800d0088800a512ae00270037003b
:101a3000a972ec00f0c1b300a972b600a9d2bf0030
:101a40000080fb0041ab260060c07800f4f1b700d5
:101a5000411f2100914078008100fb00a7d2bf0008
:101a60000000fb000088b90030938800a4d2bf00ba
:101a70000080fb0000004000418b24006080780063
:101a8000cf80de000001be0030938000cf80de00fa
:101a9000020ab800800278000200b800810042000b
:101aa000032ab80081004200609488007194880085
:101ab00002fe2000030020006094800071948000ea
:101ac0007ffa07004093880006003700a972ef00f4
:101ad0006812e200010034006832ed0069f2af00e4
:101ae0006832ec00a4d2bf000080fb000000400080
:101af000413b210060807800a08f880040938000e7
:101b0000f411b400b08f880060908000f611b4002a
:101b100020938800ff3ffc00f611f900f411f90052
:101b20003200f900ae0120000d0009004f177800c7
:101b30004f0778004400f9003600f9004200f90030
:101b40000100fc0000400600ff3ffc004200f800de
:101b50003600f8004400f8008e1f78000e002000c8
:101b60000d000900be1f78003200f8000100fc00e3
:101b70000388a900128eaa00108ea900ff3ffc0066
:101b80003200f900ae0120000d0009004f17780067
:101b90004f0778004400f9003600f9004200f900d0
:101ba0000100fc0000400600ff3ffc004200f8007e
:101bb0003600f8004400f8008e1f78000e00200068
:101bc0000d000900be1f78003200f8000100fc0083
:101bd0000168a9009172ec0091d2bf008080fb00e7
:101be00030118000429b260080707900ff3ffc008e
:101bf0003200f900ae0120000d0009004f177800f7
:101c00004f0778004400f9003600f9004200f9005f
:101c10000100fc0000400600ff3ffc004200f8000d
:101c20003600f8004400f8008e1f78000e002000f7
:101c30000d000900be1f78003200f8000100fc0012
:101c40000828a9002242ae00000037002222af007f
:101c50002222a900ff3ffc003200f900ae01200063
:101c60000d0009004f1778004f0778004400f90075
:101c70003600f9004200f9000100fc0000400600b7
:101c8000ff3ffc004200f8003600f8004400f80076
:101c90008e1f78000e0020000d000900be1f780086
:101ca0003200f8000100fc000bc8a900ff3ffc0057
:101cb0003200f900ae0120000d0009004f17780036
:101cc0004f0778004400f9003600f9004200f9009f
:101cd0000100fc0000400600ff3ffc004200f8004d
:101ce0003600f8004400f8008e1f78000e00200037
:101cf0000d000900be1f78003200f8000100fc0052
:101d00000be8a900ff3ffc003200f900ae01200003
:101d10000d0009004f1778004f0778004400f900c4
:101d20003600f9004200f9000100fc000040060006
:101d3000ff3ffc004200f8003600f8004400f800c5
:101d40008e1f78000e0020000d000900be1f7800d5
:101d50003200f8000100fc000c08a900ff3ffc0065
:101d60003200f900ae0120000d0009004f17780085
:101d70004f0778004400f9003600f9004200f900ee
:101d80000100fc00004006000a790700b3d2bf0042
:101d900093f2b70070ceb3009352b500060039003d
:101da000e0cfb3009352b5000100390001003700c5
:101db0009472ef007401370093f2ae0037003700e1
:101dc0009472ef0060c8b3009352e30005003a003c
:101dd00093d2bf0094f2b70095f2ef0096f2ef00b5
:101de0002d00370060c9b3009352e30005003a00ac
:101df00093d2bf0094f2b70097f2ef0098f2ef0091
:101e00002500370060cab3009352e30005003a0092
:101e100093d2bf0094f2b70099f2ef009af2ef006c
:101e20001d00370060cbb3009352e30005003a0079
:101e300093d2bf0094f2b7009bf2ef009cf2ef0048
:101e40001500370060ccb3009352e30004003a0061
:101e500093d2bf0094f2b7009df2ef000e0037005e
:101e600060cdb3009352e30004003a0093d2bf0068
:101e700094f2b7009ef2ef000700370060ceb30087
:101e80009352e30004003a0093d2bf0094f2b700eb
:101e90009ff2ef00a0f2ef003b0137009452e20006
:101ea00002003a00380137003701370060c8b3003c
:101eb0009452e30010003a0000e0ef009552e30076
:101ec00003003a0093d2bf0095f2b7000900370033
:101ed0009352ec0096f2b70095d2bf00a452b50021
:101ee00003003a00a512a9002108a90011e1a900e8
:101ef00095f2ef002401370060c9b3009452e3006b
:101f0000e5003a0000e0ef009752e30003003a00da
:101f100093d2bf0097f2b700de00370093d2bf0024
:101f200098f2b70097d2bf0041c3b30080cf100032
:101f30003300360010c4b3009752e30030003e0077
:101f40002068a90097d2bf000080fb00000040007d
:101f5000413b21006080780020938800209380001e
:101f600010088800aa52e20008003600aad2bf007a
:101f70000081fb00209380000200e000020032009c
:101f8000110009000280d80090938800909380008f
:101f9000a09388007432d500a092800090908800b1
:101fa000b0928000a0908800a612af000400370015
:101fb00040918000b09088001012a8000300370004
:101fc00090908000b09088001012a9000068a900cd
:101fd0002068a80097d2bf00a4f2b700a752e20081
:101fe000050036000821ef000621ef0011e1a800ee
:101ff0002108a800a972ef00a512a900a4003700cb
:1020000097d2bf0011c4b30080cf10003300360058
:1020100090c4b3009752e30030003e002068a9004e
:1020200097d2bf000080fb0000004000413b210030
:10203000608078002093880020938000100888003a
:10204000aa52e20008003600aad2bf000081fb00bd
:10205000209380000200e00002003200110009001d
:102060000280d8009093880090938000a09388000d
:102070007432d500c092800090908800d092800089
:10208000a0908800a612af000400370040918000a5
:10209000b09088001012a8000300370090908000d4
:1020a000b09088001012a9000068a9002068a8005c
:1020b00097d2bf00a4f2b700a752e2000500360095
:1020c0000821ef000621ef0011e1a8002108a80077
:1020d000a972ef00a512a9006d00370097d2bf00ca
:1020e00091c4b30080cf10003300360080c5b30028
:1020f0009752e30030003e002068a90097d2bf004d
:102100000080fb0000004000413b2100608078001f
:10211000209388002093800010088800aa52e200d3
:1021200008003600aad2bf000081fb002093800087
:102130000200e00002003200110009000280d80015
:102140009093880090938000a09388007432d5000b
:10215000e092800090908800f0928000a09088002b
:10216000a612af000400370040918000b0908800b4
:102170001012a8000300370090908000b0908800f3
:102180001012a9000068a9002068a80097d2bf001b
:10219000a4f2b700a752e200050036000821ef00c4
:1021a0000621ef0011e1a8002108a800a972ef00a4
:1021b000a512a9003600370097d2bf0081c5b30031
:1021c00080cf100032003600a0c6b3009752e30063
:1021d0002f003e002068a90097d2bf000080fb00be
:1021e00000004000413b210060807800209388007f
:1021f0002093800010088800aa52e20008003600f0
:10220000aad2bf000081fb00209380000200e00002
:1022100002003200110009000280d800909388006b
:1022200090938000a09388007432d50000938000c2
:102230009090880010938000a0908800a612af00b4
:102240000400370040918000b09088001012a80070
:102250000300370090908000b09088001012a90011
:102260000068a9002068a80097d2bf00a4f2b700b8
:10227000a752e200050036000821ef000621ef001a
:1022800011e1a8002108a800a972ef00a512a90079
:1022900097f2ef003c00370060cab3009452e300ad
:1022a0000a003a0000e0ef009952e30003003a0010
:1022b00093d2bf0099f2b7000300370093d2bf005a
:1022c0009af2b7003d0007002f00370060cbb30043
:1022d0009452e3000a003a0000e0ef009b52e30052
:1022e00003003a0093d2bf009bf2b700030037000f
:1022f00093d2bf009cf2b700ad0007002200370068
:1023000060ccb3009452e30009003a0000e0ef0013
:102310009d52e30004003a0093d2bf009df2b70043
:1023200028000700010037009df2ef00160037007b
:1023300060cdb3009452e30007003a0000e0ef00e4
:102340009e52e30003003a0093d2bf009ef2b70012
:10235000950007000c00370060ceb3009452e300f4
:1023600009003a0000e0ef009f52e30003003a004a
:1023700093d2bf009ff2b7000300370093d2bf0093
:10238000a0f2b70011000700aa52e20002003a00d2
:102390007032ef000800370019f80700a08f88009e
:1023a00090938000f411b6007093880070938000c1
:1023b0007412b5008093880073fe370099f2ef0025
:1023c000000006009df2ef0000000600a452e200ab
:1023d00071003600a0d2bf00a152b50001003a0042
:1023e0006c00370010c4b300a052b5002e003900b5
:1023f000a0d2bf000080fb0001fc2f0001004000c4
:102400006093880002002000c327240060938000ae
:1024100052fa070094f9070020948800319488004c
:10242000a4d2bf000080fb0000004000419b2400bc
:1024300060807800a08f8800020020000300240044
:10244000a08f800045fa070087f9070022948000da
:1024500033948000c7f907002094880031948800e5
:1024600020948000319480001cfa0700609388005b
:10247000a4d2bf000080fb0000004000413b2100cf
:1024800060807800a08f880060938000f411b50010
:10249000209388006c12ee0060908800a0d2bf00ec
:1024a000a1f2b7003b00370000c4b300a052e30024
:1024b0000b003a006c32ef00a4d2bf000080fb009a
:1024c00000004000413b210060807800209388009c
:1024d0000c32ef00a0d2bf00a1f2b7002d003700f0
:1024e000a0d2bf008080fb0000042000010050004b
:1024f000609388000200200003282400609380007d
:1025000016fa070058f907002094880031948800d3
:10251000a4d2bf000080fb0000004000419b2400cb
:1025200060807800a08f8800020020000300240053
:10253000a08f800009fa07004bf907002294800061
:10254000339480008bf90700209488003194880030
:102550002094800031948000e0f9070060938800a7
:10256000a4d2bf000080fb0000004000413b2100de
:1025700060807800a08f880060938000f411b40020
:10258000209388006093800060908800a0d2bf00f4
:10259000a1f2b700020037000c32ef00a1f2ef0009
:1025a000a0f2ef00000006009ef2ef00000006001f
:1025b000b0c7b3009b52e30002003a00097707005e
:1025c000430337009bd2bf0080407800e1cf50002a
:1025d00007003a009cd2bf000080fb004206de00ec
:1025e00040ad260060407e00aaf2b70038033700f5
:1025f0009bd2bf0080407800e2cf50000d003a002f
:102600009c52ec00a3f2b700a2722000a3d2bf003c
:102610000080fb000200b8004094880051948800bc
:102620004094800060088800509480007008880002
:10263000270337009bd2bf0080407800e3cf5000d3
:1026400009003a009cd2bf00a7f2b700a8d2bf0091
:102650000080fb0000004000412b210060807800da
:10266000d00888001a0337009bd2bf008040780052
:10267000e4cf500009003a009cd2bf00a8f2b70096
:10268000a8d2bf000080fb0000004000412b2100c9
:1026900060807800d00888000d0337009bd2bf000f
:1026a00080407800ebcf500006003a009c12af004b
:1026b00002003700a612a90001003700a612a800e8
:1026c000030337009bd2bf0080407800f4cf500056
:1026d0005a013a002068a9000068a90000402000c3
:1026e00030618800462cef00a472ef0000c3b300f5
:1026f0009c52e30008003a004c3b2100401b25009f
:102700007f000900301e78009cd2bf00abf2b700fa
:10271000f20307004801370010c3b3009c52e300e6
:1027200008003a004c3b2100402b25007f000900a7
:10273000301e78009cd2bf00abf2b700e703070061
:102740003d01370020c3b3009c52e30008003a006b
:102750004c3b2100403b25007f000900301e7800e3
:102760009cd2bf00abf2b700dc0307003201370098
:1027700030c3b3009c52e30008003a004c3b2100f8
:10278000404b25007f000900301e78009cd2bf001e
:10279000abf2b700d10307002701370040c3b300f5
:1027a0009c52e30008003a004c3b2100405b2500ae
:1027b0007f000900301e78009cd2bf00abf2b7004a
:1027c000c60307001c01370050c3b3009c52e3004e
:1027d00008003a004c3b2100406b25007f000900b7
:1027e000301e78009cd2bf00abf2b700bb030700dd
:1027f0001101370060c3b3009c52e30008003a00a7
:102800004c3b2100407b25007f000900301e7800f2
:102810009cd2bf00abf2b700b0030700060137003f
:1028200070c3b3009c52e30008003a004c3b210007
:10283000408b25007f000900301e78009cd2bf002d
:10284000abf2b700a5030700fb00370080c3b3005d
:102850009c52e30008003a004c3b2100409b2500bd
:102860007f000900301e78009cd2bf00abf2b70099
:102870009a030700f000370090c3b3009c52e300b6
:1028800007003a004c3b210040ab25007f000900c7
:10289000301e78009cd2bf00abf2b700e6003700d4
:1028a000a0c3b3009c52e30008003a004c3b210057
:1028b00040bb25007f000900301e78009cd2bf007d
:1028c000abf2b70085030700db003700b0c3b300ed
:1028d0009c52e30008003a004c3b210040cb25000d
:1028e0007f000900301e78009cd2bf00abf2b70019
:1028f0007a030700d0003700d0c3b3009c52e30036
:1029000008003a004c3b2100400b25007f000900e5
:10291000301e78009cd2bf00abf2b7006f030700f7
:10292000c5003700e0c3b3009c52e30008003a0042
:102930004c3b210040eb24007f000900301e780052
:102940009cd2bf00abf2b70064030700ba003700a7
:10295000f0c3b3009c52e30008003a004c3b210056
:1029600040db24007f000900301e78009cd2bf00ad
:10297000abf2b70059030700af00370000c4b30043
:102980009c52e30008003a004c3b210040ab24007d
:102990007f000900301e78009cd2bf00abf2b70068
:1029a0004e030700a400370010c4b3009c52e3009c
:1029b00008003a004c3b210040bb24007f00090086
:1029c000301e78009cd2bf00abf2b7004303070073
:1029d0009900370020c4b3009c52e30008003a007d
:1029e0004c3b210040cb24007f000900301e7800c2
:1029f0009cd2bf00abf2b700380307008e0037004f
:102a000030c4b3009c52e30008003a004c3b210064
:102a100040fb24007f000900301e78009cd2bf00dc
:102a2000abf2b7002d0307008300370080c4b3006a
:102a30009c52e30008003a004c3b210040db25009b
:102a40007f000900301e78009cd2bf00abf2b700b7
:102a5000220307007800370090c4b3009c52e300c3
:102a600008003a004c3b210040eb25007f000900a4
:102a7000301e78009cd2bf00abf2b70017030700ee
:102a80006d003700a0c4b3009c52e30008003a0078
:102a90004c3b210040fb25007f000900301e7800e0
:102aa0009cd2bf00abf2b7000c03070062003700f6
:102ab000b0c4b3009c52e30008003a004c3b210034
:102ac000400b26007f000900301e78009cd2bf001a
:102ad000abf2b7000103070057003700c0c4b300d2
:102ae0009c52e30008003a004c3b2100401b2600aa
:102af0007f000900301e78009cd2bf00abf2b70007
:102b0000f60207004c003700d0c4b3009c52e3002b
:102b100008003a004c3b2100402b26007f000900b2
:102b2000301e78009cd2bf00abf2b700eb0207006a
:102b300041003700e0c4b3009c52e30008003a00b3
:102b40004c3b2100403b26007f000900301e7800ee
:102b50009cd2bf00abf2b700e0020700360037009e
:102b6000f0c4b3009c52e30008003a004c3b210043
:102b7000404b26007f000900301e78009cd2bf0029
:102b8000abf2b700d50207002b00370000c5b30039
:102b90009c52e30008003a004c3b2100405b2600b9
:102ba0007f000900301e78009cd2bf00abf2b70056
:102bb000ca0207002000370010c5b3009c52e30092
:102bc00008003a004c3b2100406b26007f000900c2
:102bd000301e78009cd2bf00abf2b700bf020700e6
:102be0001500370020c5b3009c52e30008003a00ee
:102bf0004c3b2100407b26007f000900301e7800fe
:102c00009cd2bf00abf2b700b40207000a00370045
:102c100030c5b3009c52e30007003a004c3b210052
:102c2000408b26007f000900301e78009cd2bf0038
:102c3000abf2b700a9020700a501370080c2b300bc
:102c40009b52e3005a003a009cd2bf0080407800bb
:102c5000e1cf500005003a0060918000a09288000a
:102c600070918000b0928800500037009cd2bf0065
:102c700080407800e2cf500005003a00809180004b
:102c8000a092880090918000b092880047003700a1
:102c90009cd2bf0080407800e3cf500005003a008e
:102ca000a0918000a0928800b0918000b09288002e
:102cb0003e0037009cd2bf0080407800e4cf500037
:102cc00005003a00c0918000a0928800d091800059
:102cd000b0928800350037009cd2bf008040780059
:102ce000e5cf500005003a00e0918000a0928800f6
:102cf000f0918000b09288002c0037009cd2bf0079
:102d000080407800e6cf500005003a000092800035
:102d1000a092880010928000b092880023003700b3
:102d20009cd2bf0080407800e7cf500005003a00f9
:102d300020928000a092880030928000b09288009b
:102d40001a0037009cd2bf0080407800e8cf5000c6
:102d500005003a0040928000a092880050928000c6
:102d6000b0928800110037009cd2bf0080407800ec
:102d7000e9cf500005003a0060928000a0928800e0
:102d800070928000b0928800080037009cd2bf008b
:102d900080407800eacf500004003a008092800022
:102da000a092880090928000b0928800480137007d
:102db00090c2b3009b52e3005a003a009cd2bf007d
:102dc00080407800e1cf500005003a00609180001b
:102dd000c092880070918000d09288005000370027
:102de0009cd2bf0080407800e2cf500005003a003e
:102df00080918000c092880090918000d0928800dd
:102e0000470037009cd2bf0080407800e3cf5000dd
:102e100005003a00a0918000c0928800b091800027
:102e2000d09288003e0037009cd2bf0080407800de
:102e3000e4cf500005003a00c0918000c0928800a5
:102e4000d0918000d0928800350037009cd2bf001e
:102e500080407800e5cf500005003a00e091800006
:102e6000c0928800f0918000d09288002c0037003a
:102e70009cd2bf0080407800e6cf500005003a00a9
:102e800000928000c092880010928000d09288004a
:102e9000230037009cd2bf0080407800e7cf50006d
:102ea00005003a0020928000c09288003092800095
:102eb000d09288001a0037009cd2bf008040780072
:102ec000e8cf500005003a0040928000c092880090
:102ed00050928000d0928800110037009cd2bf0031
:102ee00080407800e9cf500005003a0060928000f1
:102ef000c092880070928000d0928800080037004d
:102f00009cd2bf0080407800eacf500004003a0015
:102f100080928000c092880090928000d0928800b9
:102f2000eb003700a0c2b3009b52e3005a003a0006
:102f30009cd2bf0080407800e1cf500005003a00ed
:102f400060918000e092880070918000f09288008b
:102f5000500037009cd2bf0080407800e2cf500084
:102f600005003a0080918000e092880090918000f6
:102f7000f0928800470037009cd2bf008040780064
:102f8000e3cf500005003a00a0918000e092880055
:102f9000b0918000f09288003e0037009cd2bf00c4
:102fa00080407800e4cf500005003a00c0918000d6
:102fb000e0928800d0918000f092880035003700c0
:102fc0009cd2bf0080407800e5cf500005003a0059
:102fd000e0918000e0928800f0918000f0928800fb
:102fe0002c0037009cd2bf0080407800e6cf500014
:102ff00005003a0000928000e09288001092800064
:10300000f0928800230037009cd2bf0080407800f7
:10301000e7cf500005003a0020928000e09288003f
:1030200030928000f09288001a0037009cd2bf00d6
:1030300080407800e8cf500005003a0040928000c0
:10304000e092880050928000f092880011003700d2
:103050009cd2bf0080407800e9cf500005003a00c4
:1030600060928000e092880070928000f092880068
:10307000080037009cd2bf0080407800eacf5000a3
:1030800004003a0080928000e092880090928000d4
:10309000f09288008e003700b0c2b3009b52e3006c
:1030a0005a003a009cd2bf0080407800e1cf500027
:1030b00005003a00609180000093880070918000c4
:1030c00010938800500037009cd2bf0080407800e9
:1030d000e2cf500005003a00809180000093880004
:1030e0009091800010938800470037009cd2bf0069
:1030f00080407800e3cf500005003a00a0918000a6
:1031000000938800b0918000109388003e00370043
:103110009cd2bf0080407800e4cf500005003a0008
:10312000c091800000938800d091800010938800a7
:10313000350037009cd2bf0080407800e5cf5000ba
:1031400005003a00e091800000938800f091800033
:10315000109388002c0037009cd2bf00804078007c
:10316000e6cf500005003a000092800000938800ee
:103170001092800010938800230037009cd2bf007b
:1031800080407800e7cf500005003a002092800090
:103190000093880030928000109388001a00370056
:1031a0009cd2bf0080407800e8cf500005003a0074
:1031b0004092800000938800509280001093880015
:1031c000110037009cd2bf0080407800e9cf50004a
:1031d00005003a00609280000093880070928000a1
:1031e00010938800080037009cd2bf008040780010
:1031f000eacf500004003a008092800000938800db
:1032000090928000109388003100370020c4b300f2
:103210009b52e30006003a009c52e20002003a0092
:10322000f773070001003700048ea800280037005c
:1032300080c6b3009b52e3000e003a009cd2bf0050
:10324000b0f2b70010c0b300b052b50002003100b8
:1032500010c0b300b0f2b700f0c7b300b052b50071
:1032600002003900e0c7b300b0f2b700af130700a7
:103270001700370090c6b3009b52e3000e003a00df
:103280009cd2bf00b1f2b70040c0b300b152b5004c
:103290000200310040c0b300b1f2b700c0c7b300b4
:1032a000b152b50002003900b0c7b300b1f2b700a7
:1032b000ed43070006003700a0c6b3009b52e300b1
:1032c00003003a009cd2bf00b2f2b700e643070009
:1032d0009bf2ef000000060000d02700a0958800b8
:1032e000a0c72500b095880050982500c09588009b
:1032f00040812500d0958800906a2500e0958800df
:1033000030542500f0958800303e25000096880056
:1033100090282500109688005013250020968800dc
:1033200060fe240030968800c0e9240040968800a2
:1033300080d524005096880090c1240060968800b3
:10334000f0ad240070968800a09a24008096880032
:10335000a087240090968800f0742400a09688002e
:1033600090622400b096880080502400c0968800a7
:10337000b03e2400d0968800302d2400e0968800ce
:10338000f01b2400f0968800000b240000978800b2
:1033900050fa230010978800e0e923002097880066
:1033a000c0d9230030978800e0c9230040978800e7
:1033b00040ba230050978800e0aa23006097880055
:1033c000c09b230070978800e08c230080978800c2
:1033d000307e230090978800d06f2300a09788004c
:1033e000a0612300b0978800b0532300c0978800e5
:1033f000f0452300d097880070382300e0978800bc
:10340000202b2300f0978800101e230000988800ce
:103410004011230010988800900423002098880011
:1034200020f8220030988800e0eb220040988800c5
:10343000d0df220050988800f0d3220060988800e6
:1034400050c8220070988800d0bc22008098880064
:1034500080b122009098880070a62200a098880071
:10346000809b2200b0988800c0902200c0988800fd
:1034700020862200d0988800c07b2200e098880037
:1034800080712200f098880060672200009988000f
:10349000805d220010998800c05322002099880086
:1034a000204a220030998800b040220040998800cc
:1034b0006037220050998800402e220060998800d1
:1034c0004025220070998800601c220080998800a5
:1034d000b013220090998800200b2200a099880048
:1034e000b0022200b099880060fa2100c0998800db
:1034f00040f22100d099880030ea2100e09988004c
:1035000050e22100f099880090da2100009a8800aa
:10351000e0d22100109a880060cb2100209a880018
:10352000f0c32100309a8800b0bc2100409a880086
:1035300080b52100509a880080ae2100609a8800f2
:1035400090a72100709a8800b0a02100809a88007e
:10355000009a2100909a880060932100a09a880028
:10356000e08c2100b09a880080862100c09a8800f3
:1035700030802100d09a8800007a2100e09a8800eb
:10358000f0732100f09a8800f06d2100009b880004
:1035900000682100109b880040622100209b880069
:1035a000805c2100309b8800e0562100409b880011
:1035b00060512100509b8800f04b2100609b8800e7
:1035c00090462100709b880050412100809b88001c
:1035d000203c2100909b880010372100a09b880090
:1035e00010322100b09b8800202d2100c09b880054
:1035f00040282100d09b880080232100e09b880088
:10360000d01e2100f09b8800301a2100009c880009
:10361000a0152100109c880020112100209c88000a
:10362000c00c2100309c880070082100409c88005c
:1036300020042100509c8800f0ff2000609c88003e
:10364000d0fb2000709c8800c0f72000809c880080
:10365000d0f32000909c8800e0ef2000a09c880020
:1036600000ec2000b09c880030e82000c09c88005e
:1036700070e42000d09c8800c0e02000e09c88001e
:1036800020dd2000f09c880090d92000009d88005b
:1036900010d62000109d8800a0d22000209d880018
:1036a00040cf2000309d8800e0cb2000409d880066
:1036b000a0c82000509d880060c52000609d880043
:1036c00030c22000709d880010bf2000809d8800bf
:1036d00000bc2000909d88000000060010c0b300d0
:1036e000a2f2b700e0c7b300a252e30022003e00fe
:1036f000a2d2bf000080fb000006e9000c064600d5
:10370000403b210060007e00a08f8800a2d2bf0055
:103710000080fb000006e8000c064600403b21004c
:1037200060007e00f411b500212a2100914078004c
:103730008180fb0081804000428b24008030790032
:10374000a2d2bf000080fb0000004000418b24009b
:10375000608078004100de00212a2100914078003d
:103760008180fb0081804000429b240080307900f2
:10377000a272ec00dbff3900609b2400100078008f
:10378000419b24008008780000ab240010007800e2
:1037900021ab240080087800608b240010007800a2
:1037a000418b240080087800009b240010007800e2
:1037b000219b24008008780000000600b040200013
:1037c000a0a5880040412000b0a58800c04120008d
:1037d000c0a5880060422000d0a58800704320006a
:1037e000e0a5880010452000f0a5880000482000d2
:1037f00000a68800a049200010a68800e04a20000a
:1038000020a68800e04b200030a68800c04c200095
:1038100040a68800704d200050a68800c04d2000b2
:1038200060a68800604d200070a68800604c2000d3
:1038300080a68800104b200090a6880060492000d8
:10384000a0a6880090472000b0a6880090452000e0
:10385000c0a68800a0422000d0a68800c04020005a
:10386000e0a68800203f2000f0a68800c03d200090
:1038700000a78800c03c200010a78800003c200062
:1038800020a78800a03b200030a78800d03b200064
:1038900040a78800203c200050a78800603c200002
:1038a00060a78800603c200070a78800303c2000a2
:1038b00080a78800103c200090a78800503c200082
:1038c000a0a78800b03c2000b0a78800e03c200002
:1038d000c0a78800e03c2000d0a78800903c2000d2
:1038e000e0a78800103c2000f0a78800a03b200043
:1038f00000a88800b03b200010a88800e03b200012
:1039000020a88800203c200030a88800403c2000ef
:1039100040a88800203c200050a88800e03b200000
:1039200060a88800e03b200070a88800303c2000a0
:1039300080a88800a03c200090a88800203d20009e
:10394000a0a88800b03d2000b0a88800503e20000c
:10395000c0a88800b03e2000d0a88800f03e20001b
:10396000e0a88800403f2000f0a88800803f2000a9
:1039700000a98800d03f200010a988001040200036
:1039800020a988005040200030a988001040200065
:1039900040a98800b03f200050a98800403f200087
:1039a00060a98800f03e200070a98800d03e200069
:1039b00080a98800b03e200090a98800903e200099
:1039c000a0a98800403e2000b0a98800d03d20007a
:1039d000c0a98800503d2000d0a98800003d2000eb
:1039e000e0a98800003d2000f0a98800203d2000cb
:1039f00000aa8800403d200010aa8800303d200029
:103a000020aa8800103d200030aa8800003d200038
:103a100040aa8800203d200050aa8800603d200078
:103a200060aa8800a03d200070aa8800e03d200028
:103a300080aa8800f03d200090aa8800003e200067
:103a4000a0aa8800203e2000b0aa8800803e200066
:103a5000c0aa8800d03e2000d0aa8800103f2000d5
:103a6000e0aa8800503f2000f0aa8800a03f200074
:103a700000ab8800d03f200010ab88001040200031
:103a800020ab88002040200030ab88003040200070
:103a900040ab88009040200050ab880020412000bf
:103aa00060ab88009041200070ab8800e0412000ae
:103ab00080ab8800f041200090ab880000422000dd
:103ac000a0ab880020422000b0ab880080422000dc
:103ad000c0ab8800e0422000d0ab8800004320004b
:103ae000e0ab880070422000f0ab8800c0412000ad
:103af00000ac88003041200010ac8800f04020006d
:103b000020ac8800c040200030ac8800b0402000cd
:103b100040ac88003040200050ac8800a03f20001e
:103b200060ac8800103f200070ac8800e03e2000b0
:103b300080ac8800f03e200090ac8800203f200040
:103b4000a0ac8800003f2000b0ac8800603e2000a0
:103b5000c0ac8800903d2000d0ac8800c03c200064
:103b6000e0ac8800303c2000f0ac8800d03b200066
:103b700000ad8800803b200010ad8800403b200055
:103b800020ad8800603b200030ad8800903b2000d5
:103b900040ad8800c03b200050ad8800103c2000a4
:103ba00060ad8800403c200070ad8800e03c200003
:103bb00080ad8800c03d200090ad8800f03e200020
:103bc000a0ad880010402000b0ad8800304120003a
:103bd000c0ad880030422000d0ad8800c043200036
:103be000e0ad880080452000f0ad8800404720000f
:103bf00000ae88000049200010ae8800f04a200086
:103c000020ae8800004d200030ae880040502000db
:103c100040ae88006052200050ae880090532000d3
:103c200060ae88001054200070ae8800a0532000c1
:103c300080ae88005052200090ae88008050200056
:103c4000a0ae8800604c2000b0ae88003049200053
:103c5000c0ae8800f0452000d0ae8800f0422000c1
:103c6000e0ae8800e0402000f0ae8800b03f2000c9
:103c700000af8800e03e200010af8800703e2000ba
:103c800020af8800e03d200030af8800503d20008c
:103c900040af8800203d200050af8800003d20004c
:103ca00060af8800b03c200070af8800f03b20007f
:103cb00080af8800103b200090af8800603a200061
:103cc000a0af8800203a2000b0af8800303a200032
:103cd000c0af8800403a2000d0af8800503a2000a2
:103ce000e0af8800403a2000f0af8800403a200062
:103cf00000b08800503a200010b08800403a200000
:103d000020b08800303a200030b08800303a2000df
:103d100040b08800803a200050b08800f03a20007f
:103d200060b08800403b200070b08800603b2000fd
:103d300080b08800803b200090b08800703b20005d
:103d4000a0b08800d03b2000b0b08800903c20009c
:103d5000c0b08800603d2000d0b08800203e200028
:103d6000e0b08800b03e2000f0b08800203f200086
:103d700000b18800803f200010b188002040200062
:103d800020b18800b040200030b188000041200000
:103d900040b188000041200050b18800c0402000a0
:103da00060b18800f03f200070b18800503f2000d3
:103db00080b18800b03e200090b18800303e2000e5
:103dc000a0b18800f03d2000b0b18800c03d2000c7
:103dd000c0b18800a03d2000d0b18800a03d2000e7
:103de000e0b18800a03d2000f0b18800e03d200057
:103df00000b28800503e200010b28800c03e200073
:103e000020b28800003f200030b28800e03e200051
:103e100040b28800a03e200050b28800503e2000f2
:103e200060b28800103e200070b28800c03d2000c3
:103e300080b28800d03d200090b28800503e200023
:103e4000a0b28800b03e2000b0b28800e03e200062
:103e5000c0b28800d03e2000d0b28800703e200062
:103e6000e0b28800103e2000f0b28800e03d200063
:103e700000b38800303e200010b38800b03e200020
:103e800020b38800403f200030b38800b03f2000be
:103e900040b38800d03f200050b38800903f2000fe
:103ea00060b38800903f200070b38800d03f2000ae
:103eb00080b388006040200090b3880080412000db
:103ec000a0b3880070422000b0b38800e042200018
:103ed000c0b3880080422000d0b38800e0412000b9
:103ee000e0b3880090412000f0b38800304120000a
:103ef00000b488009040200010b48800b03f20003b
:103f000020b48800203e200030b48800703d20009e
:103f100040b48800203d200050b48800003d2000bf
:103f200060b48800f03c200070b48800f03c2000b1
:103f300080b48800c03c200090b48800b03c2000d1
:103f4000a0b48800c03c2000b0b48800103d200020
:103f5000c0b48800603d2000d0b48800c03d20007f
:103f6000e0b48800203e2000f0b48800403e2000ed
:103f700000b58800603e200010b58800b03e2000eb
:103f800020b58800403f200030b588002040200048
:103f900040b588005041200050b588008043200083
:103fa00060b588007045200070b58800b0472000db
:103fb00080b58800304a200090b58800204d200050
:103fc000a0b5880000502000b0b5880070542000d3
:103fd000c0b5880050572000d0b58800a0592000f7
:103fe000e0b58800305b2000f0b58800905b2000d1
:103ff00000b68800205b200010b688001058200012
:1040000020b688008054200030b68800e04f2000a1
:1040100040b68800204b200050b68800d0462000d3
:1040200060b68800b042200070b68800d03e200004
:1040300080b68800a039200090b68800b0362000f5
:10404000a0b68800a0342000b0b68800203320003d
:10405000c0b6880010322000d0b68800a031200001
:10406000e0b68800e0312000f0b68800c0322000c1
:1040700000b78800e033200010b78800103520001a
:1040800020b788003036200030b78800e0362000a6
:1040900040b788007037200050b78800b037200044
:1040a00060b788000038200070b7880070382000a2
:1040b00080b78800c038200090b78800e038200022
:1040c000a0b7880050392000b0b78800b039200070
:1040d000c0b78800103a2000d0b78800403a2000ce
:1040e000e0b78800303a2000f0b78800103a20008e
:1040f00000b88800103a200010b88800a03a2000cc
:1041000020b88800403b200030b88800d03b200019
:1041100040b88800603c200050b88800003d200076
:1041200060b88800a03d200070b88800e03e200004
:1041300080b88800903f200090b888005040200050
:10414000a0b88800f0402000b0b88800504120009e
:10415000c0b8880080412000d0b8880060412000ad
:10416000e0b88800f0402000f0b8880080402000cf
:1041700000b98800c03f200010b98800003f20002f
:1041800020b98800303e200030b98800803d2000f2
:1041900040b98800c03c200050b98800703c200025
:1041a00060b98800403c200070b98800203c2000a5
:1041b00080b98800003c200090b98800003c2000b5
:1041c000a0b98800603c2000b0b98800b03c200055
:1041d000c0b98800103d2000d0b98800703d200093
:1041e000e0b98800f03d2000f0b98800803e200052
:1041f00000ba8800603f200010ba8800004020000c
:1042000020ba8800b040200030ba88003041200039
:1042100040ba88009041200050ba8800c041200078
:1042200060ba88002042200070ba880080422000d6
:1042300080ba8800d042200090ba88000043200055
:10424000a0ba8800f0422000b0ba880000432000e5
:10425000c0ba880030432000d0ba880080432000d4
:10426000e0ba880080432000f0ba88005043200064
:1042700000bb88005043200010bb8800a0432000f2
:1042800020bb88004044200030bb8800204520002f
:1042900040bb88004045200050bb8800f04420000f
:1042a00060bb88005044200070bb8800b0432000f1
:1042b00080bb88001043200090bb88006042200033
:1042c000a0bb8800f0412000b0bb880070412000f6
:1042d000c0bb8800d0402000d0bb88000040200038
:1042e000e0bb8800303f2000f0bb8800903e2000fb
:1042f00000bc8800b03d200010bc8800203d20009c
:1043000020bc8800a03c200030bc8800503c20002d
:1043100040bc8800203c200050bc8800003c2000ad
:1043200060bc8800c03b200070bc8800803b20003f
:1043300080bc8800403b200090bc8800003b2000ef
:10434000a0bc8800103b2000b0bc8800603b20006f
:10435000c0bc8800403c2000d0bc8800103d20003c
:10436000e0bc8800f03d2000f0bc8800103f200039
:1043700000bd88006040200010bd88000042200081
:1043800020bd88009044200030bd880040462000b9
:1043900040bd8800e047200050bd880080492000d3
:1043a00060bd8800004b200070bd8800a04c20003c
:1043b00080bd8800304e200090bd88003050200025
:1043c000a0bd880010512000b0bd880070512000b1
:1043d000c0bd880090512000d0bd880060512000f1
:1043e000e0bd8800d0502000f0bd8800404f200084
:1043f00000be8800a04d200010be8800e04b2000c9
:1044000020be8800404a200030be8800704820004e
:1044100040be8800c046200050be880040442000b6
:1044200060be88009042200070be880010412000cd
:1044300080be8800a03f200090be8800603e200023
:10444000a0be8800703d2000b0be8800a03c2000c7
:10445000c0be8800903b2000d0be8800503a2000ab
:10446000e0be8800a0382000f0be88007036200032
:1044700000bf88004034200010bf88007032200048
:1044800020bf8800f030200030bf880000312000bd
:1044900040bf88009031200050bf8800b03220001b
:1044a00060bf88001034200070bf880020352000d5
:1044b00080bf88008036200090bf880050372000e1
:1044c000a0bf8800e0372000b0bf8800b0382000cf
:1044d000c0bf880070392000d0bf8800203a20007b
:1044e000e0bf8800003b2000f0bf8800603b200058
:1044f00000c08800e03b200010c08800703c200015
:1045000020c08800e03c200030c08800103d200022
:1045100040c08800e03c200050c08800b03c200033
:1045200060c08800003d200070c08800803d2000f1
:1045300080c08800103e200090c08800503e2000bf
:10454000a0c08800403e2000b0c08800703e20001f
:10455000c0c08800b03e2000d0c08800d03e2000ff
:10456000e0c08800d03e2000f0c08800a03e2000bf
:1045700000c18800703e200010c18800103e20005d
:1045800020c18800d03d200030c18800a03d20001f
:1045900040c18800a03d200050c18800c03d2000df
:1045a00060c18800f03d200070c18800003e2000fe
:1045b00080c18800203e200090c18800603e20001d
:1045c000a0c18800e03e2000b0c18800803f2000ec
:1045d000c0c18800f03f2000d0c1880040402000ca
:1045e000e0c1880090402000f0c18800e040200039
:1045f00000c288003041200010c2880080412000a5
:1046000020c28800a041200030c28800a0412000c4
:1046100040c28800d041200050c2880010422000d3
:1046200060c288004042200070c2880040422000e2
:1046300080c288002042200090c28800f041200003
:10464000a0c28800b0412000b0c2880040412000d4
:10465000c0c2880030412000d0c2880060412000e4
:10466000e0c28800d0412000f0c2880060422000f3
:1046700000c38800b042200010c38800f042200030
:1046800020c388000043200030c38800204320005e
:1046900040c388001043200050c38800d04220004f
:1046a00060c388007042200070c38800d0412000a1
:1046b00080c388005041200090c38800c040200083
:1046c000a0c3880030402000b0c38800a03f200075
:1046d000c0c38800203f2000d0c38800403e200097
:1046e000e0c38800803d2000f0c38800c03c20006b
:1046f00000c48800403c200010c48800e03b20003b
:1047000020c48800a03b200030c48800703b2000fb
:1047100040c48800203b200050c48800e03a2000bc
:1047200060c48800c03a200070c48800a03a20000d
:1047300080c48800b03a200090c48800c03a2000ad
:10474000a0c48800c03a2000b0c48800c03a20004d
:10475000c0c48800f03a2000d0c48800503b20003c
:10476000e0c48800f03b2000f0c48800d03c20006a
:1047700000c58800c03e200010c588008040200091
:1047800020c58800d042200030c58800b0452000f8
:1047900040c58800e048200050c58800c04c20007b
:1047a00060c58800d050200070c58800b057200038
:1047b00080c58800305c200090c5880060602000c3
:1047c000a0c5880010642000b0c58800e066200005
:1047d000c0c5880000682000d0c58800c0652000e2
:1047e000e0c5880080612000f0c58800505b200093
:1047f00000c68800e053200010c68800004c20004e
:1048000020c68800b044200030c68800a03b2000ad
:1048100040c688002037200050c68800d0332000d2
:1048200060c68800a031200070c68800803020005b
:1048300080c688005030200090c68800b03020002c
:10484000a0c6880020312000b0c68800803120003a
:10485000c0c6880000322000d0c688008032200008
:10486000e0c68800d0322000f0c688001033200057
:1048700000c788008033200010c788000034200063
:1048800020c78800d034200030c788009035200031
:1048900040c788005036200050c7880000372000ed
:1048a00060c78800a037200070c78800b03720009c
:1048b00080c788006037200090c78800f03620004d
:1048c000a0c7880090362000b0c78800603620005e
:1048d000c0c7880090362000d0c78800103720005d
:1048e000e0c78800c0372000f0c78800a03820004b
:1048f00000c88800c039200010c88800e03a2000b5
:1049000020c88800f03b200030c88800703d20009f
:1049100040c88800903e200050c88800a03f20007a
:1049200060c88800b040200070c88800a041200006
:1049300080c888005042200090c88800d0422000e3
:10494000a0c88800a0422000b0c8880020422000f3
:10495000c0c8880040412000d0c8880060402000c6
:10496000e0c88800603f2000f0c88800503e20006a
:1049700000c98800f03d200010c98800b03d20002b
:1049800020c98800b03d200030c98800003e2000ca
:1049900040c98800603e200050c98800003f2000c8
:1049a00060c98800403f200070c98800803f200017
:1049b00080c98800c03f200090c98800f03f2000d7
:1049c000a0c9880020402000b0c9880050402000c5
:1049d000c0c9880070402000d0c988006040200015
:1049e000e0c9880070402000f0c988009040200095
:1049f00000ca8800e040200010ca88001041200052
:104a000020ca88002041200030ca880010412000c0
:104a100040ca8800f040200050ca8800f0402000c2
:104a200060ca88000041200070ca88003041200020
:104a300080ca88009041200090ca8800104220005f
:104a4000a0ca8800b0422000b0ca8800604320009d
:104a5000c0ca880010442000d0ca8800a0442000aa
:104a6000e0ca880010452000f0ca88008045200078
:104a700000cb88008045200010cb880050452000e6
:104a800020cb8800d044200030cb88000044200098
:104a900040cb88003043200050cb8800f0412000fc
:104aa00060cb88000041200070cb880000402000cf
:104ab00080cb8800e03e200090cb8800b03d2000f5
:104ac000a0cb8800703c2000b0cb8800b03a20001a
:104ad000c0cb8800b0392000d0cb8800d03820006f
:104ae000e0cb880030382000f0cb880090372000e1
:104af00000cc88002037200010cc8800d036200061
:104b000020cc8800b036200030cc8800f036200061
:104b100040cc88007037200050cc8800f03720004f
:104b200060cc88009038200070cc8800603920006c
:104b300080cc8800c03a200090cc8800003c200047
:104b4000a0cc8800803d2000b0cc8800503f2000e1
:104b5000c0cc880070412000d0cc8800f0432000f9
:104b6000e0cc8800e0472000f0cc8800904a20008c
:104b700000cd8800304d200010cd8800c04f2000af
:104b800020cd88003052200030cd8800b054200065
:104b900040cd8800a058200050cd8800605b2000e8
:104ba00060cd8800b05d200070cd8800505f20008f
:104bb00080cd88001060200090cd8800d05f20005c
:104bc000a0cd8800905e2000b0cd8800c05a2000a3
:104bd000c0cd8800f0562000d0cd88005052200073
:104be000e0cd8800504d2000f0cd880070482000b6
:104bf00000ce8800c043200010ce8800b03c2000ca
:104c000020ce88009038200030ce8800403520002b
:104c100040ce8800b032200050ce8800e030200026
:104c200060ce8800d02f200070ce8800302f20006a
:104c300080ce8800302f200090ce8800902f20005a
:104c4000a0ce8800e02f2000b0ce88007030200079
:104c5000c0ce8800e0302000d0ce88004031200057
:104c6000e0ce8800d0312000f0ce880060322000f5
:104c700000cf8800a032200010cf8800e032200052
:104c800020cf88003033200030cf8800a0332000b0
:104c900040cf8800a034200050cf8800803520000d
:104ca00060cf88006036200070cf88005037200029
:104cb00080cf88004038200090cf88001039200035
:104cc000a0cf8800003a2000b0cf8800a03a200092
:104cd000c0cf8800503b2000d0cf8800103c20007f
:104ce000e0cf8800f03c2000f0cf8800003e20009c
:104cf00000d08800903f200010d08800a040200005
:104d000020d08800a041200030d0880060422000e0
:104d100040d088000043200050d08800304320005d
:104d200060d088000043200070d08800204220001e
:104d300080d088005041200090d088009040200012
:104d4000a0d08800c03f2000b0d08800103f2000d5
:104d5000c0d08800603e2000d0d08800703d200088
:104d6000e0d08800e03c2000f0d08800903c20009b
:104d700000d18800a03c200010d18800e03c200039
:104d800020d18800503d200030d18800d03d200047
:104d900040d18800003e200050d18800503e2000c5
:104da00060d18800d03e200070d18800603f200094
:104db00080d188001040200090d18800a0402000c1
:104dc000a0d1880030412000b0d18800604120008f
:104dd000c0d18800a0412000d0d18800d04120005f
:104de000e0d1880020422000f0d18800304220002d
:104df00000d288002042200010d2880010422000fb
:104e000020d288000042200030d2880000422000da
:104e100040d288000042200050d28800104220007a
:104e200060d288003042200070d2880040422000ca
:104e300080d288006042200090d28800b0422000da
:104e4000a0d2880010432000b0d288008043200008
:104e5000c0d2880030442000d0d288009044200086
:104e6000e0d28800f0442000f0d2880030452000d5
:104e700000d388005045200010d388003045200022
:104e800020d38800e044200030d38800e043200095
:104e900040d388001043200050d3880020422000d7
:104ea00060d388001041200070d38800f03f2000bc
:104eb00080d38800b03e200090d38800e03c2000e2
:104ec000a0d38800d03b2000b0d38800e03a200077
:104ed000c0d38800003a2000d0d3880030392000a9
:104ee000e0d3880090382000f0d38800e03720001d
:104ef00000d48800a037200010d48800703720002c
:104f000020d488004037200030d48800303720007b
:104f100040d488002037200050d48800203720005b
:104f200060d488006037200070d48800b03720003b
:104f300080d488002038200090d48800c038200019
:104f4000a0d4880080392000b0d48800703a2000b6
:104f5000c0d48800703c2000d0d48800303e2000af
:104f6000e0d4880060402000f0d488000043200096
:104f700000d58800e045200010d588004049200079
:104f800020d58800b04e200030d58800a0522000e7
:104f900040d588008056200050d58800805a2000d7
:104fa00060d58800a05e200070d58800f0622000e7
:104fb00080d58800a068200090d58800c06b2000b4
:104fc000a0d58800706d2000b0d58800e06c20006e
:104fd000c0d58800c0692000d0d58800f0632000cb
:104fe000e0d58800e05b2000f0d58800904d2000df
:104ff00000d68800b043200010d68800c03a2000b8
:1050000020d688002033200030d68800002d2000d4
:1050100040d68800b028200050d688009025200077
:1050200060d68800a025200070d68800d0262000f9
:1050300080d68800b028200090d68800f02a200072
:10504000a0d68800402d2000b0d6880090302000e7
:10505000c0d68800a0322000d0d68800303420008e
:10506000e0d6880050352000f0d6880010362000a9
:1050700000d78800a036200010d788000037200015
:1050800020d788006037200030d7880040372000c4
:1050900040d788000037200050d788009036200085
:1050a00060d788004036200070d788001036200076
:1050b00080d788000036200090d788001036200066
:1050c000a0d7880030362000b0d788008036200076
:1050d000c0d7880010372000d0d78800f0372000d4
:1050e000e0d78800a0392000f0d78800d03a20000f
:1050f00000d88800f03b200010d88800003d200038
:1051000020d88800403e200030d88800a03f2000f2
:1051100040d888003041200050d8880060432000eb
:1051200060d888009044200070d888003045200066
:1051300080d888006045200090d888005045200025
:10514000a0d88800d0442000b0d88800b043200008
:10515000c0d88800b0422000d0d8880090412000fc
:10516000e0d8880090402000f0d88800c03f2000a0
:1051700000d98800f03e200010d98800403e200071
:1051800020d98800103e200030d98800403e200001
:1051900040d98800b03e200050d98800303f200020
:1051a00060d98800903f200070d98800004020001e
:1051b00080d988003040200090d9880060402000cd
:1051c000a0d9880080402000b0d98800a0402000ed
:1051d000c0d9880090402000d0d9880050402000dd
:1051e000e0d98800b03f2000f0d98800303f20008f
:1051f00000da8800c03e200010da8800703e2000ef
:1052000020da8800403e200030da8800603e20002e
:1052100040da8800203f200050da8800d03f20008c
:1052200060da8800b040200070da880080412000f9
:1052300080da88006042200090da88005043200025
:10524000a0da8800b0442000b0da88009045200041
:10525000c0da880040462000d0da8800d04620001e
:10526000e0da880020472000f0da8800204720009c
:1052700000db8800d046200010db880010462000ac
:1052800020db88003045200030db880020442000ef
:1052900040db8800d042200050db880080412000a5
:1052a00060db88002040200070db8800303e20005a
:1052b00080db8800103d200090db8800d03b200080
:1052c000a0db8800c03a2000b0db8800c039200095
:1052d000c0db8800f0382000d0db88004038200098
:1052e000e0db880020382000f0db88003038200028
:1052f00000dc88005038200010dc88006038200076
:1053000020dc88006038200030dc880080382000f5
:1053100040dc88007038200050dc880070382000a5
:1053200060dc88005038200070dc880040382000a5
:1053300080dc88002038200090dc880020382000a5
:10534000a0dc880090382000b0dc880010392000f4
:10535000c0dc8800203a2000d0dc8800703b2000b0
:10536000e0dc8800603d2000f0dc8800d03f2000b9
:1053700000dd88009044200010dd88009048200067
:1053800020dd8800104d200030dd880020522000f4
:1053900040dd8800b057200050dd8800c05d20004f
:1053a00060dd88004068200070dd8800406f2000cc
:1053b00080dd88000075200090dd88009078200056
:1053c000a0dd8800b0782000b0dd880010752000d6
:1053d000c0dd8800c06d2000d0dd8800905d200019
:1053e000e0dd880010512000f0dd8800d04420006e
:1053f00000de8800c039200010de8800b0302000b8
:1054000020de8800002a200030de880020242000d2
:1054100040de8800a022200050de8800c02220004c
:1054200060de88002024200070de880050262000e6
:1054300080de88000029200090de8800d02c20002b
:10544000a0de8800002f2000b0de8800d0302000d1
:10545000c0de880070322000d0de8800c03320001b
:10546000e0de8800d0342000f0de88000036200026
:1054700000df88007036200010df880080362000b2
:1054800020df88005036200030df88000036200002
:1054900040df8800c035200050df880090352000b4
:1054a00060df88009035200070df8800a035200084
:1054b00080df8800c035200090df88002036200083
:1054c000a0df880090362000b0df88005037200031
:1054d000c0df880080382000d0df8800b03920008d
:1054e000e0df8800203b2000f0df8800d03c200077
:1054f00000e08800c03e200010e08800b04020009e
:1055000020e088008043200030e088003045200003
:1055100040e088008046200050e08800704720006e
:1055200060e08800d047200070e08800a04720009d
:1055300080e08800d046200090e08800c044200031
:10554000a0e0880010432000b0e088004041200027
:10555000c0e08800b03f2000d0e08800703e20000e
:10556000e0e08800703d2000f0e08800603c200012
:1055700000e18800103c200010e18800103c200071
:1055800020e18800503c200030e18800e03c200011
:1055900040e18800803d200050e18800903e2000de
:1055a00060e18800503f200070e18800e03f20006b
:1055b00080e188007040200090e18800f0402000e9
:1055c000a0e1880050412000b0e188008041200027
:1055d000c0e1880070412000d0e188002041200017
:1055e000e0e18800d0402000f0e188007040200019
:1055f00000e288003040200010e28800e03f2000f8
:1056000020e28800c03f200030e28800d03f200028
:1056100040e288000040200050e288005040200016
:1056200060e28800c040200070e2880060412000f5
:1056300080e28800a042200090e288009043200091
:10564000a0e2880090442000b0e28800804520005d
:10565000c0e2880030462000d0e28800e04620000a
:10566000e0e2880070472000f0e28800a0472000b8
:1056700000e388009047200010e3880020472000c6
:1056800020e388006046200030e388006045200069
:1056900040e388001044200050e38800d0412000ff
:1056a00060e388003040200070e38800903e2000d6
:1056b00080e38800003d200090e38800903b2000bc
:1056c000a0e38800503a2000b0e388003039200081
:1056d000c0e38800e0382000d0e38800c038200014
:1056e000e0e38800d0382000f0e38800e0382000b4
:1056f00000e488000039200010e4880070392000a0
:1057000020e48800c039200030e48800003a2000fe
:1057100040e48800f039200050e48800b0392000cf
:1057200060e488005039200070e4880000392000cf
:1057300080e488009038200090e4880050382000f1
:10574000a0e4880010382000b0e48800f037200082
:10575000c0e4880030382000d0e48800b038200051
:10576000e0e48800303a2000f0e48800b03b2000fc
:1057700000e58800903d200010e5880000402000f2
:1057800020e588001043200030e588001047200005
:1057900040e58800304e200050e58800c0532000ce
:1057a00060e588009059200070e58800e05f2000e7
:1057b00080e588002067200090e58800f06e2000da
:1057c000a0e5880020782000b0e58800f07a20006d
:1057d000c0e5880040792000d0e58800f072200004
:1057e000e0e5880090682000f0e58800705b20000c
:1057f00000e68800504d200010e68800a039200007
:1058000020e68800302f200030e68800a027200006
:1058100040e68800e022200050e68800902020002a
:1058200060e688005020200070e6880020232000d9
:1058300080e688005026200090e68800d0292000cd
:10584000a0e68800202d2000b0e68800c02f2000b0
:10585000c0e68800b0312000d0e688001034200077
:10586000e0e6880090352000f0e68800f036200061
:1058700000e788002038200010e788002039200049
:1058800020e78800f039200030e78800703a2000d7
:1058900040e78800303a200050e78800a039200017
:1058a00060e78800d038200070e78800d0372000fb
:1058b00080e78800a036200090e78800b0352000ff
:1058c000a0e78800f0342000b0e788000035200011
:1058d000c0e7880060352000d0e78800103620003f
:1058e000e0e7880030372000f0e7880080382000ab
:1058f00000e88800f03a200010e88800c03c200052
:1059000020e88800903e200030e888008040200099
:1059100040e888006042200050e8880020442000d1
:1059200060e888008046200070e88800b0472000ca
:1059300080e888006048200090e8880050482000f7
:10594000a0e8880090472000b0e8880010462000ba
:10595000c0e8880020442000d0e8880020412000d2
:10596000e0e88800703f2000f0e88800203e20003a
:1059700000e98800403d200010e98800b03c20008c
:1059800020e98800903c200030e98800603d20003c
:1059900040e98800403e200050e98800403f200058
:1059a00060e988000040200070e988008040200005
:1059b00080e98800d040200090e98800f040200075
:1059c000a0e9880000412000b0e9880000412000e3
:1059d000c0e9880000412000d0e98800d0402000c4
:1059e000e0e9880070402000f0e98800f03f2000e6
:1059f00000ea8800203f200010ea8800b03e200026
:105a000020ea8800403e200030ea8800e03d200087
:105a100040ea8800903d200050ea8800903d200038
:105a200060ea8800403e200070ea8800303f200095
:105a300080ea88006040200090ea8800a0412000b1
:105a4000a0ea880000432000b0ea880080442000db
:105a5000c0ea880080462000d0ea8800c0472000c5
:105a6000e0ea8800b0482000f0ea880060492000a1
:105a700000eb88009049200010eb880020492000ae
:105a800020eb88003048200030eb8800f0452000f3
:105a900040eb88003044200050eb8800704220002a
:105aa00060eb8800b040200070eb8800103f2000c1
:105ab00080eb8800703d200090eb8800403b200088
:105ac000a0eb8800103a2000b0eb880020392000bd
:105ad000c0eb880070382000d0eb88000038200030
:105ae000e0eb8800e0372000f0eb8800f037200082
:105af00000ec88003038200010ec8800a03820002e
:105b000020ec88003039200030ec8800b0392000cb
:105b100040ec8800203a200050ec8800803a2000b9
:105b200060ec8800a03a200070ec8800a03a2000c9
:105b300080ec8800803a200090ec8800403a2000f9
:105b4000a0ec8800103a2000b0ec8800a0392000ba
:105b5000c0ec8800f0382000d0ec8800903820009d
:105b6000e0ec880080382000f0ec8800303920001c
:105b700000ed8800203a200010ed8800a03b2000b6
:105b800020ed8800e03e200030ed8800f04120004c
:105b900040ed8800e045200050ed8800c04a20001c
:105ba00060ed88006050200070ed8800e056200015
:105bb00080ed8800b061200090ed8800e069200051
:105bc000a0ed8800d0722000b0ed8800907a20000f
:105bd000c0ed8800507f2000d0ed8800307f20008d
:105be000e0ed880040792000f0ed8800806720001b
:105bf00000ee88005058200010ee8800f048200089
:105c000020ee8800103b200030ee8800802f20001e
:105c100040ee8800e026200050ee8800a01f200003
:105c200060ee8800401e200070ee8800001f2000fb
:105c300080ee88004021200090ee88008024200023
:105c4000a0ee880030282000b0ee8800202d200033
:105c5000c0ee8800c02f2000d0ee8800b0312000b8
:105c6000e0ee880020332000f0ee88006034200051
:105c700000ef88009035200010ef880040372000aa
:105c800020ef88005038200030ef88006039200075
:105c900040ef8800403a200050ef8800a03a2000f2
:105ca00060ef8800803a200070ef8800f039200013
:105cb00080ef88007038200090ef88004037200087
:105cc000a0ef880030362000b0ef8800803520003b
:105cd000c0ef880040352000d0ef880070352000ec
:105ce000e0ef8800d0362000f0ef88005038200028
:105cf00000f08800203a200010f08800403c20008e
:105d000020f08800703e200030f08800a040200085
:105d100040f08800e043200050f08800e04520007b
:105d200060f08800a047200070f08800d048200074
:105d300080f088006049200090f0880060492000d1
:105d4000a0f08800b0482000b0f088006046200035
:105d5000c0f0880020442000d0f08800904120004e
:105d6000e0f08800003f2000f0f08800d03c2000e8
:105d700000f18800403b200010f18800503a2000dc
:105d800020f18800803a200030f18800f03a2000ad
:105d900040f18800d03b200050f18800e03c20001a
:105da00060f18800103e200070f18800f03f200074
:105db00080f188001041200090f18800004220000e
:105dc000a0f18800d0422000b0f1880050432000ac
:105dd000c0f1880080432000d0f18800604320009b
:105de000e0f1880000432000f0f1880080422000ac
:105df00000f28800d041200010f2880020412000ed
:105e000020f288005040200030f28800903f2000af
:105e100040f28800a03e200050f28800203e200082
:105e200060f28800d03d200070f28800a03d200084
:105e300080f28800a03d200090f28800003e200003
:105e4000a0f28800403f2000b0f28800804020008f
:105e5000c0f28800f0412000d0f2880060432000aa
:105e6000e0f28800b0442000f0f28800f045200005
:105e700000f388009047200010f38800504820006d
:105e800020f388008048200030f38800204820005c
:105e900040f388004047200050f38800f045200080
:105ea00060f388006044200070f38800e041200027
:105eb00080f388002040200090f38800603e20009e
:105ec000a0f38800a03c2000b0f38800103b200025
:105ed000c0f38800d0392000d0f38800803820003b
:105ee000e0f3880000382000f0f38800d03720006d
:105ef00000f488000038200010f48800703820007a
:105f000020f488001039200030f48800303a200056
:105f100040f48800003b200050f48800b03b200093
:105f200060f48800403c200070f48800b03c200001
:105f300080f48800d03c200090f48800a03c200031
:105f4000a0f48800103c2000b0f48800503b2000f2
:105f5000c0f48800803a2000d0f4880090392000f6
:105f6000e0f4880070382000f0f4880050372000fa
:105f700000f588003036200010f58800303620000b
:105f800020f588002037200030f58800e038200018
:105f900040f58800803b200050f58800103f20002d
:105fa00060f58800e045200070f58800d04b2000a7
:105fb00080f588006052200090f58800b0592000dc
:105fc000a0f58800c0612000b0f58800806a20003c
:105fd000c0f5880070772000d0f58800a07d2000f3
:105fe000e0f58800807f2000f0f58800f07b20003d
:105ff00000f68800d072200010f68800a06520000e
:1060000020f688006056200030f68800004020000e
:1060100040f688009033200050f68800002a2000c7
:1060200060f688007023200070f6880000202000b1
:1060300080f68800301f200090f68800f0212000b4
:10604000a0f6880060252000b0f6880050292000c6
:10605000c0f68800302d2000d0f688009030200057
:10606000e0f6880030332000f0f68800d0352000bc
:1060700000f788001037200010f788003038200023
:1060800020f788005039200030f78800703a20004f
:1060900040f78800703b200050f78800303c20001b
:1060a00060f78800503c200070f78800d03b20004b
:1060b00080f78800e03a200090f7880080392000bf
:1060c000a0f78800e0372000b0f7880010362000e5
:1060d000c0f7880000342000d0f78800203320006b
:1060e000e0f78800f0322000f0f7880070332000dd
:1060f00000f888008034200010f888004036200026
:1061000020f888005039200030f88800703b2000cb
:1061100040f88800b03d200050f88800e03f2000a3
:1061200060f888003042200070f888007044200039
:1061300080f888006047200090f88800d048200050
:10614000a0f8880080492000b0f88800804920002d
:10615000c0f88800d0482000d0f8880060472000b0
:10616000e0f8880050452000f0f88800b041200099
:1061700000f98800503f200010f98800603d2000a1
:1061800020f98800d03b200030f98800f03a200048
:1061900040f98800b03a200050f98800a03b200068
:1061a00060f98800e03c200070f98800503e200033
:1061b00080f98800b03f200090f98800004120005d
:1061c000a0f9880000422000b0f988004043200078
:1061d000c0f98800b0432000d0f98800d0432000e7
:1061e000e0f9880090432000f0f988000043200087
:1061f00000fa88003042200010fa88004041200058
:1062000020fa8800a03f200030fa8800903e20004d
:1062100040fa8800903d200050fa8800c03c2000e1
:1062200060fa8800403c200070fa8800d03b2000d3
:1062300080fa8800a03b200090fa8800f03b200004
:10624000a0fa8800a03c2000b0fa8800c03d2000e1
:10625000c0fa8800403f2000d0fa8800f0402000bb
:10626000e0fa8800f0432000f0fa8800f0452000b2
:1062700000fb8800e047200010fb880090492000c8
:1062800020fb8800e04a200030fb8800904b200073
:1062900040fb8800104b200050fb8800b0492000d4
:1062a00060fb8800b047200070fb8800504520004c
:1062b00080fb8800f042200090fb8800b040200066
:1062c000a0fb8800903e2000b0fb8800d03b20005f
:1062d000c0fb8800303a2000d0fb8800c038200086
:1062e000e0fb8800c0372000f0fb8800103720005a
:1062f00000fc8800d036200010fc88000037200009
:1063000020fc88007037200030fc88000038200016
:1063100040fc8800b038200050fc88008039200004
:1063200060fc8800503a200070fc8800603b200030
:1063300080fc8800e03b200090fc8800403c20006e
:10634000a0fc8800603c2000b0fc8800303c2000ad
:10635000c0fc8800c03b2000d0fc8800203b20000f
:10636000e0fc8800e0392000f0fc8800d0382000f4
:1063700000fd8800d037200010fd88004037200045
:1063800020fd88000037200030fd88007037200095
:1063900040fd8800c039200050fd8800303c2000be
:1063a00060fd8800703f200070fd8800a043200041
:1063b00080fd88008048200090fd8800404e20002d
:1063c000a0fd880070582000b0fd880010602000fb
:1063d000c0fd880000682000d0fd8800d06f20003c
:1063e000e0fd880090762000f0fd8800d07a200043
:1063f00000fe88005079200010fe880010722000f6
:1064000020fe8800c066200030fe88001059200061
:1064100040fe8800004b200050fe8800003e200017
:1064200060fe88003033200070fe8800d0272000f6
:1064300080fe88009023200090fe8800002220002b
:10644000a0fe880080222000b0fe8800b02420003a
:10645000c0fe8800c0272000d0fe8800c02c20008d
:10646000e0fe8800b02f2000f0fe880010322000ef
:1064700000ff8800e033200010ff88003035200046
:1064800020ff88005036200030ff8800f0372000c1
:1064900040ff88001039200050ff8800303a20006b
:1064a00060ff8800303b200070ff8800e03b200048
:1064b00080ff8800303c200090ff8800003c2000d6
:1064c000a0ff8800c03a2000b0ff8800803920007b
:1064d000c0ff880020382000d0ff8800d036200080
:1064e000e0ff8800d0352000f0ff88002035200034
:1064f0000100220080087800f034200021002200f2
:1065000080087800a0352000410022008008780033
:10651000c03620006100220080087800703820001a
:106520008100220080087800703a2000a10022003b
:1065300080087800b03c2000c1002200800878006c
:1065400050402000e10022008008780080422000b6
:106550000101220080087800a044200021012200cf
:1065600080087800904620004101220080087800d1
:10657000f04720006101220080087800b048200028
:106580008101220080087800b0482000a10122008b
:106590008008780030472000c10122008008780080
:1065a00090452000e10122008008780090432000ff
:1065b00001022200800878006041200021022200b0
:1065c00080087800303f20004102220080087800d7
:1065d000203d20006102220080087800b03a2000af
:1065e0008102220080087800d0392000a102220018
:1065f0008008780090392000c102220080087800cd
:10660000e0392000e102220080087800c03a200032
:106610000103220080087800303c20002103220082
:1066200080087800d03e20004103220080087800d6
:106630009040200061032200800878002042200062
:10664000810322008008780050432000a10322002b
:106650008008780030442000c103220080087800c0
:10666000c0442000e103220080087800e0442000bc
:1066700001042200800878008044200021042200c8
:1066800080087800b0432000410422008008780090
:10669000a0422000610422008008780060412000b0
:1066a000810422008008780030402000a1042200ec
:1066b00080087800f03e2000c104220080087800a5
:1066c000403d2000e104220080087800703c20005a
:1066d0000105220080087800d03b2000210522001f
:1066e00080087800703b2000410522008008780077
:1066f000803b20006105220080087800d03b20000c
:106700008105220080087800003d2000a1052200bc
:1067100080087800503e2000c105220080087800e3
:1067200010402000e105220080087800e0412000b0
:106730000106220080087800c043200021062200c4
:1067400080087800a04520004106220080087800db
:10675000204820006106220080087800804920003f
:106760008106220080087800704a2000a1062200dd
:1067700080087800a04a2000c10622008008780026
:10678000e0492000e10622008008780070482000df
:10679000010722008008780080462000210722009f
:1067a00080087800404320004107220080087800dc
:1067b000104120006107220080087800d03e2000b0
:1067c0008107220080087800a03c2000a107220059
:1067d00080087800a03a2000c107220080087800d5
:1067e000e0382000e10722008008780050372000c0
:1067f0000108220080087800d036200021082200fd
:1068000080087800d03620004108220080087800f7
:1068100050372000610822008008780010382000de
:10682000810822008008780010392000a108220089
:1068300080087800c03a2000c10822008008780053
:10684000e03b2000e108220080087800e03c2000c6
:106850000109220080087800d03d20002109220093
:1068600080087800903e20004109220080087800ce
:10687000003f20006109220080087800d03e2000ff
:106880008109220080087800103e2000a109220022
:1068900080087800f03c2000c109220080087800c0
:1068a000903b2000e109220080087800003a200097
:1068b000010a22008008780060382000210a2200a6
:1068c00080087800d0362000410a22008008780035
:1068d000c0342000610a2200800878004034200083
:1068e000810a22008008780080342000a10a22005a
:1068f00080087800d0352000c10a22008008780086
:10690000f0372000e10a220080087800c03a200019
:10691000010b220080087800f03f2000210b2200ac
:106920008008780000000600003e2000410b220095
:106930008008780040382000610b22008008780031
:1069400060342000810b220080087800203e200067
:10695000a10b220080087800b04b2000c10b220060
:106960008008780040512000e10b22008008780068
:1069700050512000010c22008008780010502000a7
:10698000210c220080087800f04f2000410c2200ea
:1069900080087800604f2000610c22008008780099
:1069a000404e2000810c220080087800304d2000ed
:1069b000a10c220080087800a04d2000c10c22000c
:1069c0008008780030502000e10c22008008780018
:1069d00020522000010d2200800878007054200011
:1069e000210d22008008780020562000410d220051
:1069f0008008780020582000610d2200800878006f
:106a000040592000810d220080087800e0592000c4
:106a1000a10d220080087800805c2000c10d2200ba
:106a20008008780090622000e10d22008008780044
:106a300090702000010e220080087800c07c2000a9
:106a4000210e220080087800e0742000410e220010
:106a500080087800d05e2000610e22008008780057
:106a600020542000810e22008008780080482000f9
:106a7000a10e22008008780030452000c10e2200bf
:106a800080087800403f2000e10e22008008780056
:106a9000c0372000010f220080087800a0322000bb
:106aa000210f220080087800b02c2000410f220026
:106ab00080087800e0272000610f2200800878001d
:106ac000401d2000810f2200800878003017200030
:106ad000a10f220080087800b0102000c10f220012
:106ae00080087800900f2000e10f220080087800d5
:106af0004010200001102200800878003012200091
:106b00002110220080087800c011200041102200ce
:106b100080087800900c2000611022008008780026
:106b2000e00e20008110220080087800202620003e
:106b3000a110220080087800c0312000c11022007e
:106b40008008780070372000e1102200800878006b
:106b5000003920000111220080087800503a2000fe
:106b60002111220080087800203d200041112200e0
:106b700080087800d03d2000611122008008780054
:106b8000f03d20008111220080087800103d200097
:106b9000a111220080087800c03f2000c11122000e
:106ba0008008780050422000e1112200800878001f
:106bb000c04420000112220080087800c046200056
:106bc0002112220080087800a046200041122200f5
:106bd000800878004045200061122200800878007b
:106be000904220008112220080087800804120001d
:106bf000a11222008008780040422000c112220029
:106c000080087800b0432000e1122200800878005c
:106c100070442000011322008008780050452000b5
:106c20002113220080087800304520004113220003
:106c300080087800604520006113220080087800f9
:106c4000e0452000811322008008780020452000c4
:106c5000a113220080087800a0442000c113220064
:106c60008008780050442000e1132200800878005a
:106c7000b04220000114220080087800404120002a
:106c80002114220080087800b04020004114220026
:106c900080087800104020006114220080087800ed
:106ca000203f20008114220080087800803f2000cf
:106cb000a11422008008780010412000c114220095
:106cc00080087800c0412000e1142200800878008c
:106cd000a04120000115220080087800b04020006b
:106ce0002115220080087800704020004115220004
:106cf000800878002041200061152200800878007b
:106d0000d0402000811522008008780060412000da
:106d1000a115220080087800a0412000c1152200a2
:106d200080087800b0422000e11522008008780039
:106d300010432000011622008008780070412000d6
:106d400021162200800878006040200041162200b1
:106d500080087800603f20006116220080087800db
:106d6000c03e20008116220080087800603d20008f
:106d7000a116220080087800603d2000c116220084
:106d800080087800303d2000e1162200800878005d
:106d9000003e20000117220080087800d03e20002d
:106da0002117220080087800003f200041172200b0
:106db00080087800403f200061172200800878009a
:106dc000003f20008117220080087800803f2000cb
:106dd000a11722008008780010402000c11722006f
:106de00080087800d03f2000e1172200800878005a
:106df000603e20000118220080087800103c20002e
:106e00002118220080087800a03a200041182200b2
:106e100080087800a03a20006118220080087800dd
:106e2000003b20008118220080087800103b2000e1
:106e3000a118220080087800e03a2000c118220042
:106e400080087800803a2000e1182200800878004d
:106e5000f03920000119220080087800103a200043
:106e60002119220080087800e03920004119220011
:106e700080087800703920006119220080087800ad
:106e8000703920008119220080087800403a2000e3
:106e9000a119220080087800703b2000c11922004f
:106ea00080087800b03b2000e119220080087800bb
:106eb000903b2000011a220080087800403b20000f
:106ec000211a220080087800203b2000411a22006d
:106ed00080087800d03b2000611a220080087800ea
:106ee000803d2000811a220080087800203f200089
:106ef000a11a22008008780010402000c11a220048
:106f000080087800d0402000e11a22008008780034
:106f100070412000011b22008008780030412000d1
:106f2000211b220080087800203f2000411b220006
:106f300080087800d0372000611b2200800878008c
:106f400040352000811b220080087800e0402000ae
:106f5000a11b220080087800b04b2000c11b22003a
:106f600080087800904f2000e11b22008008780004
:106f7000804f2000011c220080087800b04e2000c5
:106f8000211c220080087800b04e2000411c220005
:106f900080087800b04d2000611c22008008780035
:106fa000404c2000811c220080087800104c2000fa
:106fb000a11c220080087800a04d2000c11c2200e6
:106fc00080087800f04f2000e11c22008008780043
:106fd000b0512000011d22008008780020542000bc
:106fe000211d220080087800a0552000411d2200ac
:106ff0008008780080572000611d220080087800fa
:1070000050592000811d220080087800305b20004c
:10701000a11d220080087800d05d2000c11d220043
:107020008008780050642000e11d2200800878006c
:1070300020722000011e220080087800207d2000a0
:10704000211e22008008780040732000411e22008b
:107050008008780060612000611e220080087800ae
:10706000b0552000811e220080087800f04a2000e0
:10707000a11e22008008780090482000c11e220036
:107080008008780020412000e11e2200800878005e
:1070900070392000011f2200800878008034200011
:1070a000211f220080087800502e2000411f22005e
:1070b0008008780060282000611f22008008780086
:1070c000601d2000811f22008008780030162000fb
:1070d000a11f22008008780030102000c11f22006c
:1070e00080087800500e2000e11f22008008780000
:1070f000f00e20000120220080087800801120007e
:107100002120220080087800b011200041202200b8
:1071100080087800d00b20006120220080087800d1
:10712000700f20008120220080087800a028200015
:10713000a12022008008780090312000c120220088
:1071400080087800b0362000e12022008008780016
:10715000603720000121220080087800a03920003b
:107160002121220080087800203c200041212200bb
:1071700080087800603d20006121220080087800ae
:10718000603d20008121220080087800203d200001
:10719000a12122008008780080402000c121220027
:1071a0008008780040422000e12122008008780019
:1071b00080442000012222008008780050462000f0
:1071c000212222008008780030462000412222003f
:1071d0008008780070442000612222008008780036
:1071e000d042200081222200800878003042200016
:1071f000a122220080087800c0422000c122220083
:1072000080087800b0432000e12222008008780046
:1072100040442000012322008008780040452000df
:10722000212322008008780080452000412322008d
:107230008008780010462000612322008008780032
:1072400060462000812322008008780070452000dd
:10725000a123220080087800e0442000c1232200fe
:107260008008780030442000e12322008008780064
:107270007042200001242200800878001041200084
:107280002124220080087800c040200041242200f0
:1072900080087800b03f2000612422008008780038
:1072a000103f200081242200800878002040200028
:1072b000a12422008008780060412000c12422001f
:1072c00080087800f0412000e12422008008780046
:1072d000f04120000125220080087800f0402000c5
:1072e00021252200800878006040200041252200ee
:1072f00080087800b04020006125220080087800d6
:10730000504020008125220080087800e0402000c5
:10731000a125220080087800e0412000c12522003c
:1073200080087800f0422000e125220080087800e3
:10733000004320000126220080087800a0412000a0
:10734000212622008008780090402000412622005b
:1073500080087800c03f2000612622008008780065
:10736000003f20008126220080087800203e200077
:10737000a126220080087800c03d2000c1262200fe
:1073800080087800803d2000e126220080087800f7
:10739000d03d20000127220080087800703e2000a8
:1073a0002127220080087800e03e200041272200ab
:1073b00080087800f03e20006127220080087800d5
:1073c000d03e20008127220080087800003f200066
:1073d000a127220080087800b03f2000c1272200aa
:1073e00080087800e03f2000e12722008008780034
:1073f000603e20000128220080087800403c2000e8
:107400002128220080087800a03a2000412822008c
:1074100080087800003b2000612822008008780066
:10742000103b20008128220080087800903a20003c
:10743000a128220080087800f0392000c12822000d
:1074400080087800b0392000e12822008008780008
:10745000603920000129220080087800b03920001e
:107460002129220080087800c0392000412922000b
:1074700080087800503920006129220080087800b7
:10748000f03920008129220080087800003b20008c
:10749000a129220080087800103c2000c129220088
:1074a00080087800803c2000e129220080087800d4
:1074b000603c2000012a220080087800e03b200088
:1074c000212a220080087800a03b2000412a2200c7
:1074d00080087800303c2000612a22008008780073
:1074e000c03d2000812a220080087800d03e200084
:1074f000a12a220080087800c03f2000c12a220073
:1075000080087800a0402000e12a2200800878004e
:10751000e0402000012b220080087800803f2000fe
:10752000212b220080087800a03b2000412b220064
:107530008008780000342000612b22008008780049
:1075400000362000812b220080087800c0462000f1
:10755000a12b220080087800704c2000c12b220053
:1075600080087800a0502000e12b220080087800dd
:10757000e04f2000012c220080087800804f20007e
:10758000212c220080087800504f2000412c22003e
:1075900080087800d04c2000612c22008008780000
:1075a000904b2000812c220080087800b04b2000f6
:1075b000a12c220080087800104e2000c12c22004f
:1075c0008008780020502000e12c220080087800fc
:1075d000b0522000012d220080087800f0542000d5
:1075e000212d22008008780070562000412d2200b5
:1075f0008008780090582000612d220080087800d3
:10760000305a2000812d220080087800605c200024
:10761000a12d220080087800b05f2000c12d22003b
:107620008008780000682000e12d220080087800a2
:10763000b0762000012e220080087800f07f200024
:10764000212e220080087800806e2000412e22002a
:1076500080087800e05b2000612e2200800878001e
:1076600060512000812e22008008780020462000f2
:10767000a12e22008008780090482000c12e220010
:1076800080087800a03e2000e12e220080087800cb
:1076900030392000012f220080087800603320005c
:1076a000212f220080087800302d2000412f220059
:1076b0008008780090262000612f22008008780042
:1076c000c01c2000812f220080087800b016200006
:1076d000a12f220080087800d0102000c12f2200a6
:1076e00080087800700f2000e12f220080087800c9
:1076f000e00f200001302200800878007011200087
:107700002130220080087800800f200041302200c4
:1077100080087800a00a20006130220080087800ec
:10772000c01320008130220080087800302f200014
:10773000a130220080087800f0342000c1302200ff
:107740008008780040392000e1302200800878006d
:10775000a03a20000131220080087800403a200041
:107760002131220080087800d03b200041312200e6
:1077700080087800203c20006131220080087800d9
:10778000703c20008131220080087800103d2000ec
:10779000a13122008008780090402000c1312200f1
:1077a0008008780060422000e131220080087800e3
:1077b0001045200001322200800878001047200088
:1077c00021322200800878006046200041322200e9
:1077d0008008780060442000613222008008780030
:1077e000c0422000813222008008780090412000b1
:1077f000a132220080087800a0422000c13222007d
:1078000080087800f0432000e132220080087800f0
:10781000b04420000133220080087800d0452000c9
:1078200021332200800878000046200041332200e6
:1078300080087800804620006133220080087800ac
:107840002046200081332200800878003045200047
:10785000a133220080087800d0442000c1332200e8
:107860008008780000442000e1332200800878007e
:10787000e04120000134220080087800f040200020
:10788000213422008008780020402000413422006a
:1078900080087800503f2000613422008008780082
:1078a000f03e20008134220080087800a03f2000b4
:1078b000a134220080087800f0402000c13422006a
:1078c00080087800b0412000e13422008008780070
:1078d000b04120000135220080087800c04020001f
:1078e0002135220080087800d04020004135220058
:1078f00080087800d04020006135220080087800a0
:10790000504020008135220080087800204120006e
:10791000a13522008008780010422000c1352200e5
:107920008008780050432000e1352200800878006c
:1079300000432000013622008008780030412000fa
:107940002136220080087800a04020004136220025
:1079500080087800104020006136220080087800fe
:10796000503f20008136220080087800303e200001
:10797000a136220080087800b03d2000c1362200e8
:1079800080087800d03d2000e13622008008780091
:10799000503e20000137220080087800003f200080
:1079a0002137220080087800003f20004137220064
:1079b00080087800503f200061372200800878005e
:1079c000403f20008137220080087800003f2000df
:1079d000a137220080087800703f2000c1372200c4
:1079e00080087800603f2000e1372200800878009e
:1079f000f03d20000138220080087800f03b200094
:107a00002138220080087800e03a20004138220026
:107a100080087800f03a2000613822008008780061
:107a2000703a20008138220080087800c039200098
:107a3000a138220080087800c0392000c138220017
:107a40008008780010392000e13822008008780092
:107a5000403920000139220080087800c039200018
:107a60002139220080087800c039200041392200e5
:107a70008008780060392000613922008008780091
:107a8000603a20008139220080087800a03b200065
:107a9000a139220080087800603c2000c139220012
:107aa00080087800203d2000e1392200800878001d
:107ab000203d2000013a220080087800703c200020
:107ac000213a220080087800f03b2000413a220051
:107ad00080087800703c2000613a2200800878001d
:107ae000a03d2000813a220080087800b03e2000ae
:107af000a13a220080087800403f2000c13a2200cd
:107b00008008780050402000e13a22008008780088
:107b1000f03f2000013b220080087800e03d20007b
:107b2000213b220080087800b0372000413b220032
:107b300080087800c0332000613b22008008780074
:107b4000e03c2000813b220080087800404a200071
:107b5000a13b220080087800704e2000c13b22002b
:107b600080087800704f2000e13b220080087800f8
:107b7000104f2000013c220080087800004f2000b8
:107b8000213c220080087800d04d2000413c22009a
:107b900080087800104c2000613c220080087800aa
:107ba000204c2000813c220080087800204d2000dd
:107bb000a13c220080087800904f2000c13c2200a8
:107bc00080087800e0502000e13c22008008780026
:107bd00040532000013d220080087800105520000d
:107be000213d22008008780080562000413d22007f
:107bf0008008780030582000613d2200800878001d
:107c0000205a2000813d220080087800a05c2000de
:107c1000a13d22008008780030622000c13d220092
:107c200080087800a06c2000e13d220080087800e8
:107c3000807a2000013e220080087800107a20001f
:107c4000213e22008008780040662000413e22004c
:107c50008008780070582000613e2200800878007b
:107c6000004e2000813e220080087800b0472000ae
:107c7000a13e22008008780070432000c13e22000f
:107c800080087800a03a2000e13e220080087800b9
:107c900050352000013f220080087800702f20001e
:107ca000213f220080087800a02d2000413f2200c3
:107cb0008008780030242000613f2200800878008e
:107cc000201b2000813f220080087800e013200064
:107cd000a13f220080087800700f2000c13f2200e1
:107ce00080087800c00e2000e13f22008008780064
:107cf000f00f20000140220080087800a00e200034
:107d000021402200800878007008200041402200b5
:107d100080087800d00d20006140220080087800a3
:107d2000e02720008140220080087800e030200019
:107d3000a14022008008780030362000c140220097
:107d400080087800f0362000e140220080087800aa
:107d5000e03920000141220080087800903b20009b
:107d60002141220080087800c03c200041412200cf
:107d700080087800603c2000614122008008780083
:107d8000c03c20008141220080087800203f200074
:107d9000a14122008008780090402000c1412200cb
:107da00080087800c0432000e1412200800878006c
:107db000904520000142220080087800a046200063
:107dc0002142220080087800104520004142220014
:107dd000800878004043200061422200800878003b
:107de000f0412000814222008008780000422000fb
:107df000a142220080087800d0432000c142220026
:107e00008008780030442000e14222008008780099
:107e1000604520000143220080087800c045200012
:107e200021432200800878000046200041432200c0
:107e300080087800404620006143220080087800d6
:107e4000404520008143220080087800b044200093
:107e5000a14322008008780060442000c143220032
:107e60008008780080422000e143220080087800ea
:107e7000504120000144220080087800804020000a
:107e80002144220080087800903f200041442200d5
:107e900080087800d03e20006144220080087800ed
:107ea000303f2000814422008008780050402000ac
:107eb000a14422008008780030412000c144220003
:107ec00080087800a0412000e1442200800878006a
:107ed000604120000145220080087800f040200029
:107ee0002145220080087800f04020004145220012
:107ef0008008780000412000614522008008780059
:107f0000b040200081452200800878009041200088
:107f1000a14522008008780090422000c14522003f
:107f20008008780030432000e14522008008780076
:107f30004042200001462200800878008040200056
:107f4000214622008008780030402000414622006f
:107f500080087800f03f2000614622008008780009
:107f6000403f20008146220080087800403e2000eb
:107f7000a146220080087800d03d2000c1462200a2
:107f800080087800803d2000e146220080087800cb
:107f9000203e20000147220080087800d03e2000cb
:107fa0002147220080087800f03e2000414722004f
:107fb00080087800403f2000614722008008780058
:107fc000c03e20008147220080087800d03e20007b
:107fd000a147220080087800a03e2000c14722006f
:107fe00080087800603e2000e14722008008780089
:107ff000b03c20000148220080087800503b20005f
:108000002148220080087800f03a200041482200f0
:1080100080087800a03a200061482200800878009b
:10802000703a20008148220080087800003a200041
:10803000a148220080087800103a2000c1482200a0
:1080400080087800b0392000e148220080087800dc
:10805000f03920000149220080087800503a2000c1
:108060002149220080087800d039200041492200af
:10807000800878009039200061492200800878004b
:10808000803a20008149220080087800703b20005f
:10809000a149220080087800603c2000c1492200ec
:1080a00080087800403d2000e149220080087800e7
:1080b000503d2000014a220080087800c03c20008a
:1080c000214a220080087800003d2000414a220019
:1080d00080087800a03d2000614a220080087800d6
:1080e000303f2000814a2200800878004040200074
:1080f000a14a220080087800d0402000c14a220016
:108100008008780090412000e14a22008008780031
:1081100090402000014b220080087800f03f2000b2
:10812000214b22008008780000000600a272ef00b8
:10813000b0d2bf00a252e30009003e000080200040
:10814000212a2100914078008180fb00818040003d
:10815000424b220080307900a272ec00f4ff39001b
:10816000b052ec00a2f2b700f0c7b300a252e30095
:1081700009003e00a2d2bf000080fb000000d0003a
:10818000414b22000100400001002000010878005e
:10819000a272ec00f4ff390000c8b300a2f2b700ed
:1081a000a2d2bf000080fb0001f82f0001064000b2
:1081b0000c064600404b220060007e00212a210070
:1081c000914078008180fb0081804000424b22007a
:1081d00080307900a272ec00f1ff3900404b2200a0
:1081e0000008eb0010c0b300a2f2b700a2d2bf009b
:1081f0000080fb000006e9000c064600404b220010
:1082000060007e006700b800b08f8800a2d2bf0077
:108210000080fb0000004000414b2200608078009d
:10822000f611b4004300de00212a210091407800bd
:108230008180fb0081804000424b22008030790029
:10824000a272ec00e9ff3900000006007041200036
:10825000416b220080087800b0442000616b22004e
:1082600080087800a04a2000816b220080087800f6
:10827000c0512000a16b2200800878002056200009
:10828000c16b220080087800705f2000e16b220043
:1082900080087800206a2000016c220080087800a5
:1082a00010722000216c220080087800907b200052
:1082b000416c220080087800607e2000616c220002
:1082c00080087800707d2000816c22008008780092
:1082d000a0782000a16c220080087800d0782000cf
:1082e000c16c22008008780000762000e16c22003a
:1082f0008008780040762000016d22008008780018
:10830000e0732000216d220080087800e06e2000dc
:10831000416d220080087800306b2000616d2200e2
:108320008008780000682000816d220080087800b5
:1083300040672000a16d220080087800b063200013
:10834000c16d220080087800205f2000e16d2200ce
:1083500080087800c0572000016e22008008780055
:10836000f0542000216e2200800878004050200048
:10837000416e220080087800204b2000616e2200b0
:1083800080087800b0462000816e220080087800c6
:10839000603b2000a16e22008008780000302000a1
:1083a000c16e22008008780010292000e16e2200b2
:1083b00080087800f0242000016f220080087800f7
:1083c00040232000216f2200800878002024200014
:1083d000416f220080087800a0232000616f2200f6
:1083e0008008780060222000816f220080087800d9
:1083f000a0232000a16f220080087800c025200063
:10840000c16f22008008780010292000e16f22004f
:1084100080087800602b200001702200800878001e
:10842000b02c20002170220080087800f02c200061
:108430004170220080087800d02b2000617022005b
:1084400080087800702a200081702200800878005f
:10845000b0282000a170220080087800502620005b
:10846000c17022008008780050242000e1702200b2
:1084700080087800d0222000017122008008780056
:108480006022200021712200800878000023200053
:1084900041712200800878000024200061712200d0
:1084a0008008780040252000817122008008780033
:1084b000f0262000a17122008008780050292000b9
:1084c000c171220080087800402b2000e171220059
:1084d00080087800f02f20000172220080087800c8
:1084e000d03320002172220080087800f03620006e
:1084f0004172220080087800c03a20006172220098
:1085000080087800f03c200081722200800878000a
:10851000303e2000a1722200800878001040200028
:10852000c172220080087800803f2000e1722200a2
:1085300080087800f03e2000017322008008780057
:10854000603e20002173220080087800103c20004b
:108550004173220080087800903a20006173220065
:10856000800878009038200081732200800878000d
:10857000f0352000a17322008008780070332000bd
:10858000c173220080087800c0302000e17322000f
:1085900080087800102e20000174220080087800e6
:1085a000302d20002174220080087800902c2000bb
:1085b0004174220080087800802c20006174220021
:1085c00080087800a02c20008174220080087800a8
:1085d000d02c2000a174220080087800102e2000ea
:1085e000c17422008008780080302000e1742200ed
:1085f000800878007034200001752200800878001f
:10860000403820002175220080087800e03a2000e0
:1086100041752200800878003040200061752200fa
:1086200080087800e04420008175220080087800ee
:1086300090472000a175220080087800504b200050
:10864000c175220080087800a04e2000e17522004c
:1086500080087800c0502000017622008008780051
:10866000d05220002176220080087800205420007b
:108670004176220080087800205420006176220094
:1086800080087800a05320008176220080087800be
:1086900040532000a176220080087800705220000c
:1086a000c176220080087800c0502000e1762200c8
:1086b00080087800a04f2000017722008008780011
:1086c000b04d20002177220080087800a04c2000c7
:1086d0004177220080087800404a2000617722001c
:1086e00080087800204920008177220080087800e7
:1086f000b0472000a1772200800878006045200064
:10870000c17722008008780020452000e177220010
:1087100080087800704420000178220080087800ea
:108720000044200021782200800878006042200068
:108730004178220080087800904020006178220073
:1087400080087800603d2000817822008008780051
:10875000c03a2000a178220080087800003720006d
:10876000c178220080087800a0322000e178220041
:1087700080087800303120000179220080087800dc
:10878000b02d20002179220080087800302b2000b5
:108790004179220080087800302a20006179220087
:1087a00080087800a02820008179220080087800c5
:1087b000b0282000a17922008008780090282000ad
:1087c000c17922008008780040292000e179220048
:1087d00080087800f0292000017a220080087800c3
:1087e000d02b2000217a220080087800402d200024
:1087f000417a220080087800f02e2000617a220061
:108800008008780010312000817a220080087800ea
:10881000f0322000a17a220080087800f034200095
:10882000c17a220080087800c0382000e17a220056
:1088300080087800903b2000017b220080087800af
:10884000603f2000217b2200800878000043200048
:10885000417b22008008780040452000617b220097
:108860008008780080492000817b22008008780001
:10887000b0512000a17b22008008780060572000c2
:10888000c17b220080087800b0612000e17b2200db
:1088900080087800806b2000017c2200800878002e
:1088a00070722000217c220080087800e07a20008d
:1088b000417c220080087800a07d2000617c22009d
:1088c00080087800807d2000817c2200800878006c
:1088d000d0792000a17c220080087800607a2000f6
:1088e000c17c220080087800c0762000e17c220054
:1088f0008008780080752000017d220080087800c3
:1089000080732000217d220080087800006e200006
:10891000417d220080087800806d2000617d22006a
:1089200080087800f0682000817d220080087800af
:1089300070662000a17d220080087800b0622000cf
:10894000c17d220080087800405e2000e17d220089
:108950008008780090582000017e2200800878006e
:1089600000562000217e2200800878003050200030
:10897000417e22008008780090482000617e22001d
:1089800080087800e0422000817e22008008780084
:1089900060352000a17e220080087800402e200053
:1089a000c17e220080087800a0252000e17e220000
:1089b0008008780050242000017f22008008780081
:1089c000d0232000217f220080087800d0232000bf
:1089d000417f22008008780010232000617f220060
:1089e0008008780010222000817f22008008780013
:1089f00020242000a17f220080087800002620008b
:108a0000c17f220080087800b02b2000e17f220087
:108a100080087800202d2000018022008008780046
:108a2000a02d20002180220080087800c02d200089
:108a30004180220080087800002c20006180220004
:108a400080087800302b2000818022008008780088
:108a5000d0282000a180220080087800b0252000c6
:108a6000c18022008008780020232000e1802200bd
:108a700080087800d0212000018122008008780041
:108a8000302120002181220080087800402220002f
:108a9000418122008008780050232000618122005b
:108aa00080087800a02420008181220080087800be
:108ab000a0262000a181220080087800d029200073
:108ac000c181220080087800402b2000e181220033
:108ad0008008780030302000018222008008780071
:108ae0004033200021822200800878006037200077
:108af0004182220080087800403b200061822200f1
:108b000080087800903d2000818222008008780053
:108b1000303e2000a182220080087800103f200013
:108b2000c182220080087800f03f2000e18222000c
:108b300080087800803f20000183220080087800b0
:108b4000a03e20002183220080087800503d2000b4
:108b50004183220080087800203b200061832200ae
:108b600080087800103a2000818322008008780075
:108b700050362000a18322008008780000332000b6
:108b8000c18322008008780000302000e1832200a9
:108b900080087800b02d2000018422008008780031
:108ba000702c20002184220080087800202c2000d6
:108bb0004184220080087800f02b2000618422008c
:108bc00080087800502b20008184220080087800e3
:108bd000d02c2000a184220080087800a02f200043
:108be000c18422008008780030322000e184220015
:108bf00080087800b03520000185220080087800c8
:108c0000903820002185220080087800f03b200069
:108c10004185220080087800904020006185220074
:108c200080087800a0452000818522008008780017
:108c300010492000a185220080087800f04c200017
:108c4000c185220080087800204f2000e1852200a5
:108c500080087800d051200001862200800878002a
:108c6000c053200021862200800878006054200034
:108c700041862200800878009054200061862200fe
:108c800080087800e0532000818622008008780068
:108c900010532000a1862200800878003051200067
:108ca000c186220080087800304f2000e186220033
:108cb00080087800c04e20000187220080087800dc
:108cc000204d20002187220080087800204c2000c1
:108cd0004187220080087800c04920006187220077
:108ce00080087800a0472000818722008008780053
:108cf000b0462000a187220080087800204620008e
:108d0000c18722008008780070452000e18722009a
:108d100080087800804420000188220080087800c4
:108d2000b042200021882200800878000041200005
:108d30004188220080087800503f2000618822008e
:108d400080087800003d200081882200800878009b
:108d5000c03b2000a188220080087800a0362000b7
:108d6000c18822008008780010322000e1882200ab
:108d700080087800802f2000018922008008780078
:108d8000b02c20002189220080087800b02b200020
:108d90004189220080087800f029200061892200a2
:108da00080087800602920008189220080087800ee
:108db00030292000a18922008008780000292000a5
:108dc000c189220080087800702a2000e1892200f1
:108dd00080087800a02a2000018a220080087800fc
:108de000102c2000218a220080087800a02d20006d
:108df000418a220080087800902f2000618a22009a
:108e000080087800c0312000818a22008008780024
:108e1000e0322000a18a220080087800b0352000ce
:108e2000c18a22008008780010382000e18a2200e0
:108e300080087800f03a2000018b2200800878003a
:108e4000a03f2000218b2200800878007043200082
:108e5000418b22008008780060462000618b220050
:108e600080087800204b2000818b22008008780049
:108e7000e0512000a18b220080087800905720004c
:108e8000c18b220080087800f0602000e18b220076
:108e900080087800b0692000018c220080087800ea
:108ea00030742000218c220080087800a07c2000f3
:108eb000418c220080087800f07f2000618c220025
:108ec00080087800e07c2000818c220080087800f7
:108ed00000772000a18c22008008780040792000d3
:108ee000c18c22008008780090762000e18c22005e
:108ef00080087800f0772000018d2200800878003b
:108f0000d0752000218d220080087800f06e2000ae
:108f1000418d220080087800e06d2000618d2200e4
:108f200080087800f0682000818d22008008780099
:108f300030672000a18d2200800878006063200047
:108f4000c18d220080087800f05e2000e18d2200b3
:108f50008008780010592000018e220080087800d7
:108f6000a0552000218e220080087800904e20001d
:108f7000418e22008008780080492000618e220006
:108f800080087800d03f2000818e22008008780081
:108f900010322000a18e220080087800202b2000b3
:108fa000c18e22008008780040242000e18e22003b
:108fb00080087800e0232000018f220080087800dc
:108fc000f0232000218f22008008780060242000f8
:108fd000418f22008008780000232000618f22004a
:108fe0008008780010232000818f220080087800fc
:108ff00060262000a18f220080087800b028200081
:10900000c18f220080087800602d2000e18f2200af
:1090100080087800f02d2000019022008008780060
:10902000102f20002190220080087800f02d2000d1
:109030004190220080087800e02c200061902200fe
:1090400080087800702b2000819022008008780032
:10905000b0272000a1902200800878000026200080
:10906000c19022008008780000222000e1902200b8
:1090700080087800e020200001912200800878001c
:10908000202020002191220080087800302120003b
:109090004191220080087800e022200061912200a6
:1090a0008008780040242000819122008008780008
:1090b00000262000a19122008008780020292000ad
:1090c000c191220080087800902a2000e1912200be
:1090d00080087800b03020000192220080087800db
:1090e000303320002192220080087800e0382000f0
:1090f0004192220080087800303c200061922200da
:1091000080087800c03d200081922200800878000d
:10911000603f2000a192220080087800704020006b
:10912000c19222008008780000412000e1922200d4
:1091300080087800a03f200001932200800878007a
:10914000f03f20002193220080087800903d20000d
:109150004193220080087800503a20006193220059
:109160008008780070382000819322008008780001
:1091700080342000a1932200800878004032200033
:10918000c193220080087800b0302000e1932200d3
:1091900080087800d02e20000194220080087800fa
:1091a000f02c20002194220080087800502c200010
:1091b0004194220080087800a02b200061942200b6
:1091c00080087800b02b200081942200800878006d
:1091d000f02c2000a194220080087800b02f2000fd
:1091e000c19422008008780070322000e1942200af
:1091f00080087800b03520000195220080087800b2
:10920000b03920002195220080087800303d2000f0
:109210004195220080087800d0412000619522000d
:1092200080087800d04420008195220080087800d2
:10923000e0482000a195220080087800404d2000e1
:10924000c195220080087800a04f2000e1952200ff
:1092500080087800c0522000019622008008780023
:10926000705420002196220080087800705420005d
:109270004196220080087800605420006196220008
:1092800080087800605320008196220080087800d2
:10929000c0522000a19622008008780020512000b2
:1092a000c196220080087800e04f2000e19622005d
:1092b00080087800b04e20000197220080087800d6
:1092c000304c20002197220080087800304b20008d
:1092d00041972200800878002049200061972200f1
:1092e00080087800c047200081972200800878001d
:1092f00060472000a19722008008780020462000c7
:10930000c19722008008780020452000e1972200c4
:1093100080087800d043200001982200800878005f
:10932000b04220002198220080087800904120005f
:1093300041982200800878000040200061982200b7
:1093400080087800503c2000819822008008780036
:1093500060392000a198220080087800e0352000c4
:10936000c19822008008780060322000e198220035
:1093700080087800203020000199220080087800c1
:10938000702e20002199220080087800302c2000c7
:109390004199220080087800b02a200061992200bb
:1093a00080087800702a20008199220080087800c7
:1093b00090292000a199220080087800c02920006f
:1093c000c199220080087800a0292000e19922009c
:1093d00080087800e02a2000019a220080087800a6
:1093e000c02c2000219a220080087800d02d200077
:1093f000419a22008008780050302000619a2200b3
:109400008008780030322000819a2200800878009d
:10941000b0332000a19a2200800878005035200047
:10942000c19a220080087800e0372000e19a2200eb
:1094300080087800f03a2000019b22008008780024
:10944000903f2000219b22008008780030442000bb
:10945000419b22008008780030472000619b220059
:1094600080087800204b2000819b22008008780033
:10947000a04f2000a19b220080087800a057200068
:10948000c19b22008008780000622000e19b22003e
:1094900080087800c0682000019c220080087800c5
:1094a00080732000219c220080087800507b2000df
:1094b000419c220080087800e07d2000619c220011
:1094c00080087800e07b2000819c220080087800e2
:1094d000007c2000a19c220080087800c079200038
:1094e000c19c22008008780000762000e19c2200c8
:1094f0008008780060772000019d220080087800b5
:1095000000732000219d2200800878001070200048
:10951000419d220080087800206e2000619d22007d
:1095200080087800606b2000819d22008008780010
:1095300060672000a19d220080087800c0622000a2
:10954000c19d220080087800a05f2000e19d2200dc
:1095500080087800e05b2000019e220080087800ef
:1095600050572000219e220080087800604f200084
:10957000419e220080087800f0482000619e220071
:1095800080087800f03b2000819e2200800878004f
:10959000502f2000a19e2200800878008029200002
:1095a000c19e220080087800e0242000e19e220075
:1095b0008008780090242000019f22008008780015
:1095c000d0222000219f220080087800f022200075
:1095d000419f22008008780050212000619f2200d6
:1095e00080087800e0222000819f22008008780017
:1095f00080272000a19f220080087800a02a200058
:10960000c19f220080087800402e2000e19f2200a8
:1096100080087800f02e200001a022008008780049
:10962000a02f200021a0220080087800a02e20007a
:1096300041a0220080087800902e200061a0220026
:1096400080087800402c200081a02200800878004b
:1096500090282000a1a02200800878003026200059
:10966000c1a022008008780040222000e1a0220052
:10967000800878009021200001a122008008780055
:109680003020200021a122008008780070212000d5
:1096900041a12200800878008021200061a12200e1
:1096a000800878006023200081a1220080087800d3
:1096b000b0242000a1a1220080087800802620008c
:1096c000c1a1220080087800c02a2000e1a1220068
:1096d000800878007030200001a222008008780005
:1096e000f033200021a2220080087800703820008a
:1096f00041a2220080087800903b200061a2220055
:1097000080087800603e200081a222008008780056
:10971000b03f2000a1a22200800878003041200044
:10972000c1a222008008780050402000e1a222005f
:1097300080087800c03e200001a322008008780045
:10974000903e200021a3220080087800803d200068
:1097500041a3220080087800e03b200061a32200a2
:1097600080087800403a200081a322008008780019
:1097700030362000a1a3220080087800b0312000fc
:10978000c1a3220080087800c02f2000e1a322009e
:1097900080087800e02d200001a4220080087800d5
:1097a000202d200021a4220080087800e02c200039
:1097b00041a4220080087800402b200061a42200f0
:1097c00080087800602b200081a4220080087800a7
:1097d000502c2000a1a4220080087800f02f200047
:1097e000c1a4220080087800f0312000e1a422000a
:1097f00080087800f035200001a52200800878005c
:109800002039200021a5220080087800f03d2000aa
:1098100041a5220080087800e042200061a52200d6
:10982000800878003045200081a52200800878005b
:10983000f0492000a1a5220080087800b04d20004a
:10984000c1a522008008780020502000e1a5220058
:1098500080087800e052200001a6220080087800ed
:109860002054200021a6220080087800f053200018
:1098700041a62200800878004054200061a6220002
:10988000800878008054200081a62200800878009b
:1098900020532000a1a622008008780070512000eb
:1098a000c1a622008008780010502000e1a6220006
:1098b00080087800a04d200001a7220080087800d1
:1098c000104b200021a7220080087800804a200049
:1098d00041a7220080087800f048200061a72200fc
:1098e000800878002048200081a7220080087800a6
:1098f000e0462000a1a7220080087800a0452000b3
:10990000c1a7220080087800e0442000e1a72200df
:1099100080087800a043200001a822008008780079
:109920002043200021a8220080087800c0412000a8
:1099300041a8220080087800d03f200061a82200c2
:1099400080087800f03b200081a822008008780081
:10995000e0392000a1a8220080087800003520000e
:10996000c1a8220080087800f0322000e1a822007f
:1099700080087800c02f200001a92200800878000c
:10998000d02d200021a9220080087800902c2000f2
:1099900041a9220080087800702b200061a92200d4
:1099a00080087800b02b200081a922008008780070
:1099b000c02a2000a1a9220080087800202a2000c7
:1099c000c1a9220080087800502a2000e1a92200c5
:1099d00080087800f02a200001aa22008008780080
:1099e000d02c200021aa220080087800102f20000f
:1099f00041aa2200800878002031200061aa2200bc
:109a000080087800d032200081aa220080087800e7
:109a1000d0332000a1aa22008008780090352000d1
:109a2000c1aa220080087800c0382000e1aa2200e4
:109a300080087800903a200001ab2200800878006e
:109a4000f03f200021ab22008008780000000600d3
:109a5000f03d200041ab220080087800c04020008b
:109a600061ab220080087800c043200081ab220057
:109a700080087800e0462000a1ab22008008780032
:109a8000204a2000c1ab220080087800804d2000d1
:109a9000e1ab220080087800b050200001ac220029
:109aa00080087800d053200021ac22008008780084
:109ab000e056200041ac220080087800b059200018
:109ac00061ac220080087800505c200081ac22004c
:109ad00080087800d05e2000a1ac220080087800c9
:109ae00070632000c1ac220080087800b0652000bf
:109af000e1ac2200800878002068200001ad22003f
:109b000080087800e06a200021ad220080087800fb
:109b1000806d200041ad2200800878005070200048
:109b200061ad2200800878004073200081ad2200e2
:109b30008008780020762000a1ad220080087800ff
:109b4000e0782000c1ad220080087800607b200012
:109b5000e1ad220080087800407d200001ae2200a7
:109b600080087800307e200021ae22008008780036
:109b7000007e200041ae220080087800a07c2000fa
:109b800061ae220080087800b079200081ae22000a
:109b90008008780070752000a1ae2200800878004f
:109ba00050702000c1ae220080087800506a20006a
:109bb000e1ae220080087800c063200001af2200df
:109bc00080087800f05c200021af22008008780037
:109bd0003056200041af220080087800b04f2000ae
:109be00061af220080087800a049200081af2200e8
:109bf0008008780030442000a1af2200800878005f
:109c0000703f2000c1af220080087800003820009b
:109c1000e1af2200800878005035200001b022001a
:109c2000800878001033200021b0220080087800de
:109c30004031200041b0220080087800b02f200081
:109c400061b0220080087800402e200081b0220000
:109c500080087800e02c2000a1b022008008780065
:109c6000a02b2000c1b0220080087800602a2000cc
:109c7000e1b02200800878004029200001b12200d4
:109c8000800878002028200021b122008008780078
:109c90000027200041b12200800878000026200023
:109ca00061b12200800878003025200081b12200b7
:109cb0008008780080242000a1b12200800878006c
:109cc00020242000c1b1220080087800f023200069
:109cd000e1b1220080087800f023200001b22200c8
:109ce000800878005024200021b2220080087800eb
:109cf0000025200041b222008008780000262000c4
:109d000061b22200800878005027200081b2220032
:109d10008008780000292000a1b222008008780085
:109d2000e02a2000c1b2220080087800d02c200058
:109d3000e1b2220080087800f030200001b3220058
:109d400080087800d032200021b3220080087800fb
:109d5000a034200041b32200800878004036200063
:109d600061b3220080087800b037200081b3220060
:109d700080087800e0382000a1b322008008780035
:109d8000f0392000c1b3220080087800e03a2000ba
:109d9000e1b3220080087800903b200001b422004b
:109da00080087800103c200021b422008008780050
:109db000603c200041b4220080087800a03c2000d4
:109dc00061b4220080087800c03c200081b42200e9
:109dd00080087800e03c2000a1b4220080087800d0
:109de000f03c2000c1b4220080087800f03c200044
:109df000e1b4220080087800f03c200001b5220088
:109e000080087800003d200021b5220080087800fd
:109e1000003d200041b5220080087800003d200070
:109e200061b5220080087800003d200081b5220045
:109e300080087800e03c2000a1b52200800878006e
:109e4000c03c2000c1b5220080087800803c200082
:109e5000e1b5220080087800303c200001b62200e5
:109e600080087800703b200021b62200800878002e
:109e7000103b200041b6220080087800c03a200044
:109e800061b6220080087800703a200081b6220076
:109e900080087800103a2000a1b6220080087800df
:109ea000c0392000c1b62200800878007039200037
:109eb000e1b62200800878000039200001b72200b6
:109ec00080087800a038200021b7220080087800a0
:109ed0002038200041b7220080087800a0372000f9
:109ee00061b72200800878001037200081b7220077
:109ef0008008780050362000a1b722008008780042
:109f000090352000c1b7220080087800a0342000de
:109f1000e1b72200800878009033200001b82200c9
:109f2000800878007032200021b822008008780074
:109f30005031200041b822008008780020302000f5
:109f400061b8220080087800102f200081b822001c
:109f500080087800102e2000a1b822008008780028
:109f6000302d2000c1b8220080087800902c2000fd
:109f7000e1b8220080087800102c200001b92200ee
:109f800080087800d02b200021b9220080087800ba
:109f9000b02b200041b9220080087800e02b20007f
:109fa00061b9220080087800302c200081b922009d
:109fb00080087800902c2000a1b922008008780049
:109fc000002d2000c1b9220080087800802d2000db
:109fd000e1b9220080087800202e200001ba22007a
:109fe00080087800d02e200021ba22008008780056
:109ff000a02f200041ba2200800878009030200075
:10a0000061ba220080087800b031200081ba2200b5
:10a010008008780000332000a1ba22008008780070
:10a02000b0342000c1ba220080087800a036200099
:10a03000e1ba220080087800b038200001bb22007d
:10a0400080087800103b200021bb220080087800a7
:10a05000a03d200041bb2200800878007040200015
:10a0600061bb2200800878006043200081bb220091
:10a070008008780070462000a1bb2200800878008c
:10a0800080492000c1bb220080087800a04c20003d
:10a09000e1bb220080087800c04f200001bc2200f4
:10a0a00080087800f052200021bc2200800878004f
:10a0b000f055200041bc220080087800505b200051
:10a0c00061bc220080087800c05d200081bc2200b5
:10a0d0008008780010602000a1bc22008008780071
:10a0e00050622000c1bc22008008780080642000fb
:10a0f000e1bc220080087800c066200001bd22007b
:10a10000800878003069200021bd22008008780096
:10a11000c06b200041bd220080087800906e2000b6
:10a1200061bd220080087800a071200081bd22005e
:10a130008008780090742000a1bd2200800878007b
:10a1400070772000c1bd220080087800207a2000ae
:10a15000e1bd220080087800407c200001be220082
:10a1600080087800907d200021be220080087800c1
:10a17000c07d200041be220080087800b07c200015
:10a1800061be220080087800407a200081be220053
:10a1900080087800b0762000a1be220080087800f8
:10a1a000f0712000c1be220080087800e06b200022
:10a1b000e1be2200800878009065200001bf2200e7
:10a1c00080087800f05e200021bf2200800878001f
:10a1d0003058200041bf220080087800c051200084
:10a1e00061bf2200800878003046200081bf220035
:10a1f0008008780070412000a1bf2200800878000c
:10a20000503d2000c1bf220080087800e0392000c6
:10a21000e1bf2200800878000037200001c0220042
:10a22000800878009034200021c022008008780047
:10a230008032200041c0220080087800d030200009
:10a2400061c0220080087800302f200081c02200e9
:10a2500080087800c02d2000a1c02200800878006e
:10a26000502c2000c1c0220080087800f02a200075
:10a27000e1c0220080087800a029200001c122004e
:10a28000800878006028200021c122008008780022
:10a290004027200041c1220080087800402620008d
:10a2a00061c12200800878005025200081c1220071
:10a2b0008008780090242000a1c122008008780046
:10a2c00010242000c1c1220080087800c023200093
:10a2d000e1c1220080087800b023200001c22200e2
:10a2e00080087800e023200021c222008008780046
:10a2f0006024200041c22200800878003025200020
:10a3000061c22200800878006026200081c22200fd
:10a310008008780090292000a1c2220080087800df
:10a32000702b2000c1c2220080087800802d200000
:10a33000e1c2220080087800702f200001c32200b3
:10a34000800878005031200021c322008008780066
:10a350001033200041c3220080087800b034200070
:10a3600061c32200800878003036200081c32200bb
:10a370008008780080372000a1c322008008780080
:10a38000a0382000c1c3220080087800a039200036
:10a39000e1c3220080087800703a200001c4220046
:10a3a00080087800203b200021c42200800878002b
:10a3b000b03b200041c4220080087800203c2000ef
:10a3c00061c4220080087800803c200081c4220003
:10a3d00080087800c03c2000a1c4220080087800da
:10a3e000003d2000c1c4220080087800203d2000ec
:10a3f000e1c4220080087800403d200001c5220011
:10a4000080087800503d200021c522008008780097
:10a41000603d200041c5220080087800603d20009a
:10a4200061c5220080087800603d200081c52200bf
:10a4300080087800503d2000a1c5220080087800e7
:10a44000203d2000c1c5220080087800e03c2000ab
:10a45000e1c5220080087800a03c200001c622004f
:10a4600080087800503c200021c622008008780037
:10a47000103c200041c6220080087800c03b20002c
:10a4800061c6220080087800803b200081c622003f
:10a4900080087800303b2000a1c6220080087800a8
:10a4a000e03a2000c1c6220080087800703a2000ff
:10a4b000e1c6220080087800003a200001c722008f
:10a4c000800878008039200021c7220080087800a9
:10a4d000e038200041c72200800878003038200092
:10a4e00061c72200800878006037200081c7220001
:10a4f0008008780080362000a1c7220080087800fc
:10a5000080352000c1c72200800878007034200008
:10a51000e1c72200800878004033200001c82200f3
:10a52000800878000032200021c8220080087800ce
:10a53000c030200041c8220080087800702f200021
:10a5400061c8220080087800402e200081c82200c7
:10a5500080087800302d2000a1c8220080087800f3
:10a56000502c2000c1c8220080087800102b200049
:10a57000e1c8220080087800b02a200001c922002a
:10a5800080087800902a200021c9220080087800e5
:10a59000a02a200041c9220080087800d02a20008b
:10a5a00061c9220080087800202b200081c9220088
:10a5b00080087800902b2000a1c922008008780034
:10a5c000102c2000c1c9220080087800a02c200097
:10a5d000e1c9220080087800502d200001ca220025
:10a5e00080087800202e200021ca220080087800f0
:10a5f000002f200041ca220080087800003020008f
:10a6000061ca2200800878003031200081ca22000f
:10a610008008780090322000a1ca220080087800cb
:10a6200030342000c1ca2200800878001036200093
:10a63000e1ca2200800878004038200001cb2200c7
:10a6400080087800c03a200021cb220080087800e2
:10a65000503d200041cb22008008780010402000af
:10a6600061cb220080087800f042200081cb2200dc
:10a670008008780000462000a1cb220080087800e6
:10a6800010492000c1cb220080087800304c200007
:10a69000e1cb2200800878006052200001cc22002b
:10a6a000800878005055200021cc220080087800d6
:10a6b0003058200041cc220080087800005b200048
:10a6c00061cc220080087800905d200081cc2200bf
:10a6d0008008780000602000a1cc2200800878006b
:10a6e00050622000c1cc22008008780090642000d5
:10a6f000e1cc220080087800e066200001cd220035
:10a70000800878006069200021cd22008008780050
:10a71000006c200041cd220080087800d06e20001f
:10a7200061cd220080087800c071200081cd220018
:10a7300080087800c0742000a1cd22008008780035
:10a74000e0772000c1cd220080087800b07a200098
:10a75000e1cd220080087800f07c200001ce2200ac
:10a7600080087800607e200021ce220080087800da
:10a77000d07e200041ce220080087800007e20009c
:10a7800061ce220080087800e07b200081ce22008c
:10a790008008780080782000a1ce22008008780010
:10a7a000e0732000c1ce220080087800606e200097
:10a7b000e1ce2200800878002068200001cf22002e
:10a7c00080087800105a200021cf220080087800ed
:10a7d0006053200041cf220080087800304d2000d7
:10a7e00061cf2200800878008047200081cf2200be
:10a7f0008008780090422000a1cf220080087800d5
:10a80000403e2000c1cf220080087800a03a2000fe
:10a81000e1cf220080087800a037200001d022007c
:10a82000800878002035200021d0220080087800a0
:10a830000033200041d02200800878002031200021
:10a8400061d0220080087800502f200081d02200a3
:10a8500080087800c02d2000a1d022008008780058
:10a86000402c2000c1d0220080087800d02a20008f
:10a87000e1d02200800878007029200001d1220058
:10a88000800878001028200021d12200800878005c
:10a89000d026200041d1220080087800b025200079
:10a8a00061d1220080087800b024200081d12200ec
:10a8b00080087800e0232000a1d1220080087800e1
:10a8c00040232000c1d1220080087800d02220003f
:10a8d000e1d1220080087800c022200001d22200ad
:10a8e000800878000023200021d222008008780010
:10a8f0007024200041d2220080087800b02520007a
:10a9000061d22200800878003027200081d2220006
:10a910008008780000292000a1d222008008780059
:10a92000002b2000c1d2220080087800102d2000ca
:10a93000e1d2220080087800302f200001d32200cd
:10a94000800878005031200021d322008008780050
:10a950005033200041d322008008780010352000b9
:10a9600061d3220080087800b036200081d3220015
:10a970008008780020382000a1d3220080087800c9
:10a9800060392000c1d3220080087800703a20008e
:10a99000e1d3220080087800603b200001d422002f
:10a9a00080087800203c200021d422008008780014
:10a9b000b03c200041d4220080087800203d2000d7
:10a9c00061d4220080087800603d200081d42200fc
:10a9d00080087800a03d2000a1d4220080087800e3
:10a9e000c03d2000c1d4220080087800e03d200056
:10a9f000e1d4220080087800f03d200001d522003b
:10aa000080087800003e200021d5220080087800d0
:10aa1000f03d200041d5220080087800d03d200084
:10aa200061d5220080087800a03d200081d5220059
:10aa300080087800803d2000a1d5220080087800a1
:10aa4000603d2000c1d5220080087800303d200004
:10aa5000e1d5220080087800003d200001d62200c8
:10aa600080087800e03c200021d622008008780091
:10aa7000b03c200041d6220080087800803c2000b5
:10aa800061d6220080087800403c200081d6220058
:10aa900080087800003c2000a1d6220080087800c1
:10aaa000a03b2000c1d6220080087800203b200077
:10aab000e1d6220080087800a03a200001d72200c9
:10aac00080087800f039200021d722008008780023
:10aad0003039200041d7220080087800503820000b
:10aae00061d72200800878006037200081d72200db
:10aaf0008008780040362000a1d722008008780026
:10ab000010352000c1d7220080087800e0332000f3
:10ab1000e1d72200800878009032200001d822007e
:10ab2000800878005031200021d822008008780069
:10ab30001030200041d8220080087800e02e20004c
:10ab400061d8220080087800d02c200081d8220013
:10ab500080087800002c2000a1d82200800878000e
:10ab6000602b2000c1d8220080087800e02a200055
:10ab7000e1d8220080087800902a200001d9220024
:10ab800080087800602a200021d9220080087800ff
:10ab9000702a200041d9220080087800a02a2000d5
:10aba00061d9220080087800f02a200081d9220093
:10abb00080087800602b2000a1d92200800878004e
:10abc000e02b2000c1d9220080087800802c2000d2
:10abd000e1d9220080087800402d200001da22000f
:10abe00080087800102e200021da220080087800ea
:10abf000f02e200041da220080087800f02f20009b
:10ac000061da2200800878003031200081da2200e9
:10ac10008008780090322000a1da220080087800b5
:10ac200030342000c1da220080087800003620008d
:10ac3000e1da2200800878002038200001db2200c1
:10ac400080087800603a200021db2200800878002c
:10ac5000e03c200041db220080087800c03f20005b
:10ac600061db220080087800c042200081db2200e6
:10ac700080087800d0482000a1db220080087800fe
:10ac8000e04b2000c1db220080087800004f20004c
:10ac9000e1db2200800878000052200001dc220065
:10aca00080087800f054200021dc22008008780021
:10acb000d057200041dc220080087800805a200014
:10acc00061dc220080087800105d200081dc220019
:10acd00080087800805f2000a1dc220080087800d6
:10ace000f0612000c1dc2200800878004064200070
:10acf000e1dc220080087800a066200001dd22004f
:10ad0000800878003069200021dd2200800878006a
:10ad1000e06b200041dd220080087800c06e20003a
:10ad200061dd220080087800b071200081dd220002
:10ad300080087800c0742000a1dd2200800878001f
:10ad4000c0772000c1dd220080087800907a2000c2
:10ad5000e1dd220080087800f07c200001de220086
:10ad600080087800b07e200021de22008008780074
:10ad7000407f200041de220080087800907e200085
:10ad800061de220080087800a07c200081de2200a5
:10ad90008008780060792000a1de22008008780019
:10ada000a06f2000c1de22008008780080692000aa
:10adb000e1de220080087800e062200001df22004e
:10adc00080087800105c200021df220080087800d5
:10add0006055200041df220080087800b04e20003e
:10ade00061df220080087800b048200081df220067
:10adf0008008780090432000a1df220080087800be
:10ae0000203f2000c1df220080087800503b200056
:10ae1000e1df2200800878002038200001e02200d5
:10ae2000800878007035200021e02200800878003a
:10ae30001033200041e0220080087800103120000b
:10ae400061e0220080087800302f200081e022009d
:10ae500080087800702d2000a1e022008008780092
:10ae6000c02b2000c1e0220080087800202a2000aa
:10ae7000e1e0220080087800b028200001e12200f3
:10ae8000800878005027200021e122008008780007
:10ae90001026200041e122008008780000252000d3
:10aea00061e12200800878001024200081e1220066
:10aeb0008008780040232000a1e12200800878006b
:10aec000b0222000c1e1220080087800402220004a
:10aed000e1e12200800878006022200001e22200e7
:10aee00080087800e022200021e22200800878001b
:10aef000a023200041e2220080087800b024200036
:10af000061e22200800878000026200081e2220011
:10af10008008780090272000a1e2220080087800b5
:10af200060292000c1e2220080087800502b200018
:10af3000e1e2220080087800502d200001e3220089
:10af400080087800602f200021e32200800878002c
:10af50007031200041e32200800878006033200037
:10af600061e32200800878005035200081e3220050
:10af70008008780010372000a1e3220080087800c4
:10af800090382000c1e3220080087800e0392000da
:10af9000e1e3220080087800103b200001e4220059
:10afa00080087800003c200021e42200800878001e
:10afb000d03c200041e4220080087800803d200041
:10afc00061e4220080087800103e200081e4220025
:10afd00080087800803e2000a1e4220080087800ec
:10afe000d03e2000c1e4220080087800003f20000d
:10aff000e1e4220080087800303f200001e52200d3
:10b0000080087800403f200021e522008008780079
:10b01000403f200041e5220080087800303f2000ba
:10b0200061e5220080087800203f200081e52200b1
:10b0300080087800003f2000a1e522008008780009
:10b04000d03e2000c1e5220080087800903e20001c
:10b05000e1e5220080087800503e200001e6220051
:10b0600080087800003e200021e622008008780059
:10b07000b03d200041e6220080087800403d2000dd
:10b0800061e6220080087800e03c200081e6220092
:10b0900080087800703c2000a1e62200800878003b
:10b0a000003c2000c1e6220080087800803b2000a0
:10b0b000e1e6220080087800f03a200001e7220053
:10b0c00080087800403a200021e7220080087800bc
:10b0d0007039200041e72200800878009038200075
:10b0e00061e7220080087800a037200081e7220075
:10b0f0008008780090362000a1e7220080087800c0
:10b1000060352000c1e7220080087800203420004c
:10b11000e1e7220080087800d032200001e8220018
:10b12000800878004030200021e822008008780064
:10b13000f02e200041e8220080087800c02d200079
:10b1400061e8220080087800a02c200081e822001d
:10b1500080087800b02b2000a1e822008008780049
:10b16000e02a2000c1e8220080087800402a200060
:10b17000e1e8220080087800e029200001e92200af
:10b1800080087800b029200021e92200800878009a
:10b19000a029200041e9220080087800d029200061
:10b1a00061e9220080087800202a200081e922003d
:10b1b00080087800802a2000a1e922008008780019
:10b1c000f02a2000c1e9220080087800802b2000ae
:10b1d000e1e9220080087800302c200001ea2200fa
:10b1e00080087800002d200021ea220080087800e5
:10b1f000f02d200041ea220080087800102f200066
:10b2000061ea2200800878004030200081ea2200b4
:10b2100080087800a0312000a1ea22008008780090
:10b2200040332000c1ea2200800878000035200069
:10b23000e1ea2200800878000037200001eb2200bc
:10b24000800878004039200021eb22008008780037
:10b25000403e200041eb2200800878001041200091
:10b2600061eb2200800878000044200081eb22007e
:10b270008008780030472000a1eb22008008780089
:10b28000604a2000c1eb220080087800704d200049
:10b29000e1eb2200800878009050200001ec2200b1
:10b2a000800878009053200021ec2200800878006c
:10b2b0009056200041ec2200800878006059200060
:10b2c00061ec220080087800105c200081ec2200f4
:10b2d00080087800a05e2000a1ec220080087800a1
:10b2e00020612000c1ec22008008780090632000db
:10b2f000e1ec2200800878002066200001ed2200a9
:10b3000080087800d068200021ed220080087800b5
:10b31000a06b200041ed220080087800a06e200084
:10b3200061ed220080087800b071200081ed2200dc
:10b3300080087800d0742000a1ed220080087800f9
:10b34000e0772000c1ed220080087800d07a20004c
:10b35000e1ed220080087800507d200001ee2200ff
:10b3600080087800207f200021ee220080087800ed
:10b37000807f200041ee220080087800907d200030
:10b3800061ee220080087800707a200081ee2200b1
:10b390008008780000762000a1ee22008008780066
:10b3a000b0702000c1ee220080087800906a200072
:10b3b000e1ee220080087800f063200001ef220017
:10b3c00080087800205d200021ef220080087800ae
:10b3d0006056200041ef220080087800f04f2000e6
:10b3e00061ef220080087800204a200081ef2200cf
:10b3f00080087800e0442000a1ef22008008780057
:10b4000010402000c1ef220080087800403c20005e
:10b41000e1ef2200800878001039200001f02200be
:10b42000800878005036200021f022008008780043
:10b430000034200041f0220080087800f031200024
:10b4400061f02200800878002030200081f0220086
:10b4500080087800602e2000a1f02200800878008b
:10b46000b02c2000c1f0220080087800102b2000b2
:10b47000e1f02200800878008029200001f12200fc
:10b48000800878000028200021f122008008780040
:10b49000a026200041f122008008780060242000ce
:10b4a00061f12200800878008023200081f12200d1
:10b4b00080087800c0222000a1f1220080087800d6
:10b4c00050222000c1f122008008780000222000d4
:10b4d000e1f12200800878000022200001f2220021
:10b4e000800878005022200021f222008008780095
:10b4f000f022200041f2220080087800f023200092
:10b5000061f22200800878005025200081f222009c
:10b510008008780000272000a1f22200800878002f
:10b52000d0282000c1f2220080087800d02a200014
:10b53000e1f2220080087800e02c200001f32200d4
:10b5400080087800e02e200021f322008008780097
:10b55000e030200041f3220080087800b032200063
:10b5600061f32200800878006034200081f322001b
:10b5700080087800e0352000a1f3220080087800e0
:10b5800040372000c1f32200800878008038200076
:10b59000e1f32200800878008039200001f42200c5
:10b5a00080087800603a200021f4220080087800aa
:10b5b000203b200041f4220080087800c03b20009e
:10b5c00061f4220080087800a03c200081f4220071
:10b5d00080087800003d2000a1f422008008780057
:10b5e000503d2000c1f4220080087800903d2000ea
:10b5f000e1f4220080087800d03d200001f522000f
:10b6000080087800103e200021f522008008780094
:10b61000403e200041f5220080087800603e200076
:10b6200061f5220080087800803e200081f522002c
:10b6300080087800803e2000a1f522008008780074
:10b64000803e2000c1f5220080087800703e200076
:10b65000e1f5220080087800603e200001f622001b
:10b6600080087800303e200021f622008008780013
:10b67000103e200041f6220080087800d03d2000d6
:10b6800061f6220080087800903d200081f62200bb
:10b6900080087800303d2000a1f622008008780064
:10b6a000d03c2000c1f6220080087800703c2000c9
:10b6b000e1f6220080087800e03b200001f722003c
:10b6c00080087800403b200021f7220080087800a5
:10b6d000803a200041f7220080087800b03920002d
:10b6e00061f7220080087800c038200081f722002e
:10b6f00080087800a0362000a1f72200800878009a
:10b7000070352000c1f72200800878001034200036
:10b71000e1f7220080087800c032200001f8220002
:10b72000800878007031200021f82200800878001d
:10b730002030200041f8220080087800f02e200000
:10b7400061f8220080087800d02d200081f82200c6
:10b7500080087800e02c2000a1f822008008780002
:10b76000102c2000c1f8220080087800702b2000e7
:10b77000e1f8220080087800102b200001f9220057
:10b7800080087800c02a200021f922008008780073
:10b79000b02a200041f9220080087800d02a200039
:10b7a00061f9220080087800102b200081f9220026
:10b7b00080087800702b2000a1f922008008780012
:10b7c000f02b2000c1f9220080087800702c2000a6
:10b7d000e1f9220080087800202d200001fa2200e3
:10b7e00080087800d02d200021fa220080087800ff
:10b7f000b02e200041fa220080087800b02f2000ef
:10b8000061fa220080087800c030200081fa22000e
:10b810008008780010322000a1fa22008008780009
:10b8200040352000c1fa220080087800303720001f
:10b83000e1fa2200800878005039200001fb220044
:10b8400080087800a03b200021fb220080087800bf
:10b85000203e200041fb220080087800e0402000cc
:10b8600061fb220080087800b043200081fb2200a9
:10b8700080087800a0462000a1fb22008008780004
:10b88000a0492000c1fb220080087800b04c2000b5
:10b89000e1fb220080087800e04f200001fc22003c
:10b8a00080087800e052200021fc22008008780007
:10b8b000c055200041fc22008008780090582000ec
:10b8c00061fc220080087800405b200081fc22009f
:10b8d00080087800d05d2000a1fc2200800878005c
:10b8e00040602000c1fc220080087800b062200087
:10b8f000e1fc2200800878003065200001fd220074
:10b9000080087800c067200021fd220080087800b0
:10b91000806a200041fd220080087800b06d200080
:10b9200061fd220080087800e070200081fd220087
:10b930008008780010742000a1fd220080087800a3
:10b9400030772000c1fd220080087800a07c200014
:10b95000e1fd220080087800807e200001fe2200a8
:10b9600080087800607f200021fe22008008780097
:10b97000f07e200041fe220080087800407d2000fb
:10b9800061fe220080087800407a200081fe2200bb
:10b9900080087800d0752000a1fe22008008780081
:10b9a00060702000c1fe220080087800506a2000ec
:10b9b000e1fe220080087800d063200001ff220011
:10b9c00080087800205d200021ff22008008780098
:10b9d0008056200041ff220080087800405020005f
:10b9e00061ff220080087800704a200081ff220059
:10b9f0008008780040452000a1ff220080087800e0
:10ba0000c0402000c1ff220080087800d03c200008
:10ba1000e1ff220080087800803920000100230027
:10ba200080087800a03620002100230080087800dc
:10ba3000503420004100230080087800403220006c
:10ba4000610023008008780070302000810023000e
:10ba500080087800b02e2000a10023008008780024
:10ba6000102d2000c100230080087800802b2000ca
:10ba7000e100230080087800c02820000101230095
:10ba8000800878009027200021012300800878009a
:10ba900070262000410123008008780050252000f6
:10baa00061012300800878005024200081012300d8
:10bab0008008780080232000a101230080087800fe
:10bac000d0222000c10123008008780060222000dd
:10bad000e1012300800878003022200001022300c9
:10bae000800878005022200021022300800878007e
:10baf000e02220004102230080087800c0232000bb
:10bb000061022300800878000025200081022300c4
:10bb10008008780080262000a10223008008780099
:10bb200070282000c102230080087800802a2000ad
:10bb3000e102230080087800b02c200001032300dc
:10bb400080087800d02e2000210323008008780090
:10bb5000f03020004103230080087800f0322000fc
:10bb60006103230080087800c03420008103230093
:10bb70008008780070362000a10323008008780038
:10bb8000e0372000c103230080087800203920001e
:10bb9000e103230080087800303a200001042300ec
:10bba00080087800c03b2000210423008008780032
:10bbb000503c20004104230080087800c03c200055
:10bbc0006104230080087800103d200081042300d8
:10bbd00080087800503d2000a104230080087800f0
:10bbe000903d2000c104230080087800d03d200053
:10bbf000e104230080087800003e200001052300b6
:10bc000080087800303e200021052300800878005d
:10bc1000603e20004105230080087800703e20002f
:10bc20006105230080087800803e20008105230004
:10bc300080087800903e2000a1052300800878004d
:10bc4000903e2000c105230080087800803e20003f
:10bc5000e105230080087800603e200001062300f3
:10bc600080087800303e20002106230080087800fc
:10bc7000f03d20004106230080087800b03d200000
:10bc80006106230080087800603d200081062300c3
:10bc900080087800003d2000a1062300800878007d
:10bca000903c2000c106230080087800103c200052
:10bcb000e106230080087800703b20000107230084
:10bcc00080087800d03a20002107230080087800ff
:10bcd0005039200041072300800878006038200098
:10bce0006107230080087800503720008107230077
:10bcf0008008780040362000a107230080087800e3
:10bd000000352000c107230080087800c0332000e0
:10bd1000e10723008008780070322000010823002a
:10bd20008008780000312000210823008008780076
:10bd3000a02f20004108230080087800702e2000ea
:10bd40006108230080087800402d2000810823002e
:10bd500080087800202c2000a108230080087800ab
:10bd6000402b2000c108230080087800902a200082
:10bd7000e108230080087800002a20000109230040
:10bd800080087800b029200021092300800878006d
:10bd9000902920004109230080087800b029200064
:10bda0006109230080087800f02920008109230020
:10bdb00080087800702a2000a109230080087800fc
:10bdc000002b2000c109230080087800b02b200040
:10bdd000e109230080087800802c2000010a23005c
:10bde00080087800602d2000210a23008008780058
:10bdf000602e2000410a230080087800b030200027
:10be0000610a23008008780010322000810a230094
:10be100080087800a0332000a10a23008008780061
:10be200050352000c10a23008008780060372000c8
:10be3000e10a23008008780090392000010b2300dc
:10be400080087800e03b2000210b23008008780068
:10be5000603e2000410b2300800878001041200044
:10be6000610b230080087800e0432000810b230051
:10be700080087800e0462000a10b230080087800ad
:10be8000e0492000c10b230080087800f04c20001e
:10be9000e10b23008008780000502000010c2300f3
:10bea0008008780000532000210c230080087800cf
:10beb00020562000410c23008008780020592000e3
:10bec000610c230080087800f05b2000810c2300c7
:10bed00080087800905e2000a10c23008008780084
:10bee00010612000c10c230080087800a0632000ae
:10bef000e10c23008008780020662000010d23005b
:10bf000080087800b0682000210d230080087800a8
:10bf1000706b2000410d230080087800506e2000d7
:10bf2000610d23008008780070742000810d2300cb
:10bf300080087800a0772000a10d230080087800f9
:10bf4000707a2000c10d230080087800c07c20009a
:10bf5000e10d230080087800607e2000010e2300a0
:10bf600080087800007f2000210e230080087800e0
:10bf7000607e2000410e230080087800707c200045
:10bf8000610e23008008780050792000810e230084
:10bf90008008780000752000a10e2300800878003a
:10bfa000c06f2000c10e230080087800b069200017
:10bfb000e10e230080087800c0622000010f2300fa
:10bfc00080087800005c2000210f230080087800a2
:10bfd00070552000410f230080087800304f20006a
:10bfe000610f23008008780070492000810f230032
:10bff0008008780060442000a10f230080087800aa
:10c00000f03f2000c10f230080087800203c200072
:10c01000e10f230080087800f03820000110230091
:10c020008008780050362000211023008008780016
:10c03000f03320004110230080087800e031200018
:10c040006110230080087800003020008110230058
:10c0500080087800c02c2000a11023008008780000
:10c06000402b2000c110230080087800e029200028
:10c07000e11023008008780090282000011123009f
:10c0800080087800502720002111230080087800c4
:10c090003026200041112300800878003025200040
:10c0a00061112300800878004024200081112300c2
:10c0b0008008780090232000a111230080087800d8
:10c0c00000232000c111230080087800c022200036
:10c0d000e111230080087800b02220000112230023
:10c0e00080087800f02220002112230080087800c8
:10c0f0008023200041122300800878006024200063
:10c10000611223008008780090252000811223000e
:10c110008008780010272000a112230080087800f2
:10c12000d0282000c112230080087800b02a200007
:10c13000e112230080087800a02c200001132300c6
:10c1400080087800c02e200021132300800878008a
:10c15000b030200041132300800878008032200096
:10c1600061132300800878003034200081132300fd
:10c1700080087800d0352000a113230080087800c3
:10c1800080382000c113230080087800a0392000e7
:10c19000e113230080087800903a20000114230066
:10c1a00080087800603b200021142300800878007c
:10c1b000f03b20004114230080087800703c2000f0
:10c1c0006114230080087800c03c20008114230003
:10c1d00080087800003d2000a1142300800878002a
:10c1e000203d2000c114230080087800403d20003d
:10c1f000e114230080087800503d20000115230041
:10c2000080087800703d2000211523008008780008
:10c21000803d20004115230080087800a03d2000cb
:10c220006115230080087800b03d200081152300af
:10c2300080087800d03d2000a115230080087800f8
:10c24000d03d2000c115230080087800d03d20009b
:10c25000e115230080087800d03d2000011623005e
:10c2600080087800c03d2000211623008008780057
:10c27000903d20004116230080087800603d20009a
:10c280006116230080087800103d200081162300ed
:10c2900080087800c03c2000a116230080087800a8
:10c2a000503c2000c116230080087800203b20006d
:10c2b000e116230080087800703a2000011723005f
:10c2c000800878009039200021172300800878002a
:10c2d000b03820004117230080087800d0372000b4
:10c2e0006117230080087800d036200081172300d2
:10c2f00080087800c0352000a1172300800878004e
:10c3000090342000c11723008008780050332000ab
:10c31000e117230080087800003220000118230074
:10c3200080087800b03020002118230080087800b1
:10c33000602f20004118230080087800202e200064
:10c340006118230080087800f02c20008118230059
:10c3500080087800f02b2000a118230080087800c6
:10c36000302b2000c118230080087800902a20007c
:10c37000e118230080087800402a200001192300da
:10c3800080087800102a20002119230080087800f6
:10c39000102a20004119230080087800502a20002c
:10c3a0006119230080087800b02a20008119230039
:10c3b00080087800402b2000a11923008008780015
:10c3c000f02b2000c119230080087800a02c200049
:10c3d000e119230080087800502e2000011a230064
:10c3e00080087800502f2000211a23008008780050
:10c3f00050302000411a230080087800803120004e
:10c40000611a230080087800d0322000811a2300ae
:10c410008008780050342000a11a2300800878009a
:10c4200000362000c11a230080087800f037200071
:10c43000e11a230080087800103a2000011b230035
:10c4400080087800603c2000211b230080087800d1
:10c45000003f2000411b230080087800b0412000ed
:10c46000611b23008008780080442000811b23008a
:10c470008008780070472000a11b23008008780006
:10c48000704a2000c11b230080087800804d2000e6
:10c49000e11b23008008780080502000011c23004d
:10c4a0008008780070532000211c23008008780049
:10c4b00040562000411c230080087800f0582000de
:10c4c000611c230080087800905b2000811c230001
:10c4d00080087800305e2000a11c230080087800ce
:10c4e000a0602000c11c230080087800f0622000ba
:10c4f000e11c23008008780050652000011d230006
:10c5000080087800906a2000211d230080087800b0
:10c51000806d2000411d230080087800907020006d
:10c52000611d230080087800b0732000811d230066
:10c5300080087800d0762000a11d230080087800b4
:10c54000c0792000c11d230080087800707c200085
:10c55000e11d230080087800607e2000011e23007a
:10c5600080087800307f2000211e2300800878009a
:10c57000b07e2000411e230080087800d07c20007f
:10c58000611e230080087800b0792000811e2300fe
:10c590008008780060752000a11e230080087800c4
:10c5a00000702000c11e230080087800e069200090
:10c5b000e11e23008008780040632000011f230053
:10c5c00080087800705c2000211f2300800878001c
:10c5d000a0552000411f230080087800e04e200075
:10c5e000611f23008008780020492000811f23005c
:10c5f0008008780000442000a11f230080087800f4
:10c60000a03f2000c11f230080087800e03b2000ed
:10c61000e11f230080087800c0382000012023009b
:10c620008008780010362000212023008008780040
:10c63000c03120004120230080087800f02f200026
:10c640006120230080087800302e20008120230004
:10c6500080087800802c2000a1202300800878002a
:10c66000002b2000c12023008008780090292000a2
:10c67000e1202300800878005028200001212300b9
:10c6800080087800302720002121230080087800ce
:10c69000302620004121230080087800402520001a
:10c6a000612123008008780070242000812123006c
:10c6b00080087800d0232000a12123008008780082
:10c6c00060232000c121230080087800202320005f
:10c6d000e12123008008780020232000012223008c
:10c6e0008008780070232000212223008008780031
:10c6f000102420004122230080087800002520001b
:10c700006122230080087800402620008122230037
:10c7100080087800c0272000a1222300800878002c
:10c7200080292000c122230080087800602b20008f
:10c73000e122230080087800602d200001232300df
:10c7400080087800502f20002123230080087800e3
:10c75000503120004123230080087800203520003c
:10c760006123230080087800b03620008123230055
:10c770008008780030382000a1232300800878004a
:10c7800070392000c123230080087800903a2000ef
:10c79000e123230080087800803b2000012423004f
:10c7a00080087800403c2000212423008008780085
:10c7b000e03c20004124230080087800403d200018
:10c7c0006124230080087800903d2000812423000c
:10c7d00080087800c03d2000a12423008008780054
:10c7e000d03d2000c124230080087800e03d2000d7
:10c7f000e124230080087800f03d2000012523007b
:10c8000080087800003e2000212523008008780061
:10c81000003e20004125230080087800203e2000b3
:10c820006125230080087800303e20008125230008
:10c8300080087800503e2000a12523008008780061
:10c84000603e2000c125230080087800703e200053
:10c85000e125230080087800803e20000126230087
:10c8600080087800703e2000212623008008780090
:10c87000403e20004126230080087800003e200032
:10c880006126230080087800503d20008126230087
:10c8900080087800d03c2000a12623008008780082
:10c8a000403c2000c126230080087800a03b2000e7
:10c8b000e126230080087800e03a200001272300c9
:10c8c00080087800103a2000212723008008780093
:10c8d00020392000412723008008780020382000dc
:10c8e000612723008008780000372000812723007b
:10c8f00080087800d0352000a12723008008780028
:10c90000a0342000c1272300800878006033200075
:10c91000e12723008008780020322000012823002e
:10c9200080087800d030200021282300800878007b
:10c93000802f20004128230080087800402e20000e
:10c940006128230080087800202d20008128230002
:10c9500080087800102c2000a1282300800878008f
:10c96000402b2000c128230080087800902a200056
:10c97000e128230080087800202a200001292300d4
:10c9800080087800e0292000212923008008780011
:10c99000e02920004129230080087800002a200097
:10c9a0006129230080087800602a20008129230063
:10c9b00080087800802b2000a129230080087800bf
:10c9c000302c2000c129230080087800102d200081
:10c9d000e129230080087800f02d2000012a23009f
:10c9e00080087800002f2000212a2300800878008a
:10c9f00030302000412a2300800878007031200068
:10ca0000612a230080087800d0322000812a230088
:10ca10008008780060342000a12a23008008780074
:10ca200030362000c12a23008008780030382000ea
:10ca3000e12a230080087800603a2000012b2300bf
:10ca400080087800f03f2000212b23008008780028
:10ca50000000060050432000412b2300800878008e
:10ca6000f0492000612b230080087800a0512000ad
:10ca7000812b230080087800b0592000a12b2300cf
:10ca800080087800a0612000c12b23008008780076
:10ca900020692000e12b230080087800007020002e
:10caa000012c23008008780010762000212c230020
:10cab00080087800e07c2000412c2300800878006a
:10cac000f07e2000612c230080087800c07e2000ca
:10cad000812c230080087800d07b2000a12c23002b
:10cae00080087800b0762000c12c230080087800f0
:10caf000e06f2000e12c230080087800d067200040
:10cb0000012d230080087800e05e2000212d230005
:10cb100080087800b0552000412d2300800878005f
:10cb200030492000612d2300800878004042200019
:10cb3000812d230080087800703d2000a12d230066
:10cb400080087800b03a2000c12d230080087800ca
:10cb5000803a2000e12d230080087800d03c20009e
:10cb6000012e23008008780000402000212e2300a1
:10cb70008008780060432000412e23008008780060
:10cb800050452000612e230080087800604220007c
:10cb9000812e230080087800f03b2000a12e230086
:10cba0008008780060332000c12e230080087800c0
:10cbb000402a2000e12e2300800878005022200027
:10cbc000012f230080087800c01c2000212f2300a3
:10cbd00080087800b0192000412f230080087800d9
:10cbe00050192000612f230080087800c01c20000d
:10cbf000812f23008008780090202000a12f23009f
:10cc00008008780080242000c12f2300800878004d
:10cc100030282000e12f230080087800902a20008f
:10cc20000130230080087800102c200021302300e0
:10cc300080087800d02c2000413023008008780044
:10cc4000502d20006130230080087800502e2000f5
:10cc50008130230080087800902f2000a13023002d
:10cc60008008780040312000c1302300800878001f
:10cc700060332000e130230080087800a0352000d8
:10cc80000131230080087800203820002131230062
:10cc900080087800703a2000413123008008780035
:10cca000703c20006131230080087800303e200075
:10ccb0008131230080087800003e2000a13123004c
:10ccc00080087800403d2000c131230080087800b2
:10ccd000503c2000e131230080087800f03b200028
:10cce0000132230080087800403c200021322300dc
:10ccf00080087800303d2000413223008008780011
:10cd0000f03d20006132230080087800503e200072
:10cd10008132230080087800b03e2000a132230039
:10cd200080087800103f2000c1322300800878007e
:10cd3000d03f2000e13223008008780080402000ae
:10cd40000133230080087800d040200021332300e5
:10cd500080087800d040200041332300800878000c
:10cd6000a04020006133230080087800b0402000fc
:10cd7000813323008008780090412000a1332300f4
:10cd80008008780060422000c133230080087800ca
:10cd900010432000e133230080087800f042200097
:10cda0000134230080087800204220002134230031
:10cdb000800878007040200041342300800878000b
:10cdc000503e20006134230080087800403c200061
:10cdd0008134230080087800a0392000a13423008a
:10cde0008008780050382000c13423008008780083
:10cdf000d0372000e134230080087800e03720009d
:10ce00000135230080087800b03820002135230048
:10ce100080087800303a20004135230080087800ef
:10ce2000403c20006135230080087800603e2000ef
:10ce3000813523008008780070402000a135230050
:10ce40008008780090422000c135230080087800d7
:10ce5000a0432000e135230080087800d044200062
:10ce60000136230080087800104620002136230078
:10ce70008008780070472000413623008008780041
:10ce8000a048200061362300800878007049200007
:10ce90008136230080087800104a2000a136230044
:10cea00080087800604a2000c1362300800878009e
:10ceb000404a2000e136230080087800d049200055
:10cec0000137230080087800004920002137230023
:10ced00080087800e0472000413723008008780070
:10cee000604620006137230080087800c04420009d
:10cef000813723008008780020432000a1372300d9
:10cf000080087800c0412000c137230080087800e5
:10cf100020402000e137230080087800403f2000b7
:10cf20000138230080087800a03e2000213823002b
:10cf300080087800103e20004138230080087800e7
:10cf4000b03d20006138230080087800603d20005b
:10cf50008138230080087800303d2000a13823006c
:10cf600080087800003d2000c13823008008780048
:10cf7000703c2000e138230080087800703b2000de
:10cf80000139230080087800f0392000213923007e
:10cf9000800878000038200041392300800878009c
:10cfa000f03520006139230080087800103420001b
:10cfb000813923008008780040322000a139230005
:10cfc0008008780090302000c13923008008780064
:10cfd000b02d2000e139230080087800802b20004c
:10cfe000013a230080087800c0292000213a23005c
:10cff00080087800c0282000413a2300800878008b
:10d00000d0282000613a230080087800f029200011
:10d01000813a230080087800002c2000a13a2300e8
:10d0200080087800a02e2000c13a230080087800f4
:10d0300000322000e13a2300800878007038200098
:10d04000013b230080087800903d2000213b230015
:10d0500080087800e0432000413b230080087800ee
:10d06000f04a2000613b230080087800c052200075
:10d07000813b230080087800e05a2000a13b230078
:10d0800080087800d0622000c13b2300800878002f
:10d09000706a2000e13b2300800878009074200033
:10d0a000013c230080087800207a2000213c2300e6
:10d0b00080087800007e2000413c23008008780032
:10d0c000e07f2000613c230080087800607f200022
:10d0d000813c230080087800607c2000a13c230074
:10d0e0008008780010772000c13c23008008780079
:10d0f000e06f2000e13c230080087800f06220000f
:10d10000013d23008008780070592000213d230054
:10d110008008780070502000413d2300800878008e
:10d1200050482000613d23008008780070412000b5
:10d13000813d230080087800903c2000a13d230021
:10d1400080087800003a2000c13d23008008780064
:10d15000003a2000e13d230080087800b03c200028
:10d16000013e23008008780060422000213e230019
:10d170008008780020452000413e23008008780088
:10d18000a0452000613e2300800878004042200036
:10d19000813e230080087800b03b2000a13e2300a0
:10d1a0008008780030332000c13e230080087800da
:10d1b000002a2000e13e2300800878003022200071
:10d1c000013f230080087800e01a2000213f23005f
:10d1d0008008780060192000413f23008008780013
:10d1e000101a2000613f230080087800f01c200006
:10d1f000813f230080087800b0202000a13f230059
:10d2000080087800a0242000c13f23008008780017
:10d2100010282000e13f230080087800502a2000d9
:10d220000140230080087800b02b2000214023001b
:10d2300080087800d02c200041402300800878002e
:10d24000602d20006140230080087800402e2000df
:10d250008140230080087800902f2000a140230007
:10d260008008780040312000c14023008008780009
:10d2700030332000e1402300800878006035200032
:10d280000141230080087800d0372000214123008d
:10d2900080087800803b200041412300800878000e
:10d2a000303d20006141230080087800003e2000ce
:10d2b0008141230080087800d03d2000a141230057
:10d2c00080087800203d2000c141230080087800bc
:10d2d000803c2000e141230080087800703c200061
:10d2e0000142230080087800d03c20002142230026
:10d2f00080087800f03d200041422300800878003b
:10d30000903e20006142230080087800003f20000a
:10d310008142230080087800703f2000a142230052
:10d3200080087800d03f2000c142230080087800a8
:10d3300040402000e1422300800878007040200037
:10d34000014323008008780060402000214323002f
:10d350008008780030402000414323008008780096
:10d3600010402000614323008008780080402000a6
:10d37000814323008008780080412000a1432300de
:10d380008008780070422000c143230080087800a4
:10d3900030432000e1432300800878003043200020
:10d3a000014423008008780010422000214423001b
:10d3b0008008780040402000414423008008780025
:10d3c000103d20006144230080087800203b2000ad
:10d3d0008144230080087800a0392000a144230064
:10d3e0008008780070382000c1442300800878004d
:10d3f000f0372000e144230080087800f037200057
:10d400000145230080087800a03820002145230032
:10d4100080087800203a20004145230080087800e9
:10d42000403d20006145230080087800603f2000d7
:10d43000814523008008780030412000a145230069
:10d440008008780090422000c145230080087800c1
:10d45000a0432000e145230080087800c04420005c
:10d460000146230080087800f04520002146230073
:10d47000800878004047200041462300800878005b
:10d48000704820006146230080087800b0492000e1
:10d490008146230080087800204a2000a14623000e
:10d4a00080087800304a2000c146230080087800b8
:10d4b000f0492000e1462300800878005049200010
:10d4c000014723008008780080482000214723007e
:10d4d00080087800704720004147230080087800ca
:10d4e0003046200061472300800878001044200067
:10d4f000814723008008780090422000a147230044
:10d500008008780020412000c1472300800878006f
:10d5100010402000e147230080087800403f2000b1
:10d520000148230080087800b03e200021482300f5
:10d5300080087800203e20004148230080087800c1
:10d54000a03d20006148230080087800103d2000a5
:10d550008148230080087800a03c2000a1482300d7
:10d5600080087800703c2000c148230080087800c3
:10d57000103c2000e148230080087800203b200078
:10d580000149230080087800c03920002149230088
:10d5900080087800f0372000414923008008780097
:10d5a000d03520006149230080087800a033200096
:10d5b000814923008008780080302000a1492300a1
:10d5c00080087800f02e2000c149230080087800f0
:10d5d000902d2000e149230080087800102c2000c5
:10d5e000014a230080087800b02a2000214a230045
:10d5f00080087800a0292000414a23008008780094
:10d6000030292000614a230080087800202a200069
:10d61000814a230080087800502d2000a14a230071
:10d6200080087800a0302000c14a230080087800dc
:10d6300090342000e14a230080087800e038200080
:10d64000014b230080087800003e2000214b23007e
:10d650008008780050442000414b23008008780067
:10d66000e04b2000614b23008008780030542000fc
:10d67000814b230080087800c05c2000a14b230070
:10d680008008780000692000c14b230080087800e2
:10d6900050702000e14b230080087800c076200005
:10d6a000014c230080087800c07b2000214c23001f
:10d6b00080087800e07e2000414c2300800878003c
:10d6c000d07f2000614c230080087800507e20002d
:10d6d000814c230080087800507a2000a14c230060
:10d6e00080087800c0702000c14c230080087800ba
:10d6f000d0682000e14c23008008780010602000f2
:10d70000014d230080087800e0562000214d2300c1
:10d7100080087800604e2000414d2300800878008a
:10d72000e0462000614d230080087800d0402000b2
:10d73000814d230080087800103d2000a14d23007a
:10d7400080087800c03b2000c14d2300800878008d
:10d75000803d2000e14d230080087800204120001a
:10d76000014e230080087800e0442000214e230071
:10d770008008780060472000414e23008008780030
:10d7800020472000614e230080087800904220004e
:10d79000814e230080087800a03a2000a14e23008b
:10d7a0008008780000312000c14e230080087800f6
:10d7b00050232000e14e230080087800c01c200088
:10d7c000014f230080087800e0182000214f23003b
:10d7d00080087800d0172000414f2300800878008f
:10d7e00020192000614f230080087800a01c200031
:10d7f000814f230080087800e0202000a14f230003
:10d800008008780010252000c14f23008008780090
:10d8100090292000e14f230080087800202b200071
:10d820000150230080087800f02b200021502300b5
:10d8300080087800a02c2000415023008008780048
:10d84000302d20006150230080087800302e200009
:10d850008150230080087800802f2000a1502300f1
:10d860008008780060312000c150230080087800d3
:10d8700090332000e15023008008780070372000aa
:10d880000151230080087800203a20002151230014
:10d8900080087800703c2000415123008008780007
:10d8a000103e20006151230080087800a03e200037
:10d8b0008151230080087800303e2000a1512300d0
:10d8c00080087800503d2000c15123008008780076
:10d8d000803c2000e151230080087800703c20004b
:10d8e0000152230080087800003d200021522300cf
:10d8f00080087800803d2000415223008008780095
:10d90000d03d20006152230080087800103e2000a6
:10d910008152230080087800803e2000a15223001d
:10d9200080087800103f2000c15223008008780052
:10d93000b03f2000e15223008008780060402000c2
:10d9400001532300800878007040200021532300f9
:10d950008008780090402000415323008008780020
:10d96000d0402000615323008008780050412000ff
:10d97000815323008008780050422000a1532300e7
:10d980008008780030432000c153230080087800cd
:10d99000c0432000e153230080087800704320003a
:10d9a00001542300800878002041200021542300e6
:10d9b00080087800e03e2000415423008008780071
:10d9c000803c20006154230080087800803a2000c9
:10d9d0008154230080087800f0382000a1542300ef
:10d9e00080087800f0372000c154230080087800b8
:10d9f00070372000e1542300800878008037200031
:10da0000015523008008780030392000215523007b
:10da100080087800303b20004155230080087800c2
:10da2000703d20006155230080087800903f200061
:10da3000815523008008780080412000a1552300f3
:10da40008008780010432000c1552300800878002a
:10da500060442000e155230080087800b045200094
:10da600001562300800878008047200021562300bb
:10da70008008780070482000415623008008780014
:10da8000604920006156230080087800204a200069
:10da90008156230080087800a04a2000a156230068
:10daa00080087800d04a2000c15623008008780002
:10dab000704a2000e156230080087800a049200029
:10dac0000157230080087800a04820002157230038
:10dad00080087800b0462000415723008008780075
:10dae0001045200061572300800878003043200053
:10daf000815723008008780070412000a15723003f
:10db00008008780020402000c1572300800878005a
:10db1000603f2000e157230080087800d03e2000bd
:10db20000158230080087800903e200021582300ef
:10db300080087800003e20004158230080087800cb
:10db4000d03d20006158230080087800703d2000ff
:10db50008158230080087800203d2000a158230030
:10db600080087800803c2000c1582300800878009d
:10db7000903b2000e158230080087800403a2000c4
:10db80000159230080087800903820002159230093
:10db900080087800903620004159230080087800e2
:10dba000b033200061592300800878000032200043
:10dbb000815923008008780070302000a15923008b
:10dbc00080087800c02e2000c1592300800878000a
:10dbd000e02c2000e159230080087800102b200061
:10dbe000015a230080087800b0292000215a230020
:10dbf0008008780000292000415a2300800878001e
:10dc0000e0292000615a230080087800302c200091
:10dc1000815a230080087800902f2000a15a230009
:10dc200080087800b0332000c15a230080087800b3
:10dc300020382000e15a230080087800703c200042
:10dc4000015b23008008780070412000215b2300e5
:10dc50008008780070472000415b2300800878002e
:10dc600030522000615b230080087800c0592000fa
:10dc7000815b23008008780030612000a15b2300d5
:10dc80008008780010682000c15b230080087800bd
:10dc9000506e2000e15b230080087800d0732000e4
:10dca000015c23008008780030782000215c23008c
:10dcb00080087800007b2000415c23008008780009
:10dcc000207c2000615c230080087800a07920007f
:10dcd000815c23008008780050752000a15c23003f
:10dce00080087800606f2000c15c23008008780005
:10dcf00060682000e15c23008008780090602000cc
:10dd0000015d23008008780040582000215d230039
:10dd10008008780060502000415d23008008780072
:10dd200020492000615d23008008780070402000b9
:10dd3000815d230080087800603d2000a15d230004
:10dd400080087800d03c2000c15d23008008780066
:10dd5000d03e2000e15d2300800878007042200062
:10dd6000015e230080087800e0452000215e23004a
:10dd700080087800a0472000415e230080087800da
:10dd800030462000615e230080087800203d20009e
:10dd9000815e230080087800f0332000a15e23001c
:10dda00080087800102a2000c15e230080087800d7
:10ddb00060212000e15e230080087800101b200015
:10ddc000015f230080087800a0172000215f230056
:10ddd0008008780060172000415f230080087800e9
:10dde00070192000615f230080087800201d20004a
:10ddf000815f23008008780060232000a15f23005a
:10de00008008780000272000c15f23008008780088
:10de100090292000e15f230080087800302b20004b
:10de20000160230080087800402c2000216023003e
:10de300080087800002d20004160230080087800d1
:10de4000e02d20006160230080087800f02e200083
:10de5000816023008008780060312000a1602300e9
:10de60008008780080332000c1602300800878009b
:10de7000c0352000e1602300800878004038200091
:10de80000161230080087800903a2000216123007e
:10de900080087800803c20004161230080087800e1
:10dea000a03d20006161230080087800003e200032
:10deb0008161230080087800903d2000a16123004b
:10dec00080087800803c2000c16123008008780031
:10ded000103c2000e161230080087800003c200015
:10dee0000162230080087800703c2000216223003a
:10def00080087800f03c2000416223008008780010
:10df0000703d20006162230080087800003e200000
:10df10008162230080087800a03e2000a1622300d7
:10df200080087800c03f2000c1622300800878008c
:10df300060402000e162230080087800b0402000ab
:10df40000163230080087800a040200021632300a3
:10df5000800878008040200041632300800878001a
:10df6000a040200061632300800878003041200039
:10df7000816323008008780040422000a1632300d1
:10df80008008780080432000c16323008008780067
:10df900090432000e163230080087800a042200025
:10dfa0000164230080087800e04020002164230001
:10dfb00080087800c03e200041642300800878007b
:10dfc000a03c20006164230080087800b03a200063
:10dfd000816423008008780040392000a164230078
:10dfe0008008780050382000c16423008008780041
:10dff000f0372000e16423008008780070382000aa
:10e000000165230080087800c039200021652300c5
:10e0100080087800d03b200041652300800878000c
:10e02000303e2000616523008008780050402000c9
:10e03000816523008008780020422000a16523002c
:10e040008008780070432000c165230080087800b4
:10e0500020452000e165230080087800404620002c
:10e0600001662300800878007047200021662300a5
:10e0700080087800704820004166230080087800fe
:10e08000504920006166230080087800c0492000c4
:10e090008166230080087800004a2000a1662300e2
:10e0a00080087800f0492000c166230080087800cd
:10e0b00040492000e1662300800878008048200065
:10e0c0000167230080087800904720002167230023
:10e0d000800878008046200041672300800878008f
:10e0e000204520006167230080087800b0432000ad
:10e0f000816723008008780010422000a167230078
:10e1000080087800a0402000c167230080087800c4
:10e11000903f2000e167230080087800903e2000b7
:10e120000168230080087800403e20002168230019
:10e1300080087800003e20004168230080087800b5
:10e14000c03d20006168230080087800803d2000e9
:10e150008168230080087800203d2000a16823000a
:10e1600080087800603c2000c168230080087800a7
:10e17000503b2000e168230080087800103920001f
:10e18000016923008008780060372000216923009e
:10e1900080087800b03520004169230080087800ad
:10e1a000403420006169230080087800c0322000dc
:10e1b000816923008008780010312000a1692300c4
:10e1c00080087800602f2000c16923008008780053
:10e1d000902d2000e169230080087800c02b2000ea
:10e1e000016a230080087800f0292000216a2300ba
:10e1f0008008780080292000416a23008008780088
:10e20000102a2000616a230080087800d02b2000ab
:10e21000816a230080087800502e2000a16a230024
:10e2200080087800d0312000c16a2300800878007f
:10e23000f0352000e16a230080087800603a200071
:10e24000016b230080087800f03f2000216b230041
:10e250008008780000000600f03f2000416b23009a
:10e260008008780080412000616b230080087800de
:10e27000e0422000816b230080087800a044200049
:10e28000a16b23008008780030462000c16b23007a
:10e2900080087800a0472000e16b23008008780008
:10e2a00030492000016c230080087800e04a2000fb
:10e2b000216c230080087800f04c2000416c230082
:10e2c00080087800d04e2000616c23008008780020
:10e2d000d0502000816c230080087800c0522000bc
:10e2e000a16c230080087800d0542000c16c23006a
:10e2f0008008780010572000e16c23008008780027
:10e3000050592000016d230080087800d05b200068
:10e31000216d230080087800905e2000416d23006d
:10e320008008780070612000616d2300800878000b
:10e3300040642000816d230080087800a0652000e3
:10e34000a16d230080087800d0682000c16d2300f3
:10e3500080087800c06b2000e16d23008008780001
:10e36000a06d2000016e230080087800806e2000e0
:10e37000216e230080087800406e2000416e23004b
:10e3800080087800a06c2000616e2300800878006f
:10e39000f0682000816e2300800878002063200050
:10e3a000a16e230080087800605b2000c16e23000e
:10e3b0008008780060512000e16e2300800878001a
:10e3c000b0452000016f23008008780050382000fd
:10e3d000216f230080087800b02a2000416f2300bd
:10e3e00080087800801e2000616f2300800878007c
:10e3f00000142000816f230080087800a00b20000b
:10e40000a16f23008008780000062000c16f230060
:10e4100080087800f0022000e16f23008008780077
:10e4200020022000017023008008780030022000c4
:10e4300021702300800878005004200041702300e0
:10e440008008780070082000617023008008780040
:10e45000b00d20008170230080087800d0132000c8
:10e46000a170230080087800b01a2000c17023003a
:10e470008008780020212000e170230080087800c7
:10e48000902720000171230080087800802e200052
:10e49000217123008008780030342000417123006e
:10e4a00080087800403920006171230080087800de
:10e4b000e03d20008171230080087800d0402000da
:10e4c000a17123008008780010432000c17123004f
:10e4d00080087800a0442000e171230080087800c3
:10e4e000104620000172230080087800d0462000ea
:10e4f0002172230080087800f0462000417223003a
:10e50000800878002047200061722300800878008e
:10e51000f04620008172230080087800b046200079
:10e52000a17223008008780020472000c1722300d8
:10e530008008780040472000e172230080087800be
:10e54000804720000173230080087800b047200036
:10e550002173230080087800704720004173230056
:10e56000800878001047200061732300800878003d
:10e57000b04620008173230080087800c046200048
:10e58000a17323008008780040462000c173230057
:10e590008008780090452000e1732300800878000f
:10e5a000c04420000174230080087800e04320006c
:10e5b0002174230080087800004320004174230068
:10e5c00080087800404220006174230080087800b1
:10e5d000604120008174230080087800a040200062
:10e5e000a17423008008780060402000c1742300db
:10e5f0008008780030402000e17423008008780013
:10e6000010402000017523008008780000402000a1
:10e6100021752300800878006040200041752300a8
:10e620008008780000412000617523008008780090
:10e63000504120008175230080087800a04120000f
:10e64000a17523008008780080412000c175230057
:10e650008008780060412000e17523008008780080
:10e66000204120000176230080087800f04020003f
:10e670002176230080087800404020004176230066
:10e6800080087800903f20006176230080087800a1
:10e69000f03e20008176230080087800303e200084
:10e6a000a176230080087800c03d2000c1762300b9
:10e6b00080087800a03d2000e176230080087800e3
:10e6c000003e20000177230080087800103e2000e3
:10e6d0002177230080087800703e200041772300d6
:10e6e00080087800c03e2000617723008008780011
:10e6f000d03e20008177230080087800e03e200093
:10e70000a177230080087800c03e2000c177230055
:10e7100080087800803e2000e177230080087800a0
:10e72000203e20000178230080087800703d200002
:10e730002178230080087800c03c20004178230025
:10e7400080087800803c20006178230080087800f1
:10e75000403c20008178230080087800003c2000a5
:10e76000a178230080087800b03b2000c178230006
:10e7700080087800203b2000e178230080087800a2
:10e78000703a200001792300800878006039200069
:10e790002179230080087800803820004179230007
:10e7a00080087800e0372000617923008008780035
:10e7b00090372000817923008008780010372000ee
:10e7c000a179230080087800d0362000c179230089
:10e7d00080087800e0362000e17923008008780086
:10e7e00040372000017a230080087800c0372000dd
:10e7f000217a23008008780060382000417a2300c5
:10e800008008780030392000617a23008008780081
:10e81000403a2000817a230080087800803b200065
:10e82000a17a230080087800c03c2000c17a230030
:10e8300080087800303e2000e17a230080087800cc
:10e84000803f2000017b230080087800b04020003a
:10e85000217b23008008780080412000417b230039
:10e860008008780070422000617b230080087800d7
:10e8700080432000817b230080087800c044200072
:10e88000a17b23008008780060452000c17b230025
:10e8900080087800c0462000e17b230080087800d3
:10e8a00080482000017c230080087800504a200026
:10e8b000217c230080087800704c2000417c2300dc
:10e8c00080087800504e2000617c2300800878008a
:10e8d00030502000817c23008008780020522000e6
:10e8e000a17c23008008780080542000c17c230094
:10e8f0008008780080562000e17c230080087800a2
:10e90000b0582000017d230080087800605b200063
:10e91000217d230080087800105e2000417d2300c7
:10e9200080087800f0602000617d23008008780076
:10e93000b0632000817d230080087800d06620002d
:10e94000a17d230080087800106a2000c17d23008b
:10e9500080087800e06c2000e17d230080087800ca
:10e96000906e2000017e230080087800006f200058
:10e97000217e230080087800506f2000417e230014
:10e9800080087800106e2000617e230080087800e7
:10e99000606a2000817e2300800878009064200057
:10e9a000a17e230080087800005d2000c17e230046
:10e9b0008008780020532000e17e23008008780042
:10e9c00040472000017f230080087800f0392000b4
:10e9d000217f230080087800f02b2000417f230056
:10e9e00080087800401f2000617f230080087800a5
:10e9f00000142000817f230080087800d00a2000c6
:10ea0000a17f230080087800e0042000c17f23005c
:10ea10008008780090012000e17f230080087800c2
:10ea2000a000200001802300800878001002200050
:10ea300021802300800878004005200041802300c9
:10ea400080087800e00920006180230080087800b9
:10ea5000a00c200081802300800878001013200083
:10ea6000a180230080087800201a2000c1802300a4
:10ea700080087800a0202000e18023008008780032
:10ea8000b02720000181230080087800802e20001c
:10ea90002181230080087800103420004181230068
:10eaa00080087800b0392000618123008008780058
:10eab000103e20008181230080087800e040200083
:10eac000a18123008008780040432000c1812300f9
:10ead00080087800d0442000e1812300800878007d
:10eae000f045200001822300800878007046200055
:10eaf0002182230080087800e04620004182230024
:10eb000080087800d04620006182230080087800c9
:10eb1000e0462000818223008008780040472000e2
:10eb2000a18223008008780030472000c1822300a2
:10eb30008008780010472000e182230080087800d8
:10eb4000704720000183230080087800a047200040
:10eb50002183230080087800904720004183230010
:10eb600080087800604720006183230080087800d7
:10eb70005047200081832300800878000047200050
:10eb8000a18323008008780070462000c183230001
:10eb900080087800b0452000e183230080087800d9
:10eba000c04420000184230080087800c043200076
:10ebb0002184230080087800004320004184230042
:10ebc00080087800104220006184230080087800cb
:10ebd000404120008184230080087800b04020005c
:10ebe000a18423008008780050402000c1842300c5
:10ebf0008008780010402000e1842300800878001d
:10ec0000304020000185230080087800304020003b
:10ec10002185230080087800604020004185230082
:10ec200080087800f040200061852300800878008b
:10ec30005041200081852300800878009041200009
:10ec4000a185230080087800b0412000c185230001
:10ec500080087800a0412000e1852300800878002a
:10ec600050412000018623008008780000412000e8
:10ec70002186230080087800704020004186230010
:10ec800080087800b03f200061862300800878006b
:10ec9000003f20008186230080087800803e20000d
:10eca000a186230080087800203e2000c186230032
:10ecb00080087800f03d2000e1862300800878007d
:10ecc000003e20000187230080087800003e2000dd
:10ecd0002187230080087800503e200041872300d0
:10ece00080087800903e200061872300800878002b
:10ecf000b03e20008187230080087800b03e2000cd
:10ed0000a187230080087800803e2000c18723006f
:10ed100080087800603e2000e187230080087800aa
:10ed2000d03d20000188230080087800303d20007d
:10ed30002188230080087800a03c2000418823001f
:10ed400080087800303c200061882300800878002b
:10ed5000d03b20008188230080087800403b2000c1
:10ed6000a188230080087800903a2000c188230001
:10ed700080087800103a2000e1882300800878009d
:10ed8000703920000189230080087800e0382000d5
:10ed90002189230080087800503820004189230011
:10eda00080087800103820006189230080087800ee
:10edb000f037200081892300800878000038200087
:10edc000a18923008008780020382000c189230011
:10edd0008008780070382000e189230080087800de
:10ede00080382000018a230080087800c038200085
:10edf000218a230080087800f0382000418a23000f
:10ee00008008780080392000618a2300800878001b
:10ee1000503a2000818a230080087800703b20004f
:10ee2000a18a230080087800b03c2000c18a23001a
:10ee300080087800203e2000e18a230080087800c6
:10ee4000303f2000018b230080087800e03f200045
:10ee5000218b230080087800a0402000418b2300f4
:10ee60008008780060412000618b230080087800d2
:10ee700080422000818b230080087800104420000d
:10ee8000a18b230080087800c0452000c18b23009f
:10ee900080087800e0472000e18b2300800878009c
:10eea000d0492000018c230080087800a04b20006e
:10eeb000218c230080087800704d2000418c2300b5
:10eec00080087800404e2000618c23008008780084
:10eed00060502000818c2300800878006052200060
:10eee000a18c23008008780080542000c18c23006e
:10eef00080087800d0562000e18c2300800878003c
:10ef000050592000018d230080087800205c2000eb
:10ef1000218d230080087800305f2000418d230080
:10ef20008008780040622000618d2300800878000e
:10ef300020652000818d2300800878003068200043
:10ef4000a18d230080087800606b2000c18d230014
:10ef500080087800e06d2000e18d230080087800b3
:10ef6000706f2000018e2300800878003070200030
:10ef7000218e230080087800306f2000418e23000e
:10ef800080087800406c2000618e230080087800a3
:10ef9000d0662000818e230080087800305f20003a
:10efa000a18e230080087800d05a2000c18e230053
:10efb0008008780050502000e18e230080087800ff
:10efc00010442000018f230080087800c036200004
:10efd000218f230080087800a0292000418f230082
:10efe00080087800c01d2000618f23008008780011
:10eff00090132000818f230080087800700b200080
:10f00000a18f23008008780010062000c18f230004
:10f010008008780080022000e18f230080087800bb
:10f0200030012000019023008008780000022000b9
:10f030002190230080087800a00420004190230044
:10f040008008780070092000619023008008780013
:10f05000d00f200081902300800878003017200016
:10f06000a190230080087800b01e2000c1902300ea
:10f0700080087800b0252000e19023008008780007
:10f08000702c20000191230080087800502f200070
:10f090002191230080087800c03420004191230092
:10f0a00080087800d0392000619123008008780022
:10f0b000d03d20008191230080087800d0402000be
:10f0c000a19123008008780020432000c1912300f3
:10f0d00080087800b0442000e19123008008780087
:10f0e000004620000192230080087800e0462000be
:10f0f00021922300800878003047200041922300ad
:10f1000080087800f0462000619223008008780093
:10f11000004720008192230080087800d04620001c
:10f12000a192230080087800d0462000c1922300dd
:10f1300080087800e0462000e192230080087800f3
:10f14000504720000193230080087800a04720004a
:10f150002193230080087800b047200041932300ca
:10f1600080087800b0472000619323008008780071
:10f17000a04720008193230080087800504720009a
:10f18000a193230080087800f0462000c19323005b
:10f190008008780000462000e19323008008780072
:10f1a000b0442000019423008008780080432000b0
:10f1b00021942300800878005042200041942300cd
:10f1c0008008780050412000619423008008780076
:10f1d00090402000819423008008780000402000a7
:10f1e000a194230080087800c03f2000c194230030
:10f1f00080087800d03f2000e19423008008780048
:10f20000f03f200001952300800878001040200086
:10f210002195230080087800a0402000419523001c
:10f220008008780030412000619523008008780034
:10f23000a04120008195230080087800f041200043
:10f24000a19523008008780010422000c19523007a
:10f250008008780010422000e195230080087800a3
:10f26000b041200001962300800878004041200032
:10f2700021962300800878009040200041962300ca
:10f2800080087800c03f2000619623008008780045
:10f29000203f20008196230080087800603e2000f7
:10f2a000a196230080087800203e2000c19623000c
:10f2b00080087800203e2000e19623008008780036
:10f2c000303e20000197230080087800803e200017
:10f2d0002197230080087800903e2000419723006a
:10f2e00080087800903e2000619723008008780015
:10f2f000903e20008197230080087800703e200017
:10f30000a197230080087800503e2000c197230079
:10f3100080087800203e2000e197230080087800d4
:10f32000903d20000198230080087800e03c2000f8
:10f330002198230080087800803c20004198230019
:10f3400080087800203c2000619823008008780025
:10f35000703b20008198230080087800c03a20008c
:10f36000a198230080087800303a2000c19823003b
:10f370008008780090392000e19823008008780008
:10f38000203920000199230080087800c03820002f
:10f3900021992300800878005038200041992300eb
:10f3a0008008780050382000619923008008780098
:10f3b000903820008199230080087800d038200000
:10f3c000a199230080087800d0382000c19923003b
:10f3d0008008780030392000e19923008008780007
:10f3e00050392000019a23008008780070392000ed
:10f3f000219a230080087800a0392000419a230038
:10f4000080087800103a2000619a23008008780074
:10f41000c03a2000819a230080087800403b2000f9
:10f42000a19a230080087800303c2000c19a230074
:10f4300080087800b03d2000e19a23008008780021
:10f44000b03e2000019b230080087800a03f2000f0
:10f45000219b230080087800b0402000419b2300be
:10f460008008780080412000619b2300800878009c
:10f47000b0422000819b23008008780020442000b7
:10f48000a19b230080087800e0452000c19b230059
:10f4900080087800c0472000e19b230080087800a6
:10f4a000c0492000019c230080087800d04b200038
:10f4b000219c230080087800904d2000419c23006f
:10f4c00080087800904f2000619c2300800878001d
:10f4d000b0512000819c230080087800d053200088
:10f4e000a19c23008008780030562000c19c230096
:10f4f0008008780070572000e19c23008008780085
:10f50000005a2000019d230080087800b05c200094
:10f51000219d230080087800c05f2000419d2300ca
:10f5200080087800f0622000619d23008008780048
:10f53000b0652000819d230080087800c06820000d
:10f54000a19d230080087800b06b2000c19d23009e
:10f5500080087800b06d2000e19d230080087800cd
:10f56000e06e2000019e230080087800606f20007c
:10f57000219e230080087800206e2000419e2300f9
:10f5800080087800006b2000619e230080087800ce
:10f59000d0652000819e230080087800905e2000c6
:10f5a000a19e23008008780050552000c19e2300b2
:10f5b00080087800004a2000e19e2300800878003f
:10f5c000203d2000019f230080087800602f20004c
:10f5d000219f230080087800a0282000419f23005d
:10f5e00080087800501c2000619f2300800878006c
:10f5f00060112000819f230080087800d00820003f
:10f60000a19f23008008780060032000c19f230091
:10f610008008780080002000e19f230080087800a7
:10f620002000200001a02300800878006002200054
:10f6300021a02300800878006006200041a023005c
:10f6400080087800700b200061a0230080087800fb
:10f650009011200081a0230080087800d01820009d
:10f66000a1a0230080087800c01f2000c1a02300b3
:10f670008008780070262000e1a023008008780030
:10f68000102d200001a1230080087800d032200036
:10f6900021a12300800878007038200041a12300b8
:10f6a00080087800403d200061a123008008780098
:10f6b0006040200081a12300800878006041200084
:10f6c000a1a123008008780070432000c1a123007d
:10f6d0008008780030452000e1a1230080087800f0
:10f6e0005046200001a2230080087800c046200078
:10f6f00021a2230080087800f046200041a22300c8
:10f7000080087800c046200061a2230080087800ad
:10f71000c046200081a223008008780020472000f6
:10f72000a1a223008008780030472000c1a2230056
:10f730008008780020472000e1a22300800878009c
:10f74000a047200001a32300800878008047200004
:10f7500021a32300800878006047200041a32300f4
:10f76000800878006047200061a3230080087800ab
:10f770003047200081a3230080087800b046200095
:10f78000a1a3230080087800e0452000c1a3230046
:10f790008008780000452000e1a32300800878005d
:10f7a0007044200001a4230080087800404320001a
:10f7b00021a42300800878005042200041a42300a7
:10f7c000800878003041200061a423008008780080
:10f7d0006040200081a4230080087800e03f2000e2
:10f7e000a1a4230080087800b03f2000c1a423001a
:10f7f00080087800b03f2000e1a423008008780052
:10f80000c03f200001a52300800878005040200060
:10f8100021a5230080087800d040200041a52300c6
:10f82000800878004041200061a52300800878000e
:10f83000a041200081a5230080087800c04120005d
:10f84000a1a5230080087800f0412000c1a5230075
:10f8500080087800a0412000e1a5230080087800fe
:10f860006041200001a6230080087800d0402000dd
:10f8700021a62300800878000040200041a6230034
:10f8800080087800b03f200061a62300800878003f
:10f89000f03e200081a6230080087800503e200022
:10f8a000a1a6230080087800f03d2000c1a6230017
:10f8b00080087800d03d2000e1a623008008780071
:10f8c000d03d200001a7230080087800203e2000c2
:10f8d00021a7230080087800503e200041a7230084
:10f8e00080087800403e200061a72300800878004f
:10f8f000503e200081a7230080087800203e200091
:10f90000a1a7230080087800c03d2000c1a72300e4
:10f9100080087800803d2000e1a72300800878005f
:10f92000f03c200001a8230080087800803c2000e3
:10f9300021a8230080087800003c200041a8230073
:10f9400080087800c03b200061a823008008780070
:10f95000603b200081a8230080087800f03a200056
:10f96000a1a8230080087800a03a2000c1a82300a5
:10f9700080087800403a2000e1a823008008780041
:10f98000d039200001a923008008780070392000b8
:10f9900021a92300800878000039200041a9230014
:10f9a00080087800b038200061a923008008780022
:10f9b0009038200081a9230080087800803820003a
:10f9c000a1a9230080087800a0382000c1a9230045
:10f9d0008008780030392000e1a9230080087800f1
:10f9e0009039200001aa230080087800f039200017
:10f9f00021aa230080087800803a200041aa230031
:10fa000080087800703b200061aa230080087800fd
:10fa1000603c200081aa230080087800303d20004f
:10fa2000a1aa230080087800203e2000c1aa23005c
:10fa300080087800303f2000e1aa23008008780089
:10fa4000a03f200001ab230080087800f03f200099
:10fa500021ab23008008780000000600004520004c
:10fa600041ab230080087800c04d200061ab23002b
:10fa7000800878001056200081ab230080087800b1
:10fa8000605d2000a1ab230080087800d0642000d6
:10fa9000c1ab230080087800c06e2000e1ab2300da
:10faa000800878000073200001ac230080087800f3
:10fab0002075200021ac230080087800a07620006b
:10fac00041ac230080087800c078200061ac23009e
:10fad00080087800a076200081ac230080087800a0
:10fae000b0712000a1ac230080087800d06a20000b
:10faf000c1ac23008008780090612000e1ac2300b5
:10fb000080087800f052200001ad230080087800c2
:10fb10003049200021ad23008008780040402000bb
:10fb200041ad2300800878003039200061ad23000a
:10fb3000800878000033200081ad23008008780021
:10fb400020322000a1ad230080087800c0312000c1
:10fb5000c1ad23008008780070312000e1ad2300a2
:10fb600080087800a031200001ae230080087800d2
:10fb7000b030200021ae23008008780050302000f3
:10fb800041ae2300800878000030200061ae2300e1
:10fb900080087800502f200081ae23008008780074
:10fba000002d2000a1ae230080087800602a2000ec
:10fbb000c1ae23008008780060272000e1ae23005a
:10fbc000800878001025200001af2300800878000d
:10fbd0007023200021af230080087800302220000d
:10fbe00041af2300800878003021200061af23005e
:10fbf000800878001020200081af23008008780062
:10fc0000d01e2000a1af230080087800501e2000e5
:10fc1000c1af23008008780000202000e1af23005e
:10fc2000800878004023200001b02300800878007d
:10fc3000b027200021b0230080087800502d20003c
:10fc400041b02300800878003037200061b02300e5
:10fc500080087800003e200081b0230080087800f2
:10fc600070442000a1b0230080087800704a200072
:10fc7000c1b0230080087800b04f2000e1b023001d
:10fc800080087800e056200001b123008008780049
:10fc9000905b200021b123008008780010602000d4
:10fca00041b12300800878009063200061b12300f7
:10fcb000800878002066200081b123008008780049
:10fcc00080652000a1b123008008780090632000a7
:10fcd000c1b123008008780050602000e1b123000a
:10fce00080087800105c200001b2230080087800b2
:10fcf0008053200021b2230080087800104d20009e
:10fd000041b2230080087800a046200061b22300a1
:10fd100080087800d040200081b22300800878005d
:10fd200000392000a1b2230080087800d0342000e0
:10fd3000c1b223008008780070312000e1b22300b6
:10fd400080087800a02e200001b3230080087800ee
:10fd5000502c200021b3230080087800202b2000a5
:10fd600041b3230080087800e02b200061b323001a
:10fd700080087800402e200081b32300800878009e
:10fd800090312000a1b3230080087800f0362000d5
:10fd9000c1b3230080087800b0392000e1b323000c
:10fda00080087800903b200001b423008008780090
:10fdb000203d200021b4230080087800d03e2000a0
:10fdc00041b42300800878002041200061b4230062
:10fdd000800878002042200081b423008008780049
:10fde00000432000a1b42300800878008043200055
:10fdf000c1b423008008780040432000e1b4230010
:10fe000080087800f041200001b5230080087800c8
:10fe10004041200021b5230080087800f0402000f8
:10fe200041b52300800878001041200061b523000f
:10fe300080087800f041200081b523008008780018
:10fe400010432000a1b52300800878004044200022
:10fe5000c1b523008008780070452000e1b523007b
:10fe6000800878009046200001b6230080087800c2
:10fe7000b048200021b6230080087800004b200005
:10fe800041b6230080087800404d200061b6230071
:10fe900080087800e04e200081b6230080087800ba
:10fea00030502000a1b623008008780010502000b8
:10feb000c1b6230080087800804e2000e1b6230000
:10fec00080087800504c200001b72300800878009b
:10fed000e049200021b723008008780080452000f9
:10fee00041b72300800878001042200061b723004a
:10fef00080087800e03e200081b723008008780069
:10ff0000003c2000a1b7230080087800e0372000e3
:10ff1000c1b7230080087800d0352000e1b7230066
:10ff2000800878000034200001b8230080087800a1
:10ff3000a032200021b8230080087800e0312000a2
:10ff400041b82300800878008034200061b8230085
:10ff5000800878004039200081b8230080087800ac
:10ff6000403d2000a1b8230080087800b03f200069
:10ff7000c1b823008008780020412000e1b82300a8
:10ff800080087800f040200001b923008008780044
:10ff9000a040200021b9230080087800803f200085
:10ffa00041b9230080087800c03d200061b92300da
:10ffb000800878000039200081b92300800878008b
:10ffc000d0332000a1b9230080087800602e2000e3
:10ffd000c1b9230080087800b0292000e1b92300ce
:10ffe000800878001026200001ba230080087800dd
:10fff0000022200021ba230080087800a01f2000e2
:020000040001f9
:1000000041ba230080087800f01d200061ba230067
:1000100080087800a01d200081ba230080087800a5
:1000200000202000a1ba230080087800a02320002f
:10003000c1ba230080087800a0282000e1ba23007c
:1000400080087800a02e200001bb230080087800e3
:100050003035200021bb230080087800a04020001c
:1000600041bb230080087800b049200061bb230019
:1000700080087800c052200081bb230080087800ef
:10008000705b2000a1bb230080087800706720000f
:10009000c1bb230080087800206f2000e1bb230053
:1000a00080087800d074200001bc2300800878000c
:1000b0000079200021bc230080087800207d2000ea
:1000c00041bc230080087800a07f200061bc230091
:1000d00080087800107c200081bc23008008780014
:1000e00010762000a1bc230080087800d06d20008d
:1000f000c1bc230080087800305e2000e1bc2300f2
:10010000800878002053200001bd2300800878007b
:10011000f047200021bd230080087800b03d20007a
:1001200041bd2300800878008035200061bd230098
:1001300080087800702e200081bd230080087800a0
:10014000502d2000a1bd230080087800d02c200075
:10015000c1bd230080087800c02c2000e1bd230031
:1001600080087800a02c200001be230080087800c1
:10017000602c200021be230080087800502d200034
:1001800041be230080087800f02d200061be2300ce
:1001900080087800602e200081be2300800878004f
:1001a000d02d2000a1be230080087800f02b200075
:1001b000c1be230080087800a0292000e1be2300f2
:1001c00080087800a027200001bf23008008780065
:1001d0000026200021bf2300800878007024200022
:1001e00041bf2300800878005023200061bf230016
:1001f00080087800d021200081bf2300800878008b
:1002000050202000a1bf230080087800102020008b
:10021000c1bf23008008780060212000e1bf2300d7
:10022000800878000024200001c0230080087800a6
:10023000d027200021c0230080087800302d200026
:1002400041c02300800878001037200061c02300df
:1002500080087800b03d200081c02300800878002d
:1002600010442000a1c0230080087800304a2000fc
:10027000c1c023008008780090522000e1c0230014
:10028000800878008057200001c123008008780092
:10029000505c200021c1230080087800006120000c
:1002a00041c1230080087800d064200061c1230090
:1002b000800878003067200081c123008008780022
:1002c000a0662000a1c1230080087800f06420000f
:1002d000c1c1230080087800f0612000e1c1230043
:1002e00080087800805a200001c22300800878002e
:1002f0004054200021c2230080087800504d200087
:1003000041c2230080087800a046200061c223007b
:10031000800878006040200081c2230080087800b7
:1003200050382000a1c2230080087800e03320006c
:10033000c1c2230080087800e02f2000e1c2230022
:1003400080087800902c200001c3230080087800ea
:10035000202a200021c3230080087800e028200004
:1003600041c3230080087800e029200061c32300f6
:1003700080087800702c200081c32300800878005a
:1003800050302000a1c3230080087800d035200021
:10039000c1c3230080087800a0382000e1c32300f7
:1003a00080087800f03a200001c42300800878001b
:1003b000003d200021c4230080087800e03e20009a
:1003c00041c4230080087800e040200061c423007d
:1003d000800878000042200081c423008008780053
:1003e00010432000a1c4230080087800a04320000f
:1003f000c1c423008008780040432000e1c42300ea
:10040000800878008042200001c523008008780021
:10041000e041200021c523008008780090412000a1
:1004200041c52300800878009041200061c5230069
:1004300080087800e042200081c523008008780011
:1004400020442000a1c523008008780070452000ca
:10045000c1c5230080087800c0462000e1c5230004
:10046000800878006048200001c6230080087800da
:10047000d049200021c6230080087800904b20003e
:1004800041c6230080087800904d200061c62300fb
:1004900080087800204f200081c623008008780063
:1004a00040502000a1c6230080087800d04f2000d3
:1004b000c1c6230080087800704e2000e1c62300ea
:1004c00080087800704c200001c723008008780065
:1004d000e049200021c7230080087800f044200074
:1004e00041c7230080087800c041200061c7230075
:1004f00080087800c03e200081c723008008780073
:10050000a03b2000a1c7230080087800803720008e
:10051000c1c723008008780040352000e1c72300d0
:10052000800878005033200001c82300800878003c
:10053000e031200021c8230080087800d03120005d
:1005400041c8230080087800b036200061c823002d
:1005500080087800003b200081c8230080087800d4
:10056000b03d2000a1c8230080087800203f200073
:10057000c1c8230080087800a03f2000e1c8230004
:1005800080087800a03f200001c92300800878007f
:10059000103f200021c9230080087800803d200002
:1005a00041c9230080087800f03a200061c9230087
:1005b000800878002034200081c92300800878005a
:1005c000302f2000a1c9230080087800102b2000c4
:1005d000c1c923008008780020282000e1c9230039
:1005e00080087800c024200001ca23008008780019
:1005f000a022200021ca230080087800902020003b
:1006000041ca230080087800301f200061ca2300ff
:1006100080087800701f200081ca230080087800bd
:10062000d0222000a1ca230080087800d026200014
:10063000c1ca230080087800f02b2000e1ca230003
:1006400080087800f031200001cb2300800878007a
:10065000703c200021cb230080087800d04420008b
:1006600041cb230080087800a04d200061cb2300ff
:1006700080087800f055200081cb230080087800a6
:10068000a05d2000a1cb230080087800b069200085
:10069000c1cb23008008780040702000e1cb23000c
:1006a00080087800e074200001cc230080087800e6
:1006b0008078200021cc230080087800107c200066
:1006c00041cc230080087800807c200061cc23008e
:1006d00080087800c078200081cc23008008780052
:1006e00070722000a1cc230080087800b06920003f
:1006f000c1cc230080087800805a2000e1cc230080
:1007000080087800f04f200001cd23008008780099
:100710009045200021cd230080087800803c2000f7
:1007200041cd230080087800a035200061cd230052
:10073000800878002030200081cd230080087800d8
:10074000102f2000a1cd230080087800302e20003b
:10075000c1cd230080087800e02d2000e1cd2300ea
:1007600080087800e02d200001ce2300800878006a
:10077000602e200021ce230080087800102f20005a
:1007800041ce230080087800d02e200061ce2300c7
:1007900080087800402e200081ce23008008780059
:1007a000202c2000a1ce230080087800302a2000d1
:1007b000c1ce23008008780030282000e1ce23003d
:1007c000800878009026200001cf23008008780060
:1007d000a024200021cf230080087800902320004f
:1007e00041cf2300800878003022200061cf230011
:1007f00080087800a020200081cf230080087800a6
:10080000701f2000a1cf230080087800d01f200097
:10081000c1cf230080087800d0212000e1cf230041
:1008200080087800e024200001d0230080087800b0
:100830005029200021d0230080087800202f20009c
:1008400041d02300800878007039200061d0230057
:1008500080087800e03f200081d0230080087800e5
:10086000c0452000a1d0230080087800404b200024
:10087000c1d0230080087800a0522000e1d02300de
:10088000800878004057200001d1230080087800bc
:10089000e05b200021d123008008780090602000d8
:1008a00041d12300800878004064200061d12300fa
:1008b00080087800a066200081d12300800878009d
:1008c000f0652000a1d1230080087800d0632000cb
:1008d000c1d123008008780060602000e1d12300ae
:1008e000800878003059200001d223008008780069
:1008f0003053200021d2230080087800e04c2000f3
:1009000041d22300800878007046200061d2230085
:1009100080087800b040200081d223008008780051
:1009200090382000a1d2230080087800c033200036
:10093000c1d2230080087800d02f2000e1d223000c
:1009400080087800502c200001d323008008780014
:10095000d029200021d3230080087800d02920004e
:1009600041d3230080087800202b200061d323008e
:1009700080087800d02d200081d3230080087800e3
:1009800000312000a1d32300800878001036200019
:10099000c1d323008008780000392000e1d3230070
:1009a00080087800603b200001d423008008780094
:1009b000803d200021d423008008780030402000b2
:1009c00041d42300800878009041200061d42300a6
:1009d00080087800a042200081d42300800878009d
:1009e00050432000a1d4230080087800a0432000b9
:1009f000c1d423008008780020432000e1d42300e4
:100a0000800878007042200001d52300800878001b
:100a1000d041200021d523008008780070412000bb
:100a200041d5230080087800b041200061d5230023
:100a3000800878004043200081d52300800878009a
:100a400040442000a1d52300800878007045200094
:100a5000c1d5230080087800a0462000e1d52300fe
:100a6000800878008048200001d6230080087800a4
:100a7000004a200021d6230080087800004c200086
:100a800041d6230080087800e04d200061d6230085
:100a900080087800304f200081d62300800878003d
:100aa00000502000a1d6230080087800604f20006d
:100ab000c1d6230080087800d04d2000e1d6230065
:100ac00080087800904b200001d723008008780030
:100ad0005047200021d723008008780020442000c0
:100ae00041d7230080087800f040200061d7230020
:100af00080087800e03d200081d72300800878003e
:100b0000d03a2000a1d7230080087800b03620001a
:100b1000c1d7230080087800a0342000e1d723004b
:100b2000800878001033200001d823008008780066
:100b30008032200021d82300800878005036200021
:100b400041d8230080087800c03a200061d82300f3
:100b500080087800103e200081d8230080087800ab
:100b600010402000a1d8230080087800a040200079
:100b7000c1d8230080087800e03f2000e1d823009e
:100b800080087800203f200001d9230080087800e9
:100b9000e03d200021d9230080087800603b200040
:100ba00041d92300800878001037200061d9230044
:100bb00080087800f02e200081d92300800878007a
:100bc000302a2000a1d9230080087800c026200008
:100bd000c1d923008008780030242000e1d9230007
:100be00080087800a021200001da23008008780026
:100bf000f01f200021da230080087800a01e2000ca
:100c000041da230080087800f01e200061da23001a
:100c100080087800b020200081da23008008780066
:100c2000e0252000a1da230080087800502b200066
:100c3000c1da23008008780070312000e1da230057
:100c4000800878000038200001db2300800878004d
:100c5000b043200021db230080087800204c2000d6
:100c600041db2300800878008054200061db2300f2
:100c700080087800205c200081db23008008780059
:100c800000642000a1db230080087800206f200092
:100c9000c1db23008008780090732000e1db230093
:100ca000800878007075200001dc2300800878003f
:100cb0007076200021dc230080087800d0772000a7
:100cc00041dc2300800878001076200061dc2300de
:100cd00080087800b071200081dc23008008780053
:100ce000106b2000a1dc230080087800d061200078
:100cf000c1dc23008008780010532000e1dc2300d1
:100d000080087800d049200001dd230080087800a9
:100d10003041200021dd230080087800b03a200017
:100d200041dd230080087800c036200061dd23000b
:100d300080087800d035200081dd2300800878000d
:100d400050342000a1dd23008008780050332000bb
:100d5000c1dd230080087800b0322000e1dd2300ef
:100d600080087800c031200001de23008008780070
:100d70007030200021de230080087800202f200022
:100d800041de230080087800902d200061de2300e2
:100d900080087800502b200081de23008008780036
:100da000f0262000a1de23008008780030242000f7
:100db000c1de23008008780030222000e1de23001d
:100dc000800878006021200001df2300800878007f
:100dd000e01f200021df230080087800501e200043
:100de00041df230080087800101d200061df230010
:100df00080087800d01c200081df23008008780064
:100e0000f01d2000a1df230080087800a021200031
:100e1000c1df23008008780040252000e1df2300a7
:100e200080087800102a200001e023008008780064
:100e3000802f200021e023008008780080392000e6
:100e400041e0230080087800b040200061e02300ea
:100e5000800878009047200081e023008008780017
:100e6000504d2000a1e0230080087800905220001f
:100e7000c1e0230080087800d0592000e1e0230081
:100e800080087800b05d200001e123008008780030
:100e9000e060200021e1230080087800306320001a
:100ea00041e1230080087800a064200061e1230074
:100eb000800878005064200081e1230080087800d9
:100ec00080622000a1e1230080087800005f2000fc
:100ed000c1e1230080087800405a2000e1e12300ae
:100ee00080087800a051200001e2230080087800eb
:100ef000904b200021e2230080087800604520000c
:100f000041e2230080087800c03f200061e2230016
:100f100080087800e03a200081e223008008780011
:100f2000e0342000a1e22300800878008031200016
:100f3000c1e2230080087800a02e2000e1e2230017
:100f400080087800902c200001e3230080087800be
:100f5000e02b200021e3230080087800f02c200003
:100f600041e3230080087800502f200061e3230034
:100f700080087800a032200081e3230080087800f8
:100f8000f0352000a1e3230080087800f03920002c
:100f9000c1e3230080087800c03b2000e1e3230088
:100fa00080087800203d200001e4230080087800bc
:100fb000703e200021e4230080087800404020009b
:100fc00041e42300800878004041200061e42300d0
:100fd00080087800b041200081e423008008780078
:100fe000b0412000a1e42300800878008041200067
:100ff000c1e4230080087800b0402000e1e4230031
:10100000800878003040200001e523008008780047
:101010003040200021e5230080087800d0402000e7
:1010200041e5230080087800a042200061e523000c
:10103000800878001044200081e5230080087800b3
:1010400090452000a1e5230080087800f0462000ac
:10105000c1e523008008780070482000e1e5230006
:1010600080087800904a200001e62300800878007c
:10107000604c200021e6230080087800704e20009c
:1010800041e6230080087800f04f200061e623004d
:10109000800878006050200081e6230080087800f6
:1010a000a04f2000a1e6230080087800f04d20002a
:1010b000c1e6230080087800904b2000e1e6230081
:1010c000800878000049200001e7230080087800ac
:1010d0009044200021e72300800878001041200080
:1010e00041e7230080087800f03d200061e72300fd
:1010f00080087800303b200081e7230080087800da
:1011000060382000a1e723008008780030352000f7
:10111000c1e7230080087800b0332000e1e7230016
:1011200080087800d032200001e823008008780091
:101130002033200021e82300800878005038200068
:1011400041e8230080087800303d200061e823005a
:1011500080087800b040200081e8230080087800f3
:10116000b0422000a1e8230080087800104320004e
:10117000c1e823008008780010422000e1e8230045
:1011800080087800a040200001e923008008780052
:10119000a03e200021e9230080087800d03b2000f9
:1011a00041e92300800878000035200061e9230030
:1011b00080087800f02e200081e923008008780064
:1011c00080292000a1e92300800878006025200004
:1011d000c1e9230080087800c0222000e1e9230053
:1011e000800878006020200001ea23008008780051
:1011f000001f200021ea230080087800f01d200055
:1012000041ea230080087800001e200061ea2300e4
:10121000800878002021200081ea230080087800df
:10122000f0242000a1ea230080087800a02a2000f2
:10123000c1ea23008008780010312000e1ea230091
:10124000800878002038200001eb23008008780017
:10125000f03f200021eb230080087800000006000a
:10126000d03f200041eb230080087800f0422000ae
:1012700061eb2300800878005047200081eb2300b9
:1012800080087800b04b2000a1eb23008008780094
:1012900010512000c1eb2300800878002057200067
:1012a000e1eb230080087800605f200001ec230060
:1012b000800878006066200021ec23008008780018
:1012c000206f200041ec230080087800407520004a
:1012d00061ec230080087800a079200081ec2300d5
:1012e00080087800307c2000a1ec23008008780082
:1012f000107d2000c1ec230080087800a07b200036
:10130000e1ec230080087800b07b200001ed230091
:10131000800878006075200021ed230080087800a7
:10132000106d200041ed230080087800f05d200062
:1013300061ed2300800878003055200081ed230006
:1013400080087800e04e2000a1ed2300800878009e
:10135000c04a2000c1ed230080087800a049200089
:10136000e1ed230080087800504b200001ee2300bf
:1013700080087800904b200021ee23008008780040
:10138000404d200041ee230080087800f04c200002
:1013900061ee2300800878005046200081ee230093
:1013a00080087800303b2000a1ee23008008780000
:1013b000602f2000c1ee2300800878003023200039
:1013c000e1ee230080087800d018200001ef230010
:1013d00080087800f011200021ef230080087800b9
:1013e000b010200041ef2300800878002013200077
:1013f00061ef230080087800101b200081ef23009c
:101400008008780050222000a1ef23008008780097
:10141000c0282000c1ef230080087800a02d200004
:10142000e1ef230080087800e02f200001f0230086
:10143000800878005030200021f0230080087800d8
:10144000a02e200041f0230080087800e029200031
:1014500061f02300800878006027200081f02300dd
:101460008008780050252000a1f023008008780033
:1014700020242000c1f0230080087800a023200051
:10148000e1f02300800878004022200001f12300d1
:10149000800878001023200021f1230080087800c4
:1014a0005024200041f1230080087800d02520003e
:1014b00061f12300800878006028200081f123007a
:1014c00080087800c0292000a1f12300800878005e
:1014d000902b2000c1f1230080087800202e2000ee
:1014e000e1f1230080087800f031200001f22300b0
:1014f000800878000039200021f22300800878005d
:10150000603e200041f2230080087800f042200075
:1015100061f22300800878008046200081f22300d9
:1015200080087800a04a2000a1f2230080087800fb
:10153000c04c2000c1f2230080087800004f20003a
:10154000e1f22300800878007050200001f32300ae
:10155000800878004050200021f3230080087800a4
:10156000204d200041f3230080087800b04920007e
:1015700061f32300800878001046200081f32300e7
:1015800080087800f0432000a1f323008008780051
:1015900010412000c1f32300800878002040200083
:1015a000e1f3230080087800e03e200001f42300ee
:1015b00080087800c03c200021f4230080087800d7
:1015c000a039200041f42300800878004036200034
:1015d00061f4230080087800e033200081f42300c8
:1015e0008008780080312000a1f423008008780072
:1015f00060312000c1f423008008780070322000a0
:10160000e1f42300800878003035200001f5230044
:10161000800878009037200021f5230080087800aa
:10162000103a200041f5230080087800c03c2000db
:1016300061f5230080087800e03e200081f523005a
:101640008008780030412000a1f523008008780050
:10165000a0432000c1f523008008780080442000ca
:10166000e1f52300800878001045200001f62300f2
:10167000800878002044200021f6230080087800ac
:101680003044200041f623008008780050442000b8
:1016900061f62300800878005044200081f6230082
:1016a00080087800f0442000a1f62300800878002c
:1016b00050462000c1f6230080087800b047200083
:1016c000e1f6230080087800e048200001f72300bd
:1016d00080087800104a200021f723008008780055
:1016e000a04c200041f7230080087800404d2000e6
:1016f00061f7230080087800604d200081f7230007
:1017000080087800504d2000a1f723008008780061
:10171000d04d2000c1f7230080087800604c2000e5
:10172000e1f7230080087800804b200001f82300b7
:1017300080087800d049200021f823008008780034
:101740005046200041f8230080087800303e2000f9
:1017500061f82300800878000039200081f8230018
:1017600080087800f0342000a1f823008008780079
:10177000f0312000c1f8230080087800002f2000fd
:10178000e1f8230080087800f02c200001f9230004
:1017900080087800102b200021f9230080087800b1
:1017a0009029200041f9230080087800b02920000a
:1017b00061f9230080087800202f200081f92300a0
:1017c0008008780060322000a1f9230080087800aa
:1017d00010352000c1f92300800878002035200052
:1017e000e1f92300800878008035200001fa230009
:1017f00080087800f037200021fa23008008780064
:101800009039200041fa230080087800503b2000e6
:1018100061fa230080087800f03c200081fa230060
:1018200080087800203d2000a1fa2300800878007d
:10183000603d2000c1fa230080087800903d200020
:10184000e1fa2300800878000041200001fb23001a
:10185000800878009041200021fb23008008780058
:10186000b03f200041fb23008008780000432000a7
:1018700061fb230080087800b047200081fb230033
:1018800080087800904c2000a1fb2300800878009d
:1018900010502000c1fb2300800878004058200031
:1018a000e1fb2300800878003065200001fc230064
:1018b00080087800a06b200021fc230080087800bd
:1018c0003070200041fc2300800878006076200002
:1018d00061fc230080087800c07a200081fc23008e
:1018e00080087800807d2000a1fc2300800878001b
:1018f000307e2000c1fc230080087800f07f2000ab
:10190000e1fc2300800878008075200001fd2300a1
:1019100080087800006f200021fd230080087800f7
:10192000d067200041fd230080087800106020006f
:1019300061fd2300800878006058200081fd2300ad
:1019400080087800b0502000a1fd230080087800b6
:10195000e04b2000c1fd230080087800e049200012
:10196000e1fd230080087800504b200001fe230099
:1019700080087800904e200021fe23008008780027
:10198000f04d200041fe230080087800504a2000de
:1019900061fe2300800878003042200081fe230091
:1019a0008008780010362000a1fe2300800878000f
:1019b000902a2000c1fe230080087800f01e20003d
:1019c000e1fe2300800878007015200001ff23004d
:1019d00080087800c00c200021ff230080087800d8
:1019e000500d200041ff23008008780000112000e6
:1019f00061ff230080087800a018200081ff2300e9
:101a000080087800a0212000a1ff23008008780032
:101a1000502a2000c1ff230080087800d02f20002a
:101a2000e1ff230080087800a0322000010024009c
:101a300080087800e032200021002400800878002f
:101a4000f03120004100240080087800902d200013
:101a50006100240080087800002b20008100240011
:101a60008008780010292000a10024008008780058
:101a7000b0272000c100240080087800f024200056
:101a8000e1002400800878000024200001012400e7
:101a9000800878008023200021012400800878003d
:101aa000702520004101240080087800c025200016
:101ab0006101240080087800b02620008101240004
:101ac00080087800d0272000a10124008008780039
:101ad00040292000c101240080087800c02b20008c
:101ae000e101240080087800503220000102240027
:101af00080087800e0372000210224008008780068
:101b0000003e20004102240080087800e0422000ce
:101b10006102240080087800204720008102240010
:101b200080087800c04b2000a102240080087800c3
:101b3000404e2000c1022400800878007050200030
:101b4000e102240080087800705120000103240085
:101b500080087800205120002103240080087800ac
:101b6000204e20004103240080087800e04a200035
:101b7000610324008008780080472000810324004e
:101b800080087800f0442000a10324008008780039
:101b900030412000c103240080087800404020002c
:101ba000e103240080087800d03e200001042400d6
:101bb00080087800d03b20002104240080087800b1
:101bc000003820004104240080087800c032200042
:101bd0006104240080087800403020008104240043
:101be00080087800402f2000a1042400800878009d
:101bf000602f2000c104240080087800f03120000c
:101c0000e104240080087800e0332000010524006e
:101c100080087800503620002105240080087800d4
:101c2000503920004105240080087800303e200013
:101c300061052400800878005041200081052400bf
:101c40008008780080432000a105240080087800e7
:101c500020452000c105240080087800504620005f
:101c6000e105240080087800404620000106240099
:101c700080087800f04520002106240080087800c4
:101c8000904520004106240080087800704520001f
:101c90006106240080087800704520008106240039
:101ca0008008780010452000a106240080087800f4
:101cb000d0452000c106240080087800e0462000be
:101cc000e106240080087800d047200001072400a6
:101cd00080087800c0482000210724008008780090
:101ce000504b20004107240080087800504c200011
:101cf0006107240080087800c04b20008107240081
:101d000080087800f04b2000a107240080087800ac
